:020000040800F2
:20000000F0FF0120F98B0608F5F1000855D30408718C0608718C0608718C060800000000FB
:20002000000000000000000000000000F1F10008EDF1000800000000E9F10008ED9604087F
:20004000718C0608718C0608718C0608718C0608718C0608718C060859E4040885E504089F
:2000600049E504080DE50408D1E40408B5700608A57006089570060885700608717006082C
:200080005D70060849700608718C06080000000000000000000000000000000095E404082E
:2000A000D981040825820408C9810408498204081982040809820408F9810408997A060815
:2000C000A17A06088D7A0608957A0608718C0608718C0608C99804080D9804080000000091
:2000E0001DE40408718C06083D0901080000000000000000000000000000000035700608E6
:2001000000000000753D0608E9810408718C0608000000000000000000000000000000009E
:20012000217006080D700608F96F0608E56F0608D16F06080000000000000000000000006F
:200140000000000000000000000000007DEB0008BD6F0608A96F0608956F060851970408C9
:20016000817A0608897A060800000000000000000000000000000000000000000000000065
:2001800000000000718C06080000000000000000718C0608718C0608988706000100000018
:2001A0000E02010002000000DC6600203C67002000000000E00900081402010005000000FA
:2001C0007C3E00204067002000000000E209000813020100040000009424002048670020CA
:2001E00000000000E80900080D1001004C0000005C6400204C6700200000000045F90308A0
:2002000004000800800000009C630020986700200000000000000000090201000100000007
:20022000446300201868002000000000EC090008FD01010024000000E86200201C68002029
:2002400000000000EF620408FB0101000100000028610020406800200000000045820508FE
:20026000FC01010009000000F45F002044680020000000004D820508F7010100060000005D
:20028000E85F00205068002000000000EE090008F901010004000000E45F002058680020DE
:2002A0000000000099630408160215003F0000001C3200205C680020000000006D8205087C
:2002C0003400010010000000D85E00209C6800200000000049980208110201000800000058
:2002E000B05E0020AC68002000000000F40900081212010004000000A85E0020B46800200C
:2003000000000000FC0900081820010032000000745E0020B868002000000000158B050886
:200320001220010011000000945D0020EC68002000000000000A0008000201000B000000D4
:20034000D05A0020006900200000000091820508FF11010006000000785A00200C6900200C
:200360000000000025820508081203000F000000845A0020146900200000000099820508DA
:20038000FA01010003000000705400202469002000000000658205080A8001002800000026
:2003A000504C00202869002000000000A9150208061001001C00000040310020506900206B
:2003C00000000000158305080202010003000000802800206C6900200000000000000000B3
:2003E0000C0201000400000060280020706900200000000035820508110001000C00000067
:20040000A6400020746900200000000055F50308FE01010014000000AC3F0020806900205C
:2004200000000000E9810508F581010068000000DCBC0020A8C1002000000000B9930108D0
:2004400023200100100000005CBD002010C2002000000000BD160208FD07010076000000C5
:2004600030C1002020C2002000000000057C0108261001000E000000A8C2002098C2002096
:2004800000000000B51B01080B3001001A00000004BA0020E8C2002000000000140A00085F
:2004A0001F3001002400000024B9002004C3002000000000300A0008050201000400000096
:2004C00034BC002028C3002000000000540A0008030101000A00000068B900202CC300203C
:2004E0000000000055160108220201001C0100004CDA0020C4DC002000000000CD8A0508DC
:200500000C200600CC000000ACD80020E0DD002000000000BDF30308010201000B00000092
:2005200050D80020ACDE002000000000818205081B0201001000000024D80020B8DE0020B9
:2005400000000000018305081B1001000C000000C4C40020C8DE0020000000007582010864
:2005600021020100F000000044C30020D4DE002000000000159A0108231201001000000070
:2005800084D90020C4DF002000000000580A0008371001002E00000094D70020D4DF0020DD
:2005A00000000000680A0008161001000600000034D5002004E0002000000000960A0008BF
:2005C0002F1001002200000070DC00200CE00020000000009C0A00081E000100090000006B
:2005E000B8D4002030E0002000000000BE0A0008051001000600000004D500203CE00020FE
:2006000000000000C80A0008F62101000C00000050EC00208CEE002000000000D00A000804
:200620001C0202001C000000F4EB0020DCEE0020000000003D8C050828200100180000005E
:2006400010EC0020F8EE002000000000D53C02080412010002000000C8ED002010EF002050
:2006600000000000DC0A00080F02010001000000C4ED002014EF002000000000DE0A000895
:200680001400010004000000ECEB002018EF002000000000E00A0008012001000C00000003
:2006A00020E300201CEF002000000000E40A00080EF003009E01000008E1002028EF002016
:2006C000000000009198020813000100040000003CE80020C8F0002000000000F00A0008B1
:2006E000010101000400000054E00020CCF0002000000000000000000001010004000000BD
:200700004CE00020D0F0002000000000F40A0008020101000300000048E00020D4F0002074
:2007200000000000F9F30308190001000500000078FD0020D8FE002000000000F80A00080E
:200740001A0001000E000000D8FC0020E0FE002000000000FE0A0008203201000A00000011
:2007600070FB0020F0FE0020000000006D98020815001000700000004CF50020FCFE0020C1
:2007800000000000000000002A00080060000000C0FD00206CFF002000000000219802089C
:2007A0002C00040010000000DCFF0020CCFF002000000000099502082B001200240000000A
:2007C00010000120ECFF002000000000DD9402082920140078000000ECF20020340001203A
:2007E0000000000000000000190201001000000090F20020AC00012000000000718205085E
:200800000300010001000000381A0120242201200000000000000000031201003D000000A6
:20082000E019012028220120000000000C0B000825201E002C01000044170120682201205D
:2008400000000000000000001010010002000000C416012094230120000000004A0B000845
:20086000F8210100060000002017012098230120000000004C0B0008020001000C000000B6
:200880008C2501202026012000000000000000002902010040000000D42401202C26012027
:2008A00000000000520B00080A02010014000000C42301208C2601200000000089F3030850
:2008C0002802040004000000E42F0120C031012000000000FD8205082702040004000000E3
:2008E000E02F0120C431012000000000F18205081F020800100000003C2D0120C831012055
:2009000000000000018205081A0201003C000000E4280120D831012000000000C18B05083E
:200920003810010001000000C02601201432012000000000920B000827000100040000002E
:20094000DC320120E432012000000000940B00080B1201003C0000009C340120484701208F
:2009600000000000980B00080D12010014000000504101208447012000000000D40B000813
:200980000702010002000000304701209847012000000000E80B00081D0202000600000091
:2009A0000C4701209C4701200000000000000000060203000C00000018470120244C012097
:2009C00000000000858B0508100201000100000000800120FC7F012000000000EA0B0008AC
:2009E0000000000000FF00000000010000000000010000000000000001010101FFFFFFFFF6
:200A00000000000100010553343131000000000200000000AE014A015E012C0164000200F8
:200A2000000001000A019A01001E0A000002000000000000000100000005000001020300D9
:200A400000000000000000000000000000000000008007000000000000000000000000000F
:200A6000000000000000000020003200C800D00796001400320028004C0440060005500096
:200A800014000F00080064000100010005000A000000F4019600C409000019000000000045
:200AA000000000000000000000000000000000000000000000000000000000000000000531
:200AC0000100000000000000200003010000000000000000010000000202000000000000EC
:200AE00003000023E8036400040A000114001E0000204030900100000000280100007E0573
:200B0000EA05B4053200E803D0070000000000000000000000000000000000000000000039
:200B20000000000000000000000000000000000000000000000000000000000000000000B5
:200B40000000000000000000010000050201F4011400000000000000000000000000000083
:200B6000000000000000000000000000000000000000000000000000000000000000000075
:200B8000000000000000000000000000000000000000000020030000000000000000000032
:200BA000000000000000000000000000000000000000000000000000000000000000000035
:200BC000000000000000000000000000000000000100000000000000000000000000000014
:200BE0000000000000000000003C000403090412010002EF02014083045632000201020347
:200C00000100001201000202020040830440570002010203010800FFFFFFFF00600240109D
:200C20006002400000000000000000000B000000000000000000000000000000600240283D
:200C40006002400100000000000000060C00000000000000000000000000000060024040FD
:200C60006002400200000000000000100D00000000000000000000000000000060024058B9
:200C80006002400300000000000000160E0000000000000000000000000000006002407079
:200CA0006002400400000000000000200F0000000000000000000000000000006002408835
:200CC00060024005000000000000002610000000000000000000000000000000600240A0F5
:200CE00060024006000000000000003011000000000000000000000000000000600240B8B1
:200D00006002400700000000000000362F000000000000000000000000000000640240100F
:200D2000640240000000000000000000380000000000000000000000000000006402402807
:200D40006402400100000000000000063900000000000000000000000000000064024040C7
:200D60006402400200000000000000103A0000000000000000000000000000006402405883
:200D80006402400300000000000000163B0000000000000000000000000000006402407043
:200DA0006402400400000000000000203C00000000000000000000000000000064024088FF
:200DC00064024005000000000000002644000000000000000000000000000000640240A0B8
:200DE00064024006000000000000003045000000000000000000000000000000640240B874
:200E00006402400700000000000000364600000000000000000000000000007D000000012B
:200E200000000015830008118300080D83000801830008FD820008098300080583000800A7
:200E400000000035910008CDAD0008AD9000080DAF00080D92000885830008718300085531
:200E60008300082DA70008498A000839940008AD9400082D950008E5960008310F01085D1F
:200E80008300084D830008010000000000803FF5370108F93C010871380108CD0F0108B174
:200EA000110108DD0F0108F90F0108A50F0108950F0108000000000000000009022000017C
:200EC0000104C0320904000002080650050705810240000007050102400000090264000319
:200EE0000100C0320904000001030000000921110100012236000705830309000A080B01A0
:200F00000202020100090401000102020100052400100105240100020424020205240601F4
:200F200002070582030800FF09040200020A000000070501024000000705810240000009D5
:200F4000024300020100C032090400000102020100052400100105240100010424020205AE
:200F600024060001070582030800FF09040100020A00000007050102400000070581024076
:200F8000000000FF00000000FF0000000000000000AA550701000001AA55050100000898A6
:200FA000CE0608FF1FFF1F05010905A101A10005010930093109320933093509340936090F
:200FC000371581257F75089508810205091901290815002501950875018102C0C000000950
:200FE000022200010100E03209040000010301020009211101000122360007058303090075
:201000000A0000000000000102030401020304060708092D202D2D202D2D2D2D202D2D2D72
:201020002D0000000000000000000000000000000000AA550B010000AA5505010000AA5574
:201040000902000000AA5503009F0001000000C0127EFFE0C2002000000000B8C200200038
:2010600000000001000000F07307086C7307080000000081F40308A0860100040000000064
:20108000000000000000000000000000000000000000000000000000000000000000000050
:2010A00000000000000000F0730708F87307080000000031770408E80300000400000000A1
:2010C000000000000000000000000000000000000000000000000000000000000000000010
:2010E000000000000000000074070800000000000000006D6203087D000000FF0000000017
:201100000000000000000000000000000000000000000000000000000000000000000000CF
:201120000000000000000018F807080000000000000000C57403087D000000FF00000000D0
:2011400000000000000000000000000000000000000000000000000000000000000000008F
:2011600000000000000000608807080000000000000000F5BC03087D000000FF0000000040
:2011800000000000000000000000000000000000000000000000000000000000000000004F
:2011A00000000000000000087407080000000000000000616D0408E80300000300000000DC
:2011C00000000000000000000000000000000000000000000000000000000000000000000F
:2011E000000000000000000C74070800000000000000000D250308102700000300000000E9
:201200000000000000000000000000000000000000000000000000000000000000000000CE
:20122000000000000000002CF40708000000001592020809D404085F76000005000000000B
:2012400000000000000000000000000000000000000000000000000000000000000000008E
:2012600000000000000000BCF7070800000000000000006DF3040810270000010000000008
:2012800000000000000000000000000000000000000000000000000000000000000000004E
:2012A00000000000000000187407080000000000000000C15F0408E8030000050000000077
:2012C00000000000000000000000000000000000000000000000000000000000000000000E
:2012E00000000000000000247407080000000000000000B1F70308204E0000030000000023
:201300000000000000000000000000000000000000000000000000000000000000000000CD
:2013200000000000000000347407080000000000000000ADF50308204E00000300000000D8
:2013400000000000000000000000000000000000000000000000000000000000000000008D
:201360000000000000000044740708000000000000000075730408400D030003000000005F
:2013800000000000000000000000000000000000000000000000000000000000000000004D
:2013A000000000000000005474070800000000000000004D2804081027000001000000009D
:2013C00000000000000000000000000000000000000000000000000000000000000000000D
:2013E00000000000000000987307080000000000000000ADA601081027000003000000003D
:201400000000000000000000000000000000000000000000000000000000000000000000CC
:20142000000000000000005C74070800000000000000008D6F0208A086010001000000009F
:2014400000000000000000000000000000000000000000000000000000000000000000008C
:2014600000000000000000647407080000000000000000E96B040850C30000010000000011
:2014800000000000000000000000000000000000000000000000000000000000000000004C
:2014A000000000000000006C7407080000000000000000B9690408A08601000000000000E8
:2014C00000000000000000000000000000000000000000000000000000000000000000000C
:2014E00000000000000000787407080000000000000000A1650408A86100000100000000D5
:201500000000000000000000000000000000000000000000000000000000000000000000CB
:2015200000000000000000847407080000000000000000D1080208A0860100010000000099
:2015400000000000000000000000000000000000000000000000000000000000000000008B
:2015600000000000000000907407080000000000000000099E0408A00F00000100000000F5
:2015800000000000000000000000000000000000000000000000000000000000000000004B
:2015A000000000000000009C7407080000000000000000D1030208102700000100000000F6
:2015C00000000000000000000000000000000000000000000000000000000000000000000B
:2015E00000000000000000A87407080000000000000000B9F40308A00F0000010000000058
:201600000000000000000000000000000000000000000000000000000000000000000000CA
:2016200000000000000000B4740708000000000000000079DD01081A4100000100000000B8
:2016400000000000000000000000000000000000000000000000000000000000000000008A
:2016600000000000000000B87407080000000000000000891601081027000001000000004F
:2016800000000000000000000000000000000000000000000000000000000000000000004A
:2016A00000000000000000807307080000000000000000A94A020850C30000010000000017
:2016C00000000000000000000000000000000000000000000000000000000000000000000A
:2016E00000000000000000C47407080000000000000000591F0108400D03000000000000D2
:201700000000000000000000000000000000000000000000000000000000000000000000C9
:2017200000000000000000CC740708000000000000000075F50308400D0300000000000095
:20174000000000000000000000000000000000000000000000000000000000000000000089
:2017600000000000000000D47407080000000000000000B9EB010850C3000003000000004F
:20178000000000000000000000000000000000000000000000000000000000000000000049
:2017A00000000000000000E074070800000000000000002505040840420F000000000000FF
:2017C000000000000000000000000000000000000000000000000000000000000000000009
:2017E00000000000000000EC740708000000000000000071FC030850C300000000000000EF
:201800000000000000000000000000000000000000000000000000000000000000000000C8
:20182000000000000000000100000000000100E0010000FFFFFFFF01010000B58801080081
:2018400000000000000000BCD00608FFFFFFFF0800000042570200000001064257020000AD
:2018600000010601FF0101FF000000FFFFFFFF01FA0108000000000000000030D906081138
:201880003302080000000000000000E8D806082D202D2D202D2D2D2D202D2D2D000000001B
:2018A000000000000000000000000000000000000000000000000000000000A4D80608E0BE
:2018C000BB00209CFF2C0100000000FCDB0020E0150C170000000078D9002002000000DC07
:2018E000D80608ACD4002088136F1701000000AED4002088136F17000000005A660020009D
:201900000000000000000058660020000000000000000056660020000000000000000054B9
:20192000660020000000000000000052660020000000000000000050660020000000000073
:20194000000000FC050020000000000000000034D4002003000000CCD90608A4D400208868
:20196000136F17010000002ABC002088136F17000000006D8901080000000000000000DCCB
:20198000D9060879D900200100000030DA06082CBC0020010000003CDA060822BC002002A8
:2019A00000000044DA060800000000000000000000000050DA0608558901080000000000DC
:2019C000000000ECDA060800000000000000000000000040DB06080000000000000000000A
:2019E000000000B0DB0608B0D4002002000000E8DB060826BC0020E0150C1700000000C8F5
:201A0000E400201CE50020D6010000000000000000000000000000ECF106080000000000DF
:201A200000000000000000A4F2060800000000000000000000000050F206080000000000B2
:201A40000000000532020801E80020FF000000FFFFFFFF9535020800000000000000007CF1
:201A6000F1060801000000FA00000001000000010000000101000000010101000000001A4B
:201A8000E300200000F4010100000018E300200000F4010100000016E300200000F401012D
:201AA00000000014E300200000F4010100000012E300200000F4010100000010E3002000FB
:201AC00000F401010000000EE300200000F40101000000F9130208BD13020800000000FC1D
:201AE000DD0608FEE20020053201000CE300206400F401010000000AE300206400C409011B
:201B0000000000FCE20020E803D00701000000FAE20020E803D00701000000F8E20020E863
:201B200003D00701000000F6E200201E00B80B0100000004E3002005000F000100000006CE
:201B4000E3002003000A0001000000F4E200201E00F4010100000008E300200200000088D5
:201B6000DE0608F2E20020140064000100000000E300203200E80301000000F0E2002000F9
:201B800000C80001000000C9E2002000C80100C8E2002000500100C7E20020005A0100C5E4
:201BA000E200200200000094DE0608B47F0708BC7F0708166600200100C409000000001497
:201BC0006600200100C40900000000126600200100C40900000000106600200100C40900E7
:201BE0000000000C6600200100C409000000000E6600200100C409000000000A6600200192
:201C000000C40900000000086600200100C4090000000073E0002000C8010072E0002000ED
:201C2000C8010070E000200000FFFF0A0000006EE000200100C800010000006CE00020328D
:201C4000003075320000006AE000207EFF14000500000068E0002005002C010500000066A8
:201C6000E00020055A050063E0002000FF010065E00020020000005811002061E000200349
:201C8000000000B0D5060862E0002000FF010064E00020020000005811002060E0002003FD
:201CA000000000B0D506084D130208DD12020800000000A0DE060830E30020EE02CA0801AC
:201CC0000000002EE3002000C80100640000002DE3002000C80100640000002CE300200218
:201CE000000000ACDF06085AE000200000803E0500000058E0002080C1803E050000005280
:201D0000E000200083007D0500000050E0002080C1803E050000004BE0002000FF010046D9
:201D2000E000206400F4010100000045E0002004000000B8DF060844E0002002000000CC49
:201D4000DF0608F9E000200D000000D8DF0608F6E0002000640100F4E00020320010270A09
:201D6000000000F2E000200D000000D8DF0608F1E000200D000000D8DF0608F0E0002002EA
:201D800000000010E006080000000000000000000000001CE0060836E300203E0000005470
:201DA000E0060834E300200100FF7F0100000033E300200200000050E10608FBE000200309
:201DC00000000060E10608FAE000200300000060E10608B6E20020000A0100B4E2002000EF
:201DE00000E80301000000B2E200200000E80301000000B0E200200000E80301000000AE0B
:201E0000E200200000E80301000000A6E200200000E80301000000ACE200200000E80301A6
:201E2000000000AAE200200000E80301000000A8E2002000140100C4E20020020000007013
:201E4000E10608C2E200200000F40101000000C0E200200000F40101000000BEE200200061
:201E600000F40101000000BCE200200000F40101000000BAE200200000A00F01000000B894
:201E8000E200200000A00F01000000DDE2002019640100DCE20020020000007CE10608DA0E
:201EA000E20020E803D0070A000000D8E20020006401000A000000CDE2002000640100CC0B
:201EC000E2002000640100D4E20020006401000A000000D3E20020006401000A000000D240
:201EE000E20020006401000A000000D7E2002000FF01000A000000D6E2002000FF01000AAC
:201F0000000000D5E2002000FF01000A000000D1E2002001FF01000A000000D0E20020012F
:201F2000FF01000A000000CFE2002001FF01000A00000004E100200000F4010100000002BE
:201F4000E100200000A00F0100000000E100200000A00F01000000FEE000200000A00F0171
:201F6000000000FCE000200000A00F0100000051E8002000C8010050E80020006401004F87
:201F8000E80020006401004EE80020006401004DE80020006401004CE80020FF0801004BB8
:201FA000E800200164010045120208091202080000000088E1060854E800200132010053D3
:201FC000E8002001000000F8E1060852E800200400000000E206084AE800200064010048C4
:201FE000E800201400E8030100000046E80020E80330750A00000044E8002000C801004399
:020000040800F2
:20200000E8002000C8010042E8002000C8010041E800200032010056E80020004B01005561
:20202000E800200400000014E2060840E80020006401000A00000064E800200000D0070195
:202040000000005FE8002000C801005EE8002000C801005DE8002000C8010062E800200089
:2020600000D007010000005CE8002000C801005BE8002000C801005AE8002000C8010060A4
:20208000E800200000D0070100000059E8002000C8010058E8002000C8010057E8002000AE
:2020A000C80100FD0F0208E50F02080000000028E20608EDE00020005A0100ECE0002000F7
:2020C000C80100EAE00020E803D00701000000000000000000000045320208C4E206085302
:2020E000544D3332463431310000005FE00020000301005EE0002000030100290F0208E512
:202100000E02080000000018E30608AD0E02086D0E020800000000B4E306086D0F020879B0
:202120003502080000000034E406085CE0002001030100D5140208A9140208000000008C93
:20214000E70608150E0208E50D020800000000FCE706080D100208CD3602080000000098A4
:20216000E80608953A0208011502080000000040E906085D1002080000000000000000CCF6
:20218000E9060839110208E11002080000000030EA0608CD1102089111020800000000D865
:2021A000EA0608DD8B0208811202080000000064EB0608EFE2002001060100A51002087192
:2021C0001002080000000060EC0608118B02089937020800000000D0EC0608258C02086125
:2021E0003802080000000020EE0608EEE2002001030100B50F0208850F020800000000F42C
:20220000EE06087D8C0208000000000000000058EF0608450E02086135020800000000D885
:20222000EF060800000000000000000000000064F00608B5120208D938020800000000D47F
:20224000F0060801010000BC000120FFFFFFFF0000803F00000000000000000000000000E6
:2022600000000000000000000000000000000000000000000000000000803F00000000009F
:20228000000000000000000000803F0000000000000000000000000000803F0000000000C0
:2022A00000000000000000010000000000FA430000FA430000803F5D2A0408000000000051
:2022C00000000000000000FFFFFFFFFF000000000000007C26012008000000000000006CCC
:2022E00026012008000000200000004D370108C1100108E536010800000000910F0108CD6E
:202300003F010835360108813201080000000000000000510F01082583000819830008394F
:20232000900008559000081D90000801900008E58F0008053701089D1001083936010800DB
:20234000000000690F01088532010809360108E131010800000000000000005D0F010868FC
:202360005E0C00FFFFFFFF02010000A00F0000B80B000002FFFF01FFFF000020F407080060
:20238000000802050303000000000028F40708010008020504030000000000FC9B0708023E
:2023A00000FE0101100300000000001083070803001402000300000000000030F407080415
:2023C000001F02020008000000000038F4070805001F020201080000000000FFFFFFFF1A50
:2023E0000300000000000000000000000000000000000000000000000000000403090412B4
:2024000001000200000040830420570002010203010B01B5930508899305082D930508C952
:2024200083050849930508ED920508C5830508DC1A0020A9940508C994050899940508A995
:20244000830508559405080D94050899830508B81A0020C98C0508B1830508AD830508A5A8
:20246000830508118E0508A18305089D83050870450708693F01087D100108493E01080027
:2024800000000000000000E1350108F1340108000000000000000000000000450F01085141
:2024A000840508458405081995050835950508FD830508FD940508E1940508FFFFFFFF0179
:2024C00000000050C30000010100001F0000001C0000001F0000001E0000001F0000001E32
:2024E0000000001F0000001F0000001E0000001F0000001E0000001F0000000068214C014E
:20250000250000B4420708104F0708008002021F00000053544D202020202050726F6475E2
:202520007420202020202020202020302E3031008002021F00000053544D202020202050A1
:20254000726F64757420202020202020202020302E3031FF010000F4010000FF2A00000030
:2025600000040100000000000000021000000007000000000000000000000001020304062D
:2025800007080901000000381B0020000000000000000000000000000000000000000000AF
:2025A00000000000000000000000000000000000000000000000000000000000000000001B
:2025C0000000000000000000000000000000000000000000000000000000000000000000FB
:2025E0000000000000000000000000FFFFFFFFFFFFFFFFFFFFFFFFFFFFFFFFFFFFFFFFFFF0
:20260000FFFFFFFFFFFFFFFFFFFFFFFFFFFFFFFFFFFFFFFFFFFFFFFFFFFFFFFFFFFFFFFFDA
:20262000FFFFFFFFFFFFFFFFFFFFFFFFFFFFFFFFFFFFFFFFFFFFFFFFFFFFFFFFFFFFFFFFBA
:20264000FFFFFFFFFFFFFFFFFFFFFFFFFFFFFFFFFFFFFFFFFFFFFFFFFFFFFFFFFFFFFFFF9A
:20266000FFFFFFFFFFFFFFFFFFFFFFFFFFFFFFFFFFFFFFFFFFFFFFFFFFFFFFFFFFFFFFFF7A
:20268000FFFFFFFFFFFFFFFFFFFFFFFFFFFFFFFFFFFFFFFFFFFFFFFFFFFFFFFFFFFFFFFF5A
:2026A000FFFFFFFFFFFFFFFFFFFFFFFFFFFFFFFFFFFFFFFFFFFFFFFFFFFFFFFFFFFFFFFF3A
:2026C000FFFFFFFFFFFFFFFFFFFFFFFFFFFFFFFFFFFFFFFFFFFFFFFFFFFFFFFFFFFFFFFF1A
:2026E000FFFFFFFFFFFFFFFFFFFFFFFFFFFFFFFFFFFFFFFFFFFFFFFFFFFFFFFFFFFFFFFFFA
:20270000FFFFFFFFFFFFFFFFFFFFFFFFFFFFFFFFFFFFFFFFFFFFFFFFFFFFFFFFFFFFFFFFD9
:20272000FFFFFFFFFFFFFFFFFFFFFFFFFFFFFFFFFFFFFFFFFFFFFFFFFFFFFFFFFFFFFFFFB9
:20274000FFFFFFFFFFFFFFFFFFFFFFFFFFFFFFFFFFFFFFFFFFFFFFFFFFFFFFFFFFFFFFFF99
:20276000FFFFFFFFFFFFFFFFFFFFFFFFFFFFFFFFFFFFFFFFFFFFFFFFFFFFFFFFFFFFFFFF79
:20278000FFFFFFFFFFFFFFFFFFFFFFFFFFFFFFFFFFFFFFFFFFFFFFFFFFFFFFFFFFFFFFFF59
:2027A000FFFFFFFFFFFFFFFFFFFFFFFFFFFFFFFFFFFFFFFFFFFFFFFFFFFFFFFFFFFFFFFF39
:2027C000FFFFFFFFFFFFFFFFFFFFFFFFFFFFFFFFFFFFFFFFFFFFFFFFFFFFFFFFFFFFFFFF19
:2027E000FFFFFFFFFFFFFFFFFFFFFFFFFFFFFFFFFFFFFFFFFFFFFFFFFFFFFFFFFFFFFFFFF9
:202800000828000800400008FFFFFFFFFFFFFFFFFFFFFFFFFFFFFFFFFFFFFFFFFFFFFFFF50
:20282000FFFFFFFFFFFFFFFFFFFFFFFFFFFFFFFFFFFFFFFFFFFFFFFFFFFFFFFFFFFFFFFFB8
:20284000FFFFFFFFFFFFFFFFFFFFFFFFFFFFFFFFFFFFFFFFFFFFFFFFFFFFFFFFFFFFFFFF98
:20286000FFFFFFFFFFFFFFFFFFFFFFFFFFFFFFFFFFFFFFFFFFFFFFFFFFFFFFFFFFFFFFFF78
:20288000FFFFFFFFFFFFFFFFFFFFFFFFFFFFFFFFFFFFFFFFFFFFFFFFFFFFFFFFFFFFFFFF58
:020000040800F2
:20400000ADBE08000E02000000000B0014020000000000FF000A001302000000000100528B
:20402000000D00010001000000140504050000000000000000000504050000000000080039
:20404000000105040500000000000000000505040500000000000000001E05040500000012
:2040600000000000001F0504050000000064005200860004000000000000000000000000D3
:20408000000000000000000000000000000000000000000000000000000000000000000020
:2040A000000000000000000000000000000000000000000000000000000000000000000000
:2040C0000000000000000000000000000000000000000000000000000000000000000000E0
:2040E0000000000000000000000000000000000000000000000000070009020000002A0084
:20410000FD0100001912000000000000000000001A13000000000000000000000000000049
:2041200000000000000000000700FB0100001A0F00FC0100000000000000000000000C004A
:20414000F70100000000010000000A00F90100003E0000004500160200001001001801009D
:204160001A01FF2102002701002801002A0100000000000000000000000000000000000086
:2041800000000000000000000000000000000000000000000000000000160034000000DCF9
:2041A0000532000000000000000000000001040E001102000000000000010101010A001282
:2041C000020100FFFFFFFF380018000200000103020405060709000000000001006400DC28
:2041E000051A04D007020213001900750343080E00000100000001030A1E0101000000177E
:2042000000120002000000000100010553343131000008020200110000020000000000007B
:2042200000FF00000000000C00FF010100000000000000150008020100151617FFFF2D2EB7
:204240002FFFFF232425FFFF0900FA0100001802002E000A00080030000000C8001301005D
:20426000000000000000000000020000029E077D00DC002602F4010800F401960000012269
:204280000006000100E001060000020128102A270000000000010058022E04D007E8030C49
:2042A000000900020200000000000A000C020000012C020012001100000001001234567872
:2042C0009ABC000000001A00FE0100000111000001200000010000000000000001FFFF003C
:2042E0006E00F5010800980864001401000A010A0000FF1F0000142800002C3700008000E7
:20430000FFFFFFFF4600010200000000000000000000000000000000000000000000000058
:20432000000000000000000000000000000000000000000000000000000000005000C4FF6A
:2043400000FFFFFFFF0100000005180B00001600230002000A000000F4FF00000E000100F1
:20436000000000007C00FD07000061098109CD084E00CE008201960976098A09210920005A
:204380005701EA00EA00EA00EA00EA00EA00EA00EA00EA004A092C00EA00EA00EA006100ED
:2043A0004100EA000B01EA006200EA00EA00EA00A30096002100EA00EA001601EA00EA00A3
:2043C000EA00EA00EA0061018200EA00EA00EA00EA00EA00EA00EA004101EA002300EA009C
:2043E00014002600010002000000000115005802D903000020000B000300B3014A015E01A8
:204400002C0164010100000001000A019A01001E0A0000022A001F000300000000000001EB
:204420000000000500000102030000000000000000000000000000000000008007000A00E0
:20444000050200000000000010000301000004040100A81600000000220122020000050826
:20446000E916D516C116AD169916851671165D16651678168B169E16B116C416D716EA1688
:204480004916351621160D16FD161117251739176C1680169416A816BC16D016E416F81611
:2044A0001A163F1664168916AE16D316F8161D17000000000000000000000000000000006F
:2044C0000000000000000000000000000000000000000000000000000000000000000000DC
:2044E000424F5343414D5F4100424F5343414D5F4200424F5343414D5F4500464154534842
:2045000041524B005241434542414E440042414E44362020200042414E44372020200042F4
:20452000414E44382020200041424546523637383100320033003400350036003700380067
:20454000010101010100000004000000010002000300000000000000000032352000313064
:20456000300032303000333530004C5634004C5635004C5636004C563700D2000C000200A3
:20458000320000646464000000464646370078050064CE07CE07CE07010000000000000053
:2045A0000000320000646464000000464646410046050064CE07CE07CE070100000000005B
:2045C00000000000320000646464000000464646410046050064CE07CE07CE07010000003B
:2045E000000000000000320000646464000000464646410046050064CE07CE07CE0701001B
:204600000000000000000000320000646464000000464646410046050064CE07CE07CE07FB
:2046200001000000000000000000320000646464000000464646410046050064CE07CE07AF
:20464000CE0701000000000000000000110001020000000000000200000000000016001B3D
:2046600002000006000000E8030000000000000000000012001B000100002100020301F4FE
:204680000132000100F60021020000000200001002000000000000000000000000000000B9
:2046A0000000000000000000000000000000000000000000000000000000000000000000FA
:2046C0000000000000000000000000000000000000000000000000000000000000000000DA
:2046E0000000000000000000000000000000000000000000000000000000000000000000BA
:204700000000000000000000000000000000000000FFFF000000FF1E0000FF3C0000FF5AEA
:204720000000FF780000FF960000FFB40000FFD20000FFF00000FF0E0100FF2C0100FF4A77
:204740000100FF0000000000000000010B020D0A03050B030D0A030A0B040D0A03080B04BA
:204760000D0A03070B030D0A03000000000000060A01000002030600000003160023020195
:20478000000000000000000000000000000000000034003700010020003200C800D0079626
:2047A000001400320028004C0440060005500014000F00080064000100010005000A000000
:2047C00000F40196000C0016000100C4090000B40028002F0001004D6574656F723635205B
:2047E00070726F000000000000000000000000000000000000000000000F001E000000003B
:2048000005010000000000000C00050001002000010100001200F601020000000000010052
:2048200000000000000022001C02000000020114000026020000000084030102000000006F
:2048400000010000000000001E00280002000000000102000000000000000000000000000C
:20486000000000000000080004020100000007000F020000000A00140000000300002312BB
:204880000001000200E8036400040A000114001E00A4010E000F000000A500000000002EF0
:2048A000552B006300335A2E006900325A0000630032324B0000002800000000000064F4D3
:2048C00001900101374B000000FA00B80B00000000320090015E01F40100000A640000C8B9
:2048E000009001A50000050F00010F0114004B3200005A140B00004D00BB0000140028010E
:2049000000C80000000025146400000F000000000000000000003232C89602643C25050095
:204920000000009600000000002A5523005A002E5A26005F002D5A00005A0032324B000048
:20494000002800000000000064F401900101374B000000FA00AC0D00000000320090015EEE
:2049600001F40100000A640000C8009001960000050F00010F0114004B3200005A140B00B5
:20498000004600AA00001400280100C80017190025146400000F0000000000000000000046
:2049A0003232C89602643C2505000000009600000000002A5523005A002E5A26005F002D9D
:2049C0005A00005A0032324B0000002800000000000064F401900101374B000000FA00AC39
:2049E0000D00000000320090015E01F40100000A640000C8009001960000050F00010F0111
:204A000014004B3200005A140B00004600AA00001400280100C80017190025146400000FBB
:204A2000000000000000000000003232C89602643C250500000A0013000000000044320A4B
:204A40000001010000000000000A0000010000B30000000900020100006E0A010B001900ED
:204A60000000000028010014001A0000007E05EA05B4053200E803D007000010002002038B
:204A8000000364F4010064F401960076001500000000000000000000000000000000000040
:204AA0000000000000000000000000000000000000000000000000000000000000000000F6
:204AC0000000000000000000000000000000000000000000000000000000000000000000D6
:204AE0000000000000000000000000000000000000000000000000000000000000000000B6
:204B00000066002A00000000000000E803D007DC0564FF00000000E803D007DC0564FF00F9
:204B2000000000E803D007DC0564FF00000000E803D007DC0564FF00000000E803D007DCCB
:204B40000564FF00000000E803D007DC0564FF00000000E803D007DC0564FF00000000E8F9
:204B600003D007DC0564FF16002C000000E803D007E803D007E803D007E803D0072A002B78
:204B8000000000001E001E001E0005011E011E011E011E011E011E011E011E011E011E017F
:204BA0001E011E011E011E7E00290002000000203000000101001000000201102000000B31
:204BC00003203000001B022030000000000000000000000000000000000000000000000015
:204BE0000000000000000000000000000000000000000000000000000000000000000000B5
:204C0000000000000000000000000000000000000000000000000000000000000000000094
:204C200000000000001600190200000900000000000000001F03223F013D0007000300006F
:204C400000004300030201000000000000000000000000000000000000000000000000000B
:204C6000000000000000000000000000000000000000000000000000000000000000000034
:204C80000000000001320125000200000000000000000000000000000000000000000000B9
:204CA0000000000000000000000000000000000000000000000000000000000000000000F4
:204CC0000000000000000000000000000000000000000000000000000000000000000000D4
:204CE0000000000000000000000000000000000000000000000000000000000000000000B4
:204D0000000000000000000000000000000000000000000000000000000000000000000093
:204D2000000000000000000000000000000000000000000000000000000000000000000073
:204D4000000000000000000000000000000000000000000000000000000000000000000053
:204D6000000000000000000000000000000000000000000000000000000000000000000033
:204D8000000000000000000000000000000000000000000000000000000000000000000013
:204DA000000000000000000000000000000000000000000000000008001000010000050CC9
:204DC00000F80102000101F40114001200020000000000000000000000000000004600294A
:204DE0000200000000000000000000000000000000000000000000000000000000000000B1
:204E0000000000000000000000000000000000000000000000000000000000000000000092
:204E20000000001A000A02000000004A01B400D6010000C2010E019600440000000A002898
:204E4000020000000000000A00270200000000000016001F020000FFFFFFFFFFFFFFFFFFEF
:204E6000FFFFFFFFFFFFFF42001A02000000000000000000000000000000000000000000DB
:204E8000000000000000000000000000000000000000000000000000000000000000000012
:204EA000000000000000000000070038000100000A00270000002003000042000B0201000E
:204EC000007C06D0057A04790378027701760175EA74E973E872E771E670E56FE46EE36DEB
:204EE000E26CE16BE06ADF69DE68DD67DD66DB65DA64D9000000000000291D1E1A000D02D5
:204F000001000000000000000000000000000000000000000000080007020000003C0C0037
:204F20001D020000000000000000120006020000000001000000010000000100070010021C
:204F40000000000000C3C700FFFFFFFFFFFFFFFFFFFFFFFFFFFFFFFFFFFFFFFFFFFFFFFFDF
:204F6000FFFFFFFFFFFFFFFFFFFFFFFFFFFFFFFFFFFFFFFFFFFFFFFFFFFFFFFFFFFFFFFF51
:204F8000FFFFFFFFFFFFFFFFFFFFFFFFFFFFFFFFFFFFFFFFFFFFFFFFFFFFFFFFFFFFFFFF31
:204FA000FFFFFFFFFFFFFFFFFFFFFFFFFFFFFFFFFFFFFFFFFFFFFFFFFFFFFFFFFFFFFFFF11
:204FC000FFFFFFFFFFFFFFFFFFFFFFFFFFFFFFFFFFFFFFFFFFFFFFFFFFFFFFFFFFFFFFFFF1
:020000040800F2
:020000040800F2
:20800000F0B401292A4C2B4D23684FF0000694BF00270127EE626662A6626763676B47EA45
:2080200042076763EE63EC6B002A38D144F49574EC631C6824F001041C601C68E407FCD46A
:20804000490289085960D8601968EAB921F04001196019498B421DD018494FF47410C860F8
:20806000196841F01E011960596941F080015961196841F00101196022B90E4AD36A43F0B8
:208080000803D362F0BC704741F0400119600A498B42E1D14FF0746041F8500CE0E744F0DD
:2080A0001A04EC63EC6A44F00804EC62C1E700BF981B0020002C0140586402400064024024
:2080C0001148002302461178032902F1060216D00133062BF7D10D4AD36D052B0ED0591CFF
:2080E00003EB4303D16500EB4303032040F2EB3140F2FF32187059809A807047704703EB3A
:20810000430300EB4303F0E7D01B0020981B002070B4C3080D4CE25C00F00706B24004EBCF
:20812000D004D2B20020C6F108038B4228BF0B46C3F108052A419840C91A40EA02004FF0AE
:20814000000614F8012FEED170BC7047381C0020084AD2E9343199420AD0D118013391F8FA
:20816000D8100170C3F30A03C2F8D0300120704700207047981B0020064AD2F8D838D2F8B3
:20818000DC28934294BF4FF400600020013B9B1A18447047981B0020012380F85130704745
:2081A00007B501A8FFF7D4FF0028FAD09DF8040003B05DF804FB044BD3E93403984288BF9C
:2081C00003F50063181A7047981B002001207047024BC3F8E028C3F8E4187047981B00205F
:2081E000024BC3F8E828C3F8EC187047981B00207047704730B4134DD5E934239A4286BF36
:2082000003F50064A21A9A1A0A44B2F5006F13D8A9B101444A1E013810F8014FE9188242E6
:2082200003F1010381F8D840C3F30A03F4D1C5F8D430002030BC7047022030BC7047084696
:20824000F8E700BF981B0020212838B50C4605D022282ED0202813D0002038BD0029FBD0D4
:20826000072AF9D11A4BD3F8F00893F8F41893F8F52893F8F638206021716271A371EBE718
:208280000029E9D0072AE7D1114DD5F8E4381BB10968D5F8E0089847206821796279A379E2
:2082A000C5F8F00885F8F41885F8F52885F8F638D2E70029D0D0022ACED1054AD2F8EC38B1
:2082C000002BC9D00988D2F8E8089847C4E700BF981B0020024B0020C3F8F808704700BFD5
:2082E000981B0020044B00200522C3F8F828C3F8EC08C3F8E4087047981B0020704700BFE4
:20830000704700BF704700BF704700BF704700BF704700BF704700BF042301480B807047E7
:208320009801002010B4074A074B92F8FC08122403F114020C8001280CBF184610465DF8C6
:20834000044B7047981B00209C01002000487047201C002000487047201C0020034B93F8F8
:208360008400032894BF002001207047981B0020034B93F88400032894BF0020012070475D
:20838000981B0020034B93F88400003818BF0120704700BF981B0020A0B182680D4B12B1DE
:2083A00007229A7070471978DA6003294FF004000CBF80214FF48071C3E901111A611A7531
:2083C00098707047034B41F2E47101225A545A70704700BF949900200378022B10D00069B9
:2083E00008B9012070470C4B1B78032B0EBF0B4B80B24FF6F773984294BF002001207047A3
:208400000549436841F650028A58B3EB422F2CBF01200020704700BF94990020F7FFFF0FF6
:208420000378022B14D030B4104A4368006941F6480402F5C2511559096841F63C042B4010
:2084400012595B0A023801FB0030104430BC7047064B426841F6340141F630005958185800
:2084600000EB410000EB5220704700BF949900200E4B70B5D3F8BC4041F06CF8A38905465F
:2084800042F20F7623899B0705D52046FF21BDE870405EF017BE41F05DF8401BB042F1DD5C
:2084A000204646F083FAC0B270BD00BF981B002070B505460E460924FFF7DAFFFF2803D1B7
:2084C000013CF9D1012070BDFE2801D0022070BD064933462A46D1F8BC0000215EF03CFE9B
:2084E000FFF7C6FFFFF7C4FF002070BD981B00202DE9F04383B040F040060C0E05460A0A7D
:20850000080C95238DF801408DF804108DF800608DF802008DF803208DF805300824FFF740
:20852000A7FFFF2802D0013CF9D125BB1E4BD3F8BC40A3890627E84642F20F76B8F1000F8D
:2085400030D018F8015B41F005F8814623899A0715D5ADB2A58140F0FDFF05462389DB07F9
:2085600017D5013FA389E9D10924FFF781FFFF2802D1013CF9D1FF2003B0BDE8F08340F02B
:20858000E9FFA0EB0900B042E0DD204646F00EFAEAE740F0DFFF401BB042DFDD204646F088
:2085A00005FAE1E7FF25CEE7981B0020F8B5194F0023C7F88030FFF75BFFD7F8BC4040F056
:2085C000C9FFA389054642F20F7623899B0710D52046FD215EF076FDFFF74AFFFF2811D1E3
:2085E000FFF746FFFF280DD10423022087F88430F8BD40F0AFFF401BB042E6DD204646F080
:20860000D5F9E9E7D7F800397B670923002087F88430F8BD981B00202DE9F041684C0023AD
:208620004FF4F0722021064604F6081084F8043963F005FE04F6E8204FF4F072202163F0AC
:20864000FEFD94F8C90C10B194F8CA2C1AB900252846BDE8F08144F05FFB0746C4F8D40C88
:2086600044F02EFE05460028F1D00FB12323FB800921384640F04CFAD4F8D40C514F44F047
:2086800041FE94F8CA0C013840B246F0D1FA0223102184F8CC3CC4F8D00C5EF02BFD798D1F
:2086A000494846F039F9D4F8D40C44F025FEFF218C205AF07FFC8046D4F8D40C44F022FE67
:2086C000D4F8D00C04215EF015FDB8F11B0F05D0D4F8D40C202140F01BFAB8E7D4F8D43C18
:2086E000012284F804290BB12322DA80798D364846F012F9D4F8D40C44F0FEFD40210A2028
:208700005AF058FCFF218A205AF054FCC0F38013D4F8D40C84F8D83C44F0F4FDD4F8D00C08
:2087200004215EF0E7FC94F8C83C012B3FD0022B37D0CBB394F8D93C182B08D194F8D82C19
:208740007B8DA4F8DC6CA4F8DE2CA4F8E03C798D1D4846F0E1F8798D1B4846F0DDF8D4F815
:20876000D40C44F0C9FD022100205AF023FCD4F8D40C44F0C7FD0421D4F8D00C5EF0BAFCFE
:2087800094F8E92C94F8EA3C94F8E81C84F8E41CC2F12002C3F1100384F8EB2C84F8EC3CA7
:2087A00056E708237B85C5E710237B85C2E7002EF7D094F8D83C002B14BF08231023F1E700
:2087C000981B002098010020642800202DE9F84F564B984210D003F568530833984267D0AA
:2087E000534B0020A3F8480DA3F8540DC3F84C0DC3F8500DBDE8F88F4D4C4E4E02224FF0DF
:20880000000BC4F8F02C04F6F445D9464FF4007A4FF48078F26A01275A455946BB4403D097
:20882000D4F8640D53F004FF94F8682D85F82420D4F8640DA5F804A04FF000724FF48031B0
:20884000A960EA60A5F8108085F81290A5F806802F762862B72154F0E1F8D4F8F02C364BC9
:208860006F76934545F8283BD4DB84F8569DD4F8F01CB4F8F82CD4F8003DD4F8FC0CB4F84C
:20888000045DC4F86C3D12FB01F203FB01F3A4F8482DB4F8FA1C294AC4F84C0DC4F8503D7C
:2088A000A4F8545DA4F84A1DC4F8442D0120A1E71F4C204E0223C4F8F03C04F6F4454FF03A
:2088C000000B4FF4806A4FF040094FF40068F26A01275A455946BB4403D0D4F8640D53F019
:2088E000A7FED4F8641D94F8682D296285F824204FF400314FF00062C5E90212A5F804A001
:20890000A5F81090A5F80680AF74FFF7D9FB28466F7653F0D5FFD4F8F02C094B45F8283BC4
:208920009345D4DB84F8567DA1E700BF1971EF00981B002098010020E0C2060838C306085C
:208940000CC30608F8B51A4C94F8703D002BFBD159B301444E1E451ED4F8DC28D4F8D8184B
:2089600015F8017F531CC3F30A038B422CBF4FF400600020C91A22440144012982F8747D9A
:20898000C4F8DC380FD1012040F010FED4F8D838D4F8DC188B4294BF4FF4006200225B1AD0
:2089A0001344012BEFD0B542D6D10020F8BD00BF981B002010B5094CD4F8F83808461146B5
:2089C0005BB1D4F8F838052B07D1002AD4F8003903DDFFF7B7FFD4F8003910BD981B002027
:2089E00010B590F85010002380F8503081B10B4CD4F8F82872B1D4F8F828052A0CD13C30B3
:208A0000D4F80039FFF79EFFD4F80039012010BD0120FCE71046FAE71846F8E7981B002080
:208A2000002280F85120DBE790F85020531C0244DBB280F8503082F83C1090F851200AB1BD
:208A4000132B00D9CCE770472DE9F8434379574D002B14BF0122002285F8B02003D185F803
:208A60008430BDE8F88390F8018008F1FF3676B2044630460F4646F0DBF80223C5F8BC0007
:208A800085F8B8302378002B63D1E478002C54D14FF48071D5F8BC00C5F8C0405EF02AFBDD
:208AA0004FF47A7040F082FDD5F8C00044F02AFCD5F8BC404FF00A08A38942F20F764FF0B5
:208AC000FF090BE0A4F80C9040F044FD07462389D9072CD5B8F10108A3890DD040F03AFDFE
:208AE000074623899807EDD440F034FDC01BB042F7DD204645F05AFFD5F8BC102C4B0A8984
:208B000092070AD50A8912F0800206D1D5F8001985F8782001236967A1E7013BEFD195F8EF
:208B2000782085F88430531C85F8783099E740F011FDC01BB042CADDDBE7204644F0ECF866
:208B4000044608B11E23C380092120463FF0E0FF9EE706EB86063E44414696F90320002013
:208B600041F0E2F8064630B1406841F0CBF8B36885F8CE3018B9002385F8C43085E70D4A63
:208B8000431E02EB4311303291F8486002EB4313C5F8C830002EEED11723A1F848305DF023
:208BA000A1FE012385F8C4306FE700BF981B0020A1860100980100202DE9F04FCF4ED04D29
:208BC00086468C4617460FCE05F27C442DED068B0FC40FCE0FC496E807008BB095F8B234A5
:208BE000059784E80700CDE906EC042B00F24981DFE813F0A801470142010500B8019FED8B
:208C0000C18ADFEDC18AC149C5F89814C049C14BC14AC5F894140599002918BF134638EEDD
:208C2000887AF5EE006AC6EE879ABC4EC5F8A034A6F11503039306F1C0080027DFEDBF7A45
:208C40009FEDB79A28EE278AB0EE67AA079BBB4200F00C81039B13F8014B039307F1010B16
:208C60005FFA8BF3002C00F08081002203E00132152A00F07A8102EB42014FEA420918F8DA
:208C80000100A042F3D12944049391F88D15002900F0738120463FF021FD824600683FF0DF
:208CA000C1FC9AF805103FF039FD90F800C0BCF1000F40F05A8105EB09014FEA141909F182
:208CC000FF39049B81F8CD350322B9F1040F81F8CC2504F00F0000F2FF80924C04EB49016B
:208CE000B1F8B0C04CFA00F111F0010100F02881012101FA00F0013800EA0C00A1440493D0
:208D00005FF002FE99F8BCC0DFF82CE2049B60440EEBC00C03228CF807308CF806205EF82A
:208D20003000C6F814C000F13F4303F57E0304EB9324012194F8C4309AF8082003F01F046D
:208D40005B09032B01FA04F100F0D380042B00F0CB80022B00F0C380BCF804300893B3FA54
:208D600083F3C3F11F03C3F3CC0100EB810103F007030C6A9B004FF00F0C0CFA03FC24EA3C
:208D80000C040C620C6A02FA03F323430B62022308A909930BF02AFC059B002B76D0B5F8C9
:208DA000B034D5F8781807EE903AF8EEE77AFCEEE77A17EE900AB1FBF0F202F57F42FF320B
:208DC000120CB1FBF2F295F8B214B2FBF0F0042983B272D007EE902AF8EE676A66EE887AA5
:208DE00029EE677A95F8B30406990091A8EEA67A019051463046C6ED027A86ED037A36F06E
:208E00004BFF002F64DD7368D5F8D024934261D0012F5DD0D5F8E82493425BD0022F57D068
:208E2000D5F80025934255D0032F51D0D5F8182593424FD0042F4BD0D5F83025934249D097
:208E4000052F45D0D5F84825934243D0062F3FD0D5F86025D31A18BF01235F460122082F2A
:208E60003374727406F118067FF4F0AE2E480BB0BDEC068BBDE8F08F9FED2C8AF0EE488ABE
:208E8000C1E69FED2B8AF0EE488ABCE6B0EE690A60F02AFEFCEEC07A4FF6FF7317EE902A75
:208EA000D5F87818B1FBF2F21A44120CB1FBF2F295F8B214042918468CD107EE900A07EEFA
:208EC000102AF8EE677AF8EE476A67EE8A7A87E70123C2E70023C0E7C6F814C05CE7154B67
:208EE0005C6C2143596437E7124B1C6B2143196332E7104B1C6C214319642DE764C3060881
:208F0000902C0020ACC5A737ACC5A7364162030885630408A55F0308796304085C31002092
:208F200000007A44E0C206080C310020282930386F12033900380240883200206F12833A5E
:208F4000716129E71FED038A0D4A0E4BC5F89824C5F8943400220123CDE90532F0EE488A05
:208F6000094B5CE69FED098AEEE7094A064BC5F89824C5F8A034002079E70B68FFDE00BF2A
:208F800041620308856304087963040800000000F5600308104B70B5D3F878480546006829
:208FA0000E4664080BF026FAB4FBF6F1B1F5803F03D3012CFAD96408F6E72246284689B2AB
:208FC0003FF02AFA0549064B0B6028460022BDE870403FF041B900BF902C0020703D0020BE
:208FE0004DFF010810B5044C04480A4621460AF07BF8204610BD00BF783D002054710708FC
:2090000010B5044C04480A4621460AF06DF8204610BD00BF783D00206471070810B5044C19
:2090200004480A4621460AF05FF8204610BD00BF783D00207071070810B5044C04480A4674
:2090400021460AF051F8204610BD00BF783D00207C71070810B5044C04480A4621460AF091
:2090600043F8204610BD00BF783D00208871070810B50C4C94F8CD200023C4F8803012B1FE
:20908000094AC2F8F0305AF0D5FE20B10423022084F8843010BDD4F800396367092384F8F8
:2090A000843010BD981B0020883D002070B50D4D95F88430042B04460E460AD0082B06D106
:2090C000EB6F83420CD0FFF7D3FF022801D0012070BD0823C5E91F4685F88430022070BDC6
:2090E000022070BD981B002010B509F0D1FF104C58B194F88430032B12D894F8783001339B
:20910000DBB2072B84F8783003D9002384F8843010BDD4F800396367012384F8843010BD80
:20912000D4F8BC004FF480715DF0E4FFE5E700BF981B002070B54379234C002B14BF012373
:20914000002384F8B03003D1002384F8843070BD1E4D002195F9F720032040F0E5FD0028AE
:20916000F2D04668304640F0CDFD84F8CC000028EAD095F8F530003B18BF0123304684F80B
:20918000CD305AF01BFA09F083FF38B994F8783084F88400013384F8783070BD5AF030FFD5
:2091A00040B194F878300022013384F8783084F8842070BDD4F8002984F8780001236267ED
:2091C00084F8843070BD00BF981B0020883D002010B55AF015FF58B10B4C94F878300133D0
:2091E000DBB2072B84F8783003D9002384F8843010BD09F04DFF0028F7D0D4F8003963678D
:20920000012384F8843010BD981B00202DE9F041874C94F8B050002D00F0F88094F88420EF
:20922000844F0226531E082B41D8DFE803F037399E406850154005005AF0FCFD002840F0C1
:20924000EC80636FD4F80029FA3393422CD2FFF7BFFF94F88420E5E75AF0ECFD0028F0D010
:20926000D4F880300022012B84F8782040F2D980E16F94F8CD00013B0131C4E91F1310B1CE
:209280006C4BC3F8F020082284F88420A2F10805B5FA85F56D092846BDE8F08184F88460DF
:2092A0005AF0C8FD002841D194F88420531EDBB2022B09D8D4F80039616F5B1AC82BE5D92E
:2092C000FFF786FF94F88420042ADFD1E3E7236B002BDBD1E66ED4F800396367072284F80E
:2092E0008420002ED2D0D4E91821236F0120B047DAE7636FD4F8001964338B42C6D2D4F81A
:209300002C80B8F1000FF4D15AF094FD0028A0D0E66E84F87880042384F88430002E7AD01A
:20932000D4E91821236F4046B047BDE75AF028FA0028B9D197F8F930002BA3F10203B3FA3D
:2093400083F314BF022201225B0984F8792084F87A305AF015FA00287FF479AFD7F848317A
:20936000C4F88830032384F884305AF009FA00289AD1304BC4F8800093F82C61B3F82E019A
:20938000D3F830E1D3F830C1D3F83071D3F8302184F88E6093F83411A4F88C0093F835612A
:2093A00084F8922093F83501D3F83821C4F89420B3F83E81B3F83E2184F89310B3F83E119D
:2093C000C2F30B1343EA182303F00F0301F00F024FEA1E6E4FEA1C4C3F0A360900F00F005E
:2093E00003F5FA63042184F8990084F88FE084F890C084F8917084F89860A4F89A3084F854
:209400009C2084F884102846BDE8F08184F884502846BDE8F08105463DE7042384F8843062
:2094200039E7FAD1FFF724FE94F88420531E3EE7981B0020883D00202DE9F8431A4C94F868
:209440008460042E0546894690461F4608D0082E02D00020BDE8F883FFF7A8F80228F8D1F8
:20946000D4F8C00043F048FF94F87A3093B969021120FFF73DF898B9D4F80039C4F860909B
:209480000522C4E91B87656684F8842063670120BDE8F88329461120FFF72AF80028EBD0C5
:2094A00009F0CCFDD5E700BF981B002070B51E4C94F88430042B06460D4608D0082B22D101
:2094C000E36F83422DD0FFF771F802281BD1D4F8C00043F011FF00213720FFF709F8294656
:2094E0001720FFF705F8B0B994F87A306BB971021920FEF7FDFF70B90823C4E91F6584F8E1
:209500008430022070BD012070BD31461920FEF7EFFF0028F0D009F091FDFFF7E5FD0320FD
:2095200070BD022070BD00BF981B00202DE9F04F95B0CDE902236A4C0646884694F8843098
:20954000042B0DD0082B07D1E36FB34200F0C480FFF72CF80228F1D0012015B0BDE8F08F6A
:20956000D4F8C00043F0C8FE94F87A30002B40F0998071021820FEF7BBFF002840F0A680E4
:2095800094F88450FEF774FF082D0CBFFC21FE21D4F8BC9001913FF0DDFFB9F80C3001998B
:2095A000054642F20F77B9F8083098074BD548465DF088FD94F8C430002B52D005A80AF02A
:2095C00041FD94F8CE20D4F8BC30D4F8C810CDF81C8052060C33486805920693402200231A
:2095E000CDE90C3308920F934FF480620A930E934FF400730B9209930AF062FDD4F8C830CB
:2096000005A958680AF030FDD4F8C830D4F8BC2059680B6843F001030B6093889BB243F0D8
:20962000020393800299E1660399C4F860800122062300206666216784F8682084F8843004
:2096400015B0BDE8F08F01913FF084FF431BBB420199A8DD484645F0A9F994F8C430002B53
:20966000ACD1D4F8BC50CDF80480AB894FF4807B42F20F79019BBBB113F8017B01933FF0CC
:2096800069FF82462B899A0710D5BFB2AF813FF061FF07462B89DB0712D5BBF1010BAB897A
:2096A000E8D1BFE7314665E7FF27E8E73FF052FFA0EB0A004845E5DD284645F077F9B1E784
:2096C0003FF048FFC01B4845E4DDF5E709F0B6FCFFF70AFD032040E7FEF7CAFEFC2157E705
:2096E000981B00202DE9F04F944C94F8B07087B0002F00F0AF8194F8842042F20F75531ED7
:20970000082B00F28180DFE813F09300BC004A017F006D000900FA007F00E70094F8C430EA
:20972000002B40F02682D4F8BC6094F868A0236EB28903EB0A2A4FF4807BBAF1000F00F0D4
:20974000C9821AF8018B3FF005FF81463389980740F1C8811FFA88F8A6F80C803FF0FAFE67
:2097600080463389D90740F1C881BBF1010BB389E3D194F868300133DBB2022B84F868303F
:209780003FD1D4F8BC603FF0E5FEB389804633899A0740F19C81304600215DF093FCD4F8D3
:2097A000BC603FF0D7FEB389804633899B0740F18381304600215DF085FCFEF759FE00F053
:2097C0001F00052800F0A882FFF78EFCE66E002E00F0C9810022236F616E0120B04794F8C0
:2097E00084208CE7206E4FF40071FEF761FE012800F0A481022800F0A8810646002800F0D7
:20980000ED8194F88420531EDBB2022B00F22C81D4F80039616F5B1AC82B00F22181A2F17C
:209820000807B7FA87F77F09384607B0BDE8F08FD4F8C00043F060FD00210846FEF758FE33
:20984000064609F0FBFB012EDBD10023D4F8C00084F8793043F050FD40F2AB110820FEF793
:2098600047FE052800F08281012800F0018109F0E5FB94F87920002A00F06182022384F84C
:209880008430D4F8C00043F037FD94F87930022B0CBF4FF08046002600213720FEF728FE36
:2098A00031462920FEF724FE064609F0C7FB002EA7D194F87930022B00F0A48184F87A6057
:2098C000D4F8C00043F018FD00210920FEF710FEB0B309F0B3FB94E70826FEF7C9FDFF28D2
:2098E00000F03082013EF8D1636FD4F80029FA33934286D2FFF7F8FB94F88420FFE6FEF7AA
:20990000B7FDFF284FF0080605D0013EECD0FEF7AFFDFF28F9D1D4F880300022012B84F877
:20992000782040F21582E26F08210132013BC4E91F2384F884100A4671E700BF981B0020A4
:20994000C7481021FEF7B4FD06460028C1D101217F20FEF7DDFB01288046BAD1304602217A
:20996000FEF7D6FB002800F0B8810128B1D116213A20FEF7CDFB01308002C4F8880009F0E7
:209980005DFBD4F8C00043F0B7FC00210A20FEF7AFFD002840F08381032384F8843010212E
:2099A00002A8FEF785FD00287FF42BAF9DF815309DF816109DF810209DF809609DF80A001A
:2099C0001B01DBB243EA111303F5FA63A4F89A30DDF8113001F00F0184F89C101BBA1109A4
:2099E00002F00F0240EA062084F8981084F899209DF808109DF80B20C4F89430039BC4F874
:209A00009030A4F88C0084F88E1084F88F2009F015FB94F87A3073B9D4F8C00043F06CFC87
:209A20004FF400711020FEF763FD064609F006FB002E7FF45FAFD4F8BC0004215DF05AFBA9
:209A4000002204233846C4F8802084F8843007B0BDE8F08F384684F8847007B0BDE8F08F0F
:209A6000FFF742FB94F88420042A7FF4D8AEDBE6D4F8BC600DF1080AB3893B464FF0040B98
:209A800057464FF0FF099A463FF064FD8046338998073AD5A6F80C903FF05CFD80463389FE
:209AA000D90744D5B3899BB20FB107F8013BBBF1010BE9D1574632E03FF04CFDA0EB0800FD
:209AC000A8427FF772AE304644F070FF75E63FF041FDA0EB0800A8427FF759AE304644F081
:209AE00065FF5CE63FF036FDA0EB0900A8427FF72DAE304644F05AFF3BE63FF02BFDA0EB89
:209B00000800A8427FF72DAEF3E73FF023FDA0EB0800A842BBDD3046574644F047FF9DF8A2
:209B20000B30AB2B04BF022384F879309FE63FF011FDA0EB0800A842B1DDECE7636FD4F8C9
:209B4000002964339342BFF45CAE09F077FAFFF7CBFAE66E3EB100221046236F616EB0477B
:209B600094F88420CBE594F88420C8E584F879607DE6D4F8C8303B485968D3F81CE03A4E19
:209B80003A4B994288BF30461EF0005F00F095804668DFF8DCC006EA0E0616EA0C0F3FF4C3
:209BA0003EAE0EEA0C03C3600B68D4F8BC6023F001030B603389D80703D5B3893389D90767
:209BC000FBD433899A07FCD533891B06F9D4B38823F002031B041B0CB380D4E509F02EFA38
:209BE000E56E84F87860042384F88430002D3FF41BAED4E91821236F3046A84794F8842021
:209C0000531E01E6D4F8C00043F076FB31463A20FEF76EFCD4F8BC6001900DF1080AB389C7
:209C20003B464FF0040B57464FF0FF099A463FF091FC804633899A071CD5A6F80C903FF058
:209C400089FC80463389DB0730D5B3899BB20FB107F8013BBBF1010BE9D1574614E000BFD0
:209C6000381C002000600240006402400F6402407D0F7D0F3FF06EFCA0EB0800A842D9DD8F
:209C80003046574644F092FE019B43B909F0D6F9029B1BBAC3F3807384F87A3010E609F05D
:209CA000CDF9FFF721FA94F8842028E53FF052FCA0EB0800A842C5DDE2E70668DFF8B0C076
:209CC00006EA0E0616EA0C0F3FF4A9AD0EEA0C03836069E74FF0FF0835E504212C20FEF7DC
:209CE00017FA032106464E20FEF712FA0C2181463620FEF70DFA09F10209431C03FA09F3D1
:209D000008FA06F6A3FB0601430A43EAC153C4F8883009F093F934E6E56ED4F800396367DD
:209D2000072284F88420002D3FF479ADD4E91821236F0120A84794F88420531E64E584F856
:209D400084206CE509F07AF9042384F884306BE508D0042384F8843009F070F994F884203A
:209D6000531E51E5FEF722FC02287FF44AADB0E57D0F7D0F2DE9F04FC14C94F8581183B05E
:209D80000546C1F34001D4F8600143F0C1FA94F85811D4F85C01C94301F001016F1E43F08B
:209DA000B7FAFBB20193002D00F0D080B54EDFF8DC82B54D4FF01009D4F8600143F08CFACC
:209DC000D4F85C0143F088FAB4F86831002B40F04E8194F86A11D4F86C0143F099FA4FF0F1
:209DE000FA0A4FF47A710120D8F80430C3F30803002B40F00F81EFF31183002B40F00A8104
:209E0000D6F80029D5F808C0D6F800399A42F7D1D4F890319C45F3D8D4F88C7101FB07F313
:209E2000A3EB0C03B3FBF7F301FB0232D8F80430C3F30803002B40F0AB80EFF31183002BD1
:209E400040F0A680D6F80039D5F808B0D6F80079BB42F7D1D4F89071BB45F3D8D4F88C71B3
:209E600001FB07FCACEB0B0CBCFBF7FC01FB03C39B1AB3F57A7FD9D3BAF1010AB4D1D4F8C0
:209E8000600143F029FAD4F85C0143F025FAB4F86831002B40F0DF8094F86A11D4F86C0151
:209EA00081F0010143F034FAFA204FF47A714FF0010CD8F80430C3F30803002B40F0898011
:209EC000EFF31183002B40F08480D6F80029D5F808E0D6F800399A42F7D1D4F890319E45E6
:209EE000F3D8D4F88CA101FB0AF3A3EB0E03B3FBFAF301FB0232D8F80430C3F3080343BB78
:209F0000EFF311832BBBD6F80039D5F808B0D6F80079BB42F7D1D4F89071BB45F3D8D4F8E9
:209F20008CA101FB0AFEAEEB0B0EBEFBFAFE01FB03E39B1AB3F57A7FDDD30138B9D1019B46
:209F40005F1EFBB2FF2B01937FF436AF03B0BDE8F08FEFF3118A89F31288AF682B68DB03CF
:209F600044BFC4F888C1AF68D6F80039D4F888E15FFA8AFA8AF31188D4F88CA1734401FBE7
:209F80000AFEAEEB070EBEFBFAFE01FB03E3D0E7EFF3118E89F31288D5F808B02B68DF0330
:209FA00044BFC4F88801D5F808B0D6F80039D4F888C15FFA8EFE8EF31188D4F88C71634449
:209FC00001FB07FCACEB0B0CBCFBF7FC01FB03C34EE7EFF3118E89F31288D5F808A02B6894
:209FE000DA0344BFC4F888C1D5F808A0D6F80039D4F888215FFA8EFE8EF31188D4F88CE153
:020000040800F2
:20A000001A4401FB0EF3A3EB0A03B3FBFEF301FB023270E7EFF3118C89F31288D5F808E0DA
:20A020002B68DB0344BFC4F88801D5F808E0D6F80039D4F888215FFA8CFC8CF31188D4F871
:20A040008C711A4401FB07F3A3EB0E03B3FBF7F301FB0232EAE6D4F88431002B3FF424AFC6
:20A06000D4F87031C3F800A084F881A11CE7D4F88431002B3FF4B3AE3FF058FBAFE600BF61
:20A08000883D0020981B002010E000E000ED00E02DE9F04FBD4CBE4E94F85811D4F86001DF
:20A0A000DFF8F482BB4D83B0C1F3400143F030F994F85811D4F85C01C94301F0010143F077
:20A0C00027F9052301934FF01009D4F8600143F003F9D4F85C0143F0FFF8B4F86831002B2D
:20A0E00040F04C8194F86A11D4F86C0143F010F932274FF47A710120D8F80430C3F308037A
:20A10000002B40F00F81EFF31183002B40F00A81D6F80029D5F808C0D6F800399A42F7D1C1
:20A12000D4F890319C45F3D8D4F88CE101FB0EF3A3EB0C03B3FBFEF301FB0232D8F8043040
:20A14000C3F30803002B40F0AB80EFF31183002B40F0A680D6F80039D5F808B0D6F800C99E
:20A160006345F7D1D4F890C1E345F3D8D4F88CE101FB0EFCACEB0B0CBCFBFEFC01FB03C3FF
:20A180009B1AB3F57A7FD9D3013FB5D1D4F8600143F0A2F8D4F85C0143F09EF8B4F86831C6
:20A1A000002B40F0E08094F86A11D4F86C0181F0010143F0ADF832204FF47A710127D8F8E1
:20A1C0000430C3F30803002B40F08B80EFF31183002B40F08680D6F80029D5F808E0D6F8D3
:20A1E00000399A42F7D1D4F890319E45F3D8D4F88CA101FB0AF3A3EB0E03B3FBFAF301FB1F
:20A200000232D8F80430C3F3080343BBEFF311832BBBD6F80039D5F808B0D6F800E97345F0
:20A22000F7D1D4F890E1F345F3D8D4F88CA101FB0AFEAEEB0B0EBEFBFAFE01FB03E39B1A1F
:20A24000B3F57A7FDDD30138B9D1019B5F1E17F0FF0301937FF439AF03B0BDE8F08FEFF320
:20A26000118A89F31288D5F808B02B68DB0344BFC4F88871D5F808B0D6F80039D4F888E1BE
:20A280005FFA8AFA8AF31188D4F88CA1734401FB0AFEAEEB0B0EBEFBFAFE01FB03E3CEE71D
:20A2A000EFF3118E89F31288D5F808B02B68DB0344BFC4F88801D5F808B0D6F80039D4F871
:20A2C00088C15FFA8EFE8EF31188D4F88CE1634401FB0EFCACEB0B0CBCFBFEFC01FB03C32F
:20A2E0004EE7EFF3118E89F31288D5F808A02B68DA0344BFC4F88871D5F808A0D6F8003979
:20A30000D4F888215FFA8EFE8EF31188D4F88CE11A4401FB0EF3A3EB0A03B3FBFEF301FBFF
:20A3200002326EE7EFF3118C89F31288D5F808E02B68DA0344BFC4F88801D5F808E0D6F80F
:20A340000039D4F888215FFA8CFC8CF31188D4F88CC11A4401FB0CF3A3EB0E03B3FBFCF3A8
:20A3600001FB0232EAE6D4F88431002B3FF423AFD4F870311F6084F881711CE7D4F884314E
:20A38000002B3FF4B5AE3FF0D1F9B1E6883D0020981B002010E000E000ED00E00E4B30B4DA
:20A3A000DB68427801780D4CDB43C3F30223C3F10403DBB202FA03F360181B0101F01F05F2
:20A3C0000122490903F0F003AA4080F8003344F8212030BC704700BF00ED00E000E100E020
:20A3E00000F01F0240090123032803FA02F304D004280CD0022805D07047074A116C0B4314
:20A4000013647047044A516C0B4353647047024A116B0B43136370470038024000285FD033
:20A420000368374A2DE9F04103F13F4404F57E0402EB9422012492F8C42002F01F05520950
:20A44000032A04FA05F456D0042A4FD0022A48D08588B5FA85F0C0F11F00C0F3CC0603EBAD
:20A46000860600F0070082000F24306A944020EA04003062306A01FA02F202430021326213
:20A480004FF0010E0A464FF0030C02270EFA02F838EA050002F101021CD118680CFA01F420
:20A4A00020EA04001860186807FA01F606431E609E6826EA04069E6098689860586820EAF7
:20A4C0000800586058685860D86820EA0400D860D868D860102A01F10201D7D1BDE8F08159
:20A4E0007047084A556C2C435464B1E7054A156B2C431463ACE7034A156C2C431464A7E748
:20A50000E0C20608003802402DE9F0410378012B84B00446164635D0022B24D1836841F006
:20A52000800113B11A689B885383656803913FF011F8AB890399074642F20F782B899B0794
:20A5400015D528465CF0BEFD01236068324600215CF002FEA368FBB11A689B8813830120B8
:20A5600004B0BDE8F081002004B0BDE8F08103913EF0F0FFC31B43450399DFDD284644F016
:20A5800015FAE1E700920A46417990F904005DF09DF904B0BDE8F0810120E5E758B183880D
:20A5A0004FF00042B3FA83F332FA03F303D002490A6813430B607047003C0140134B026888
:20A5C000196821EA02011960596821EA0201596019680A431A609968026821EA0201996031
:20A5E000D96821EA0201D9604179102907D001F1804303F59E3319680A431A60704799688B
:20A6000011439960D9680A43DA607047003C0140002864D0F0B58388B3FA83F3202B0A4627
:20A6200085B00446C3F11F0143D02D4D2D4E05EB81037718C3F89421002197F8CC703EF032
:20A6400067FAB4F804C02268274CBCFA8CFCCCF11F0303F0FC0101F1804101F59C3103F0B6
:20A66000030398004FF00F0E02F13F438A680EFA00FE22EA0E0203F57E038A60C3F3872394
:20A68000834088684FF0004222FA0CF203433D448B6002A8626101234FF400618DF80E30C2
:20A6A0000292ADF80C10FFF789FF95F8D431F02B01D805B0F0BD3E44F02196F8DC308DF82D
:20A6C000043003224FF4807301A885F8D4118DF80520ADF80630FFF761FE05B0F0BD7047ED
:20A6E000883D0020E0C20608003C014010B4B8B10D4CD4F8DC31102B05D15DF8044B05210E
:20A7000000203EF0EDBC03EB4302224482F8E11101210B4482F8E00182F8E211C4F8DC313B
:20A720005DF8044B704700BF883D0020C0782021DCE700BF2DE9F04FDFF8A4A32DED028B05
:20A740009AF824120022CAE98522CAE9872297B0CAF8102219B19AF825228AF810229AF835
:20A7600026221AB19AF827228AF81F229AF82A221AB19AF82B228AF81A229AF828221AB13B
:20A780009AF829228AF815229AF82C3205935A1ED3B257B203937B1C00F0AA80C54AC64E2B
:20A7A00052F83790029602EBC70200231279019308EE102A1D46344698462678394630467A
:20A7C00044F0DCFC83463046BBF1000F1ED042F0A3FAEA1D1321D2B220B14FF0000E8271E6
:20A7E00080F807E03EF094F9207844F0F1FC4FF0070308F1010223714FF0010384F802806C
:20A800006070CDF804B05FFA82F8E3700135042D04F10504D1D118EE100A029ECDF81080AD
:20A82000FFF7DEFDA549A64A4868024042F440324A600FB9019B5BB9A24C4820FFF7D0FD94
:20A84000204602215DF03EF9A26842F00102A2609A489C4A4168BAF82E4241F40001416040
:20A86000516821F480515160916B21F4401141F480119163D16841F46001D160956B85F4F3
:20A880004011C1F3015101EB81011F2000FA01FC25EA0C0C112505FA01F141EA0C01916343
:20A8A000D16841F0E061D160956BC5F30151C1F10401C9B201EB810188404FF0120C25EADE
:20A8C00000000CFA01F108439063E4B1BAF83012CAF83842A1B1BAF83222CAF83C1262B102
:20A8E000019B7948521A90FBF2F2CAF840226BB917B0BDEC028BBDE8F08F744A1288EFE789
:20A90000734A1188E7E7734A1488DFE7484604995DF0D8F8684B012003F114080723F27834
:20A92000441CE4B252B375783279A5F10A0101EB410105EB450C092D03FA01FE03FA0CFB3E
:20A9400002FA01F140F29F80D9F80C2022EA0E0E41EA0E01C9F80C10421E02EB82021F216B
:20A96000062801FA02FC05FA02F272D8D9F8341021EA0C010A432046C9F834200536B0454E
:20A98000CDD1D9F80820039942F40072C9F80820D9F8082042F48072C9F80820D9F80820F0
:20A9A000574442F00102C9F8082097F9342202203FF0BAF9044600289AD0466830463FF0C5
:20A9C000A1F9454B421E03EB421393F84850002D8ED1059983F84910062283F84820002856
:20A9E00086D030463FF08EF95BF07CFF606809F067FB07A809F026FB049EA268374807925F
:20AA0000012E8CBF4FF4806300230D9309F14C034FF48072CDE90A56089309904FF4003395
:20AA200060680C9507A94FF400674FF40056CDE91023CDE90E7609F017FB6268136843F014
:20AA400001031360D9F8083043F08043C9F808304EE7C11FA0F10D0201EB81014FF01F0EF8
:20AA600002EB82020C280EFA01FC0EFA02F005FA01F113D8D9F8302022EA0C021143204661
:20AA8000C9F830107AE7D9F8101002FA0CF221EA0B0B42EA0B02C9F810205DE7D9F82C10CD
:20AAA00005FA02F221EA00010A432046C9F82C2064E700BFC4C30608983F002000230140DD
:20AAC000E030FCFF00200140803801002E7AFF1F2C7AFF1F2A7AFF1F98010020CC3F002021
:20AAE000883D00202DE9F84F2E4F00EBC00407EB8404D4F850622EB1054694F8610200F0E7
:20AB0000FF0820B14FF000084046BDE8F88F89469A4693463EF01EFD4FEA49010123C9B271
:20AB200084F8621284F863B284F8653284F8668284F8643284F8613284F86082B288C4F8A8
:20AB400068A291058146C4F86CA21DD43388DA0510D442F20F7405E03EF0FCFCA0EB0903FC
:20AB6000A34215DC33889B05F6D433889BB243F480733380B3889BB243F440734FF001083B
:20AB8000B3804046BDE8F88F98464046BDE8F88FB7F8B83201339BB22846A7F8B8325CF0E3
:20ABA00023FCB1E7883D002070B5464E96F8BA4204EB440306EBC303650093F8BC32032BBD
:20ABC0006ED8DFE803F059291E02254406EBC505D5F8C002002870D196F81C339C425FD0CD
:20ABE000013404F00302934286F8BA2258D002EB420406EBC4040223C4F8C00284F8BC32D7
:20AC000070BD2B1906EBC303D3F8C02272B1013AC3F8C022002070BD2B1906EBC303D3F851
:20AC2000C022002AF3D1022283F8BC22254406EBC50595F8C832013BDBB285F8C8328BBB96
:20AC4000214B96F81C63D3F83012D5F8C402621C02F003024B1E0324B242034485F8BC4220
:20AC6000B3FBF1F0C5F8C0021AD0994218D80138C5F8C002012070BD44F08AF980B1124BC6
:20AC80002C44D3F8302206EBC404012102F51C5384F8BC120F33B3FBF2F3C4F8C03270BDEC
:20ACA000012070BD084BD3F83022012002F2E733B3FBF2F3C5F8C03270BD0138C5F8C00280
:20ACC000002070BD883D002098010020054B93F81D23002AFBD1D3F8803E03491B6801F12E
:20ACE0000C001847883D0020A84000202DE9F84F3249DFF8D4B091F8F9100124022907469A
:20AD000019461046CBF82C404FF000022C4C1D4618BF7F02FDF774F92A4B63626B02A362CE
:20AD2000E36A40F2FF5943F093034FF400704FF48A62E3620121C4F83890A0601020E26034
:20AD400058F06AFE012D40F251434E46C4F83890CA4640F252488EBF4FF0120998464FF097
:20AD600011090A25C4F838A00121A7604846C4F80C8058F051FE03464FF0000C40F27742E1
:20AD800001213720A6632BB900231846CBF82830BDE8F88FA663C4F808C0E26058F03CFE34
:20ADA000013DA6630028EFD015F0FF05DAD10346CBF82C50CBF82830BDE8F88F883D0020FD
:20ADC000002C014000E1F505981B00202DE9F843184C94F88460042E0546894690461F46AC
:20ADE00008D0082E02D00020BDE8F883FEF740F90228F8D101234A4628460021FFF776FF64
:20AE000050B1FEF7E5F9E56E002DECD00022236F616E1046A847E6E7D4F80039C4F86090DC
:20AE20000522C4E91B87656684F8842063670120BDE8F883981B00202DE9F84F2F49DFF827
:20AE4000C49091F8F9101E4602292D4B07464FF0010418BF4702012E40F259481C6398BF7C
:20AE60004FF48B683B469346474640F2FF55B0468CBF4FF0190A4FF0180A0A241E4640F267
:20AE8000FF53C9F838300121C9F808605046C9F80C7058F0C1FD03464FF0000C40F2774294
:20AEA00001213720C9F83850A3B9584641460122FDF7A6F84646134A134B5362760296622E
:20AEC000D36A43F09103D3620D4B002108469962BDE8F88FC9F83850C9F808C0C9F80C208C
:20AEE00058F09AFD013CC9F838500028DDD014F0FF04C4D1024B1C63BDE8F88F883D00209F
:20AF0000981B0020002C014000E1F5052DE9F047374C82B005460E461746984694F884002A
:20AF200004280CD0082806D1E36FAB4207D0FEF79FF80228F2D0012002B0BDE8F087DFF8AE
:20AF4000B8A02666DAF8F0906566C9F34F210F294FEA592223D8D4F880300193FBB194F895
:20AF6000CD00E0B1B9F5005F13D0224831464FF40072484461F002F909F50072C2F34F2180
:20AF80001029CAF8F0204FEA522202D0019B012B21D192B2013A174EAD1A0B4600E001236D
:20AFA00032462846062601250021E766C4F8708084F8685084F88460FFF73EFF0028BBD0C5
:20AFC000FEF706F9E66E86B12846236F616E0022B0470320B0E7E26F013B01320421C4E9BE
:20AFE0001F2384F884100220A6E70320A4E700BF981B002094690020883D00202DE9F047C1
:20B00000274D95F8843E022B82B004460F46164611D0012B0BD10091134695F8891E0246C4
:20B0200095F9880E5CF052FC02B0BDE8F087002002B0BDE8F087D5F88C3E13B11A689B8896
:20B040005383D5F888AE3EF085FABAF80C30804642F20F79BAF808309B0714D52146504688
:20B060005CF030F83346D5F8880E3A4600215CF073F8D5F88C3E83B11A689B881383012001
:20B0800002B0BDE8F0873EF065FAA0EB08034B45E0DD504643F08AFCE4E70120C4E700BFCD
:20B0A000883D002030B40578022D14D0012D02D0002030BC7047044690F90400084B421CEC
:20B0C00083F8C45EF4D00328F2DC0A4603F6C463617930BC06E530BC012243F03FBD00BFF8
:20B0E000883D002010B50C4C94F8843E022B11D1D4F88C0E42F006F9D4F88C0E08B12123F7
:20B10000C38001213DF004FDBDE810400348082143F002BC10BD00BF883D00200C4C002059
:20B1200073B50D4E05460C46FF230A46014630468DF8073043F012FD01230DF1070245F062
:20B140008001304643F0D8FC9DF80700031B5842584102B070BD00BF0C4C0020094B93F80F
:20B16000B234042B08D9053B032B08D801231A4600B103701046704700230122F8E700238E
:20B180001A46F5E7902C0020F0B40D6800240CE0BCF1050F18D8A0F137030A2B14D104EBE9
:20B1A000840415F8010B03EB4404A0F13003DEB2092EA0F16107A0F1410CF0D9052FE7D89A
:20B1C000A0F157030A2BEAD00D601460F0BC70479FED737A07EE901A20EE070AF8EE677A53
:20B1E00027EE800AFDEEC07A17EE903A2033402B00F2C780DFED6B7AB4EEE70AF1EE10FA98
:20B20000F0EE407A0CDD9FED686ADFED686AB0EE677AB4EEE67AF1EE10FA77EEC67AF6DCD0
:20B220009FED637AF4EEC77AF1EE10FA0CD59FED5E6ADFED606AB0EE677AB4EEE67AF1EE6E
:20B2400010FA77EE867AF6D49FED5B7AF4EEC77AF1EE10FA00F38D809FED587AF4EEC77AC7
:20B26000F1EE10FA44BF9FED527A77EE677A27EEA76ADFED535A9FED537ADFED536AA6EE2F
:20B28000257A67EE865AE6EE076AB6EE007AE5EEA67A27EE877ADFED486A70EE267ABDEE47
:20B2A000E76A16EE103A2033402B67D8B4EEE60AF1EE10FA0CDDDFED3C5A9FED3C6AF0EE1C
:20B2C000676AF4EEC66AF1EE10FA77EEE57AF6DCDFED376AF4EEE67AF1EE10FA0CD5DFEDC7
:20B2E000325A9FED346AF0EE676AF4EEC66AF1EE10FA77EEA57AF6D4DFED2F6AF4EEE67AF9
:20B30000F1EE10FA40DDDFED276A76EEE77A67EEA75A9FED2B5A9FED2B6ADFED2B6AA5EE89
:20B32000856A27EEA55AE5EE866AB8EE006AE5EE267A67EE867AC7EE206A00238361436185
:20B340000362C361B7EE006A76EE865A76EE666A86EE257A67EE277A66EE876AC0ED017A67
:20B36000C0ED037A80ED007A80ED027AC0ED046A70479FED0C7A77EE677A78E7DFED137AF1
:20B38000D9E79FED127A86E7DFED0C6AF4EEE67AF1EE10FA44BFDFED066A76EEE77AB6E75A
:20B3A00027D4D236DB0F4940DB0FC940E4CB1641DB0F49C0E4CB16C1DB0FC93FDB0FC9BF41
:20B3C00092E741B99730083C15A82ABE000000002DE9F047944C82B094F8C53E0190002BA0
:20B3E00040F01D8194F8E83EB4F8EA2EDFED8F6AB4F8EC9EA4F8FC9E07EE103AB8EEC76AC2
:20B40000B7EE007A07EE902AF0EE475AB4F8E62EE6EE665A4FEA49059542A6EE267AB8BF82
:20B42000154604F56F61F8EEE77A04F6F46267EEA67AC1ED005AAEB204F6F86182ED007A38
:20B440000122A4F8FE6EC1ED007A84F8C52E002B00F0E180DDED017A9FED750A754FF8EEB4
:20B46000677AADB280EE270A5EF084FB6D00B0FBF5F5012DB8BF0125EDB2B0FBF5F39BB2D4
:20B48000804684F8005F00EE103ABBEEED0A87ED000A5EF06FFB684BDFED686AB9FBF0F018
:20B4A000A3FB08384FEAD80807EE908AF8EEE77A022886EEA77AB8BF022084F8080F07F15C
:20B4C0000C0100239FED5E1A9FED5E6ADFED5E1ADFED5E5A9FED5E2ADFED5E2A9FED5E3A90
:20B4E000DFED5E3A9FED5E4A87ED027A07EE903AB8EEE77AF0EE467AE7EE017AFDEEE76AD4
:20B5000016EE902A2032402A00F28280B4EEE17AF1EE10FA0CDDDFED536A9FED537AB0EE6E
:20B52000675AB4EEC75AF1EE10FA77EEE67AF6DCF4EEE57AF1EE10FA0CD5DFED4A6A9FEDF0
:20B540004B7AB0EE675AB4EEC75AF1EE10FA77EEA67AF6D4F4EEC67AF1EE10FA50DD74EE32
:20B56000677A67EEA76AF0EE624AE6EE824AF0EE430AE6EEA40AB7EE007A27EEE65A77EED4
:20B58000677AB6EE007AE5EE207A67EE877A0133202BE1EC017AA9D107EE905AF8EEE77A82
:20B5A000F7EE006A86EEA77A314B324A41F2AC5741F2A851E35141F2B85003F12807675004
:20B5C000A83341F2094107EE906A2350F8EE677A41F2A45741F2B45041F2B0536554102660
:20B5E00020251421E6532552E15282ED007AC2EDAC7AC2EDAD7AC2EDAE7A02B0BDE8F087B5
:20B60000F4EEE37AF1EE10FA48BF75EEE77AA8E7F6EE007ABBE7184A82F834321AE794F8D9
:20B62000005FB4F8FE6EB7E7883D00200AD7233C002474498C4C0020ABAAAAAADB0FC9415A
:20B640003C8C4F3EDB0FC93F0100F840DB0F49C092E741B99730083C15A82ABEDB0FC9BFE2
:20B66000DB0F4940DB0FC940E4CB1641E4CB16C1CCC306089451002098010020084800230A
:20B6800002461178022902F1060204D00133062BF7D10020704703EB430300EB43007047C2
:20B6A000D01B002010B50021094C82B00846C4F8E01533F05BFE074B0193042304F2E45060
:20B6C0000DEB0302062143F0E7F902B010BD00BF804E00205475C52A70B5461E00F131059F
:20B6E000344614F8011F601E801BFF29C0B201D033F03CFEAC42F4D1A02051F087FD012169
:20B70000022033F033FE0E4D40F2E93401E0013C05D04221284643F06DF90028F7D1622139
:20B72000074843F067F91321242033F01FFE2520092133F01BFEBDE87040A02051F066BD4B
:20B74000645400202DE9F04F2DED108B034697B004331593DFEDCACA149002238A461392FA
:20B760008B461293149C4FEADB0604EB461202EB06103101A6EB86034FEAC60806EB4605B0
:20B78000CDE9000100EBC303043108F104001196204421442C01C6EBC60C0394EC00119DBE
:20B7A00004944FEACC0405946C0106EB860E0294159D009C03EB46174FEACE0E02EBC60660
:20B7C0004FEACB094FF0000C51ED01AAD3ED001A92ED007A94ED005A96ED004AD7ED007A6F
:20B7E00015ED012A50ED016A32EE07BA76EE840A7AEE855A31EEA70A3BEE256A70EE804AAA
:20B8000076EEC46A36EE244A36EE646A05ED014A82ED006AD0ED00BAD6ED012AD3ED019A3C
:20B8200095ED00AA92ED016A97ED013A91ED00CAD4ED014A7BEEE23A36EEE19A32EE472A2A
:20B8400073EEE98A3AEE464A39EE279A78EE838AB0EE428AA9EE6C8ADC44E24573EEC33A65
:20B86000B0EE441AA8EEEC1A76EEE77A33EEA97A7CEE643A77EEA17A3AEE066A7AEEC51AC0
:20B880003CEE24AA74EECC4A39EE833A35EE6A5AF0EE639AF0EE48AAE7EE2C9AA8EEAC4A9B
:20B8A000E7EE2C4AE7EE6CAAF0EE418AB0EE427AB0EE612A7BEE656A7BEEA22A76EE4A5AB1
:20B8C000A9EE2C7AA7EEAC2AA7EEAC5AE7EEEC8A32EE83BA76EEC3BA35EEE09A75EEC07A62
:20B8E00036EE0A6A76EEE26A36EE0BAA76EE836A77EEA07A34EE423A77EE290A36EE4B6A48
:20B900007BEEA22A39EE000A73EEAA3A78EE244A37EE697A31EE055A71EEA85A32EE044A53
:20B9200085ED00AA82ED016A4D4441ED012A4A44C4ED006A81ED000AC4ED017A494440ED20
:20B94000010A4C4487ED007AC6ED003AC3ED004A80ED003A87ED014A484486ED015A4F4424
:20B96000C3ED015A4E444B443FF62EAF119B072B40F2C781029D149E019B03980499059A6D
:20B98000083575190C330E95354608F108080EF10804EB1808300831083246442C192818AE
:20B9A0006918AA18079305F10C030D960C940B900A91099208934FF001084FF0000E129BB4
:20B9C0009E44139B03EBCE0303EBCE02109302EBCE0303EBCE01029101EBCE0101EBCE052F
:20B9E00005EBCE06D6ED007A0F93AEEB8E03019106EB031303EBCE07D3ED01AACDED067A79
:20BA0000019BD5ED007A97ED01BACDED057AD3ED007A029BCDED047AD3ED007A0F9BCDED29
:20BA2000037A07EBCE0CD3ED007ADCED01BACDED027A0CEBCE01D2ED007A109A009101EBA3
:20BA4000CE00014691ED01DACDED017A0099D2ED007A91ED01CA00EBCE0000EBCE0494ED31
:20BA600001EAD0ED01DACDED007ADDE90776DDE90954DDE90B01DDE90D23C44602E000BF36
:20BA8000F304353F94ED009A90ED00FA91ED006AD5ED007AD3ED006A57ED014A92ED005AF3
:20BAA00056ED013A96ED00AA35EE060A73EEA65A39EE278A34EE8F7A70EE082A75EE87EAE0
:20BAC00035EE465A3EEEA26A73EEE63A06ED016AD1ED019AD2ED01FAD4ED016AD3ED011A72
:20BAE00095ED013AD0ED018A97ED004A3FEEE96A35EE491A76EE660A31EE271A3AEE612A86
:20BB000075EE677A70EE830A3FEEA95A74EECF9A77EE897A7AEE211AB0EE42AA74EE68FAA2
:20BB2000A0EEECAADC44E24535EEC77AB0EE639A74EE285A38EEC44AF0EE698AA1EE6C9A1D
:20BB4000E7EEAC8A36EE436A7FEE644A36EE266AA0EEAC2AF0EE4A0AE7EEEC0AE7EEAC4A0E
:20BB6000F0EE687AF0EE498A36EE833AE6EE6C8AE1EE2C3AB0EE6F1AA6EE2C1A71EEE56AC5
:20BB8000A6EE2C4A71EEA55A75EE031A7EEEE22A37EE43FA75EEE1EAB0EE686A76EEC08A97
:20BBA00039EE044A7FEE86FA76EEC86A33EE816A38EE888A73EEC13A37EE457A2CEE2E1AA7
:20BBC0003FEE055A22EECC9A9DED03FA70EE266A33EE077AAFEE221AAFEE2E9A7AEE244A38
:20BBE0009DED01FA79EEA09A25EE4BAA72EE670A37EE822A6BEE087AAFEE08AAEFEE057AEF
:20BC00002DEEA63A9DED05FA67EE6D8AAFEE073AEFEE268A66EE6A2A9DED00FA2AEEA00ABB
:20BC2000EFEE202A6EEE02EADDED060A23EECE5AE0EEA3EA2BEEA98ADDED023AAFEE060A28
:20BC4000A3EE848A24EE6B7A6DEE246A9DED044A2FEECD6AA0EE825AA3EEA97AE4EE2F6AB0
:20BC6000A4EE246A75EEA15AC6ED005A83ED001A83ED019A4E4447ED017A87ED00AA4B44B6
:20BC800080ED003AC0ED018A4F4482ED000A4844C2ED012AC5ED00EA85ED015A4A44C1EDAE
:20BCA000006A81ED016A4D4484ED008A84ED017A49444C443FF6E6AE0E9B08330E930D9BB6
:20BCC00008330D930C9B08330C930B9B08330B930A9B08330A93099B08330993089B0833B3
:20BCE0000893079B08330793119B08F1010843457FF465AE129BDDF844B0DB009BB2129333
:20BD000030E517B0BDEC108BBDE8F08F30B5044683B000BF806841F0EFFA4CF2050301AACB
:20BD20006946ADF800306068032300258DF802505BF012FAA06841F0E5FA00BF9DF80600CC
:20BD400003B030BDF0B5BE4FBE4885B02422002160F075FA97F8F165002E3AD1BA4C354691
:20BD6000D4F8443D5BB39B6A4BB3B848984783682BB30388DFF8CCC2013B9BB260466646F2
:20BD800000213778032F06F106061BD001310629F7D100220178022900F1060000F0A580B8
:20BDA0000132062AF6D1E16D052908D0481C02FB01C2E06502200021938010705180284687
:20BDC00005B0F0BD062303FB01414B8F013B9BB2DFE797F8F00507F5BF63C7F8F43510B91C
:20BDE000994C0025BCE740F097FF0446C7F8000641F066FA05460028F2D0013E022370B275
:20BE000087F8F83542F014FF0028E9D0C7F8FC050CB12023E380204609213CF079FED7F82B
:20BE2000F435894C986841F06DFAD7F8F435102158685BF05FF9864BD7F8F425C4F8642DDA
:20BE400093E803000123009032208DF8041084F8683D00263DF0AAFB052302AA6946D7F85A
:20BE6000F4058DF80A608DF8096042F08DFD9DF80A009DF809109DF80B20764B000240EA36
:20BE800001401043984200F0AE8032DCA3F5F11398425ED042DD704B984252D0023398427F
:20BEA00062D14FF400724FF48073A4F8482DA4F8543DB4F8542DB4F8483D120202FB03F3C1
:20BEC00000204FF48071B3F1807FC4F84C2DC4F8503D84F8560DA4F84A1D7BD85F4BC4F852
:20BEE000443D012284F85D2D3AE7062101FB02C260E75B4B984234DC053B984234DD594BEA
:20BF00000344032B77D801A252F823F053BF000843BF000835BF0008A3BE0008A3F5220317
:20BF2000013B984267D051DD4F4B984209D00133984219D14FF48073A4F8483DA4F8543DBD
:20BF4000B7E780224FF48073A4F8482DA4F8543DAFE740224FF48073A4F8482DA4F8543DC1
:20BF6000A7E7424B9842E5D00023A4F8483DA4F8543DC4F84C3DC4F8503DFCF727FC0346B9
:20BF800000287FF4EDAE9DF80B009DF80A209DF80C10000240EA0240354A0843904232D04F
:20BFA000A4F8483DA4F8543DC4F84C3DC4F8503DFCF70CFC064600287FF4D2AE97F8F005BF
:20BFC00040F0AAFE42F088FC3546C9E6294B9842B0D0C9E70123D4F8640D84F85C3DB721DD
:20BFE00050F01CFD7AE74FF480621023A4F8482DA4F8543D5DE720224FF48073A4F8482D24
:020000040800F2
:20C00000A4F8543D55E71C4BC4F8483D4FF4003140234FF000620126A4F8543DC4F84C1D1E
:20C02000C4F8502D84F8566DFCF74AF8074884F85D6D50F045FC114BC4F8443D90E600BF6F
:20C04000804E0020D01B0020981B0020DC280020F4C406081640E0001720C200E0C206084B
:20C060001940EF00EABF10FF17BA20001870EF0021AAEF0018600100000400080CC306083C
:20C080002DE9F041C54BC64EC64DC74C0822C3F88820336B82B043F00103336307464FF455
:20C0A000C052284640F2023388466946CDE9002308F09CFA6B6AC4F8E88B23F470436B621A
:20C0C0006B6AC4F8F07B43F420436B626B6AB749C4F8EC1B23F470236B626B6AB448C4F861
:20C0E000040643F420236B62736CB249C4F8081643F480437364736BAF48B049C4F81406C6
:20C1000043F0800302257363AD4F84F80C56AD4EAD4DC4F858164FF0A043C4F81036AB4A5A
:20C12000C4F8207603F53463A1F5D071C4F85C56C4F82466C4F86036C4F828160123DFF84C
:20C14000BCC2C4F81CC607F51077A5F5E465A6F5A066A1F58C61C4F86476C4F81856C4F8BD
:20C16000D06684F80F3605F5A075536106F5B076C4F8941684F816371946954B954AC4F8DB
:20C180009C56A7F5BC67A035C4F8A866924EC4F8A476C4F8AC3607F5D45703F56953C4F864
:20C1A000B0564FF050250020DFF854E2C4F8D426ACF5687C02F5A042C4F8D876C4F8DC667C
:20C1C00007F5A04706F5A046C4F8E036C4F8E456A3F5485304F20465C4F8E826C4F8F06665
:20C1E000C4F81037C4F898E6C4F8A0C60246C4F8EC762B4684F81807402683F81C21A3F8B5
:20C2000022210132042AC3E9496083F81D1183F81F01C3F8300103F12803EED1002211469E
:20C220002B46402083F87423A3F87A230132042AC3E9DF0183F8751383F87713C3F8881398
:20C2400003F12803EED14FF0A04364489A6822F001029A60DA6842F04002DA6007F084FABC
:20C2600094F80D360022212161F317420BB142F4801294F80716D4F8103601299A6300F088
:20C28000E480DA68D4F81067D4F81406C2F3076121F0600141F0400161F31F620021DA609E
:20C2A0003160026861F3CC22026094F80F26012A00F0B88010214A4807F0A8FD484807F0E5
:20C2C0008BFDD4F8140694F8053600224FF0FF31026142618161C26153B305F11407414EE7
:20C2E000114607EB83074FEA830C4FF0FF0E56F8042F1368002BACBF00234FF09043B74297
:20C3000013601161C2F808E0F1D105F15003364963440027FF2651F8042F1568002DACBF88
:20C3200000254FF090459942156017619660F2D1036994F8071643F480730129036161D045
:20C34000D4F8102629480023936100294FF0FF336FF0804151615360516114BF0023102359
:20C36000906143F470139069D4F8EC1B43F4605343F00803034393619368096843F0010341
:20C38000936088471A4B1B4ADA6068461A4B0093FEF704F802B0BDE8F08100BF00E100E0F8
:20C3A0000038024000000240804E0020D0030020080401004000400100080050000B00509F
:20C3C0002009005040090050200B0050003C0140C00500500010005000300050905400205A
:20C3E0008454002098540020D45400200008008000ED00E00005FA054302000100090050F9
:20C4000020050050D4F81026144B03636FF08041134D00234FF0FF309361516150605161C7
:20C4200095619EE701680F4A0F4E41F003010160802159629E62C3F80421E022C3F80821AA
:20C44000C0F24002C3F80C2134E79A6822F03E0141F02A0161F307029A6012E70301810061
:20C4600000080080A00040008000200010B51A4C94F8FA0BC0B9194B83F8B100C3F8B40080
:20C4800094F8FD3B012B05D0022B21D0D4F8003C1BB910BD124BC4F8003C12495B68BDE8F8
:20C4A0001040A1F10C00184740F036FC94F8FC2B0A49003A18BF012281F8B120C1F8B400DC
:20C4C0000028DDD01F22C28020213CF021FBD7E7054BC4F8003CE0E7804E0020981B0020ED
:20C4E00010040020845A0020EC03002099B10A6B824216D9154BD3F8442C914221D34C39A2
:20C5000091421ED30B6B9842F9D38B6B9842F6D80B46184670470D4BD3F8441C0A6B90426D
:20C5200012D30B680BB9F4E70A6B90420B4602D38A6B9042EDD951F84C3F002BF4D11846E8
:20C5400070470023184670470A46D8E7804E00202DE9F047CC0143D10346224A43F8082B9E
:20C560004FF0FF324260022418467E26DFF87880D8F8489C2644013E051D49466FF070478E
:20C580004FF0010A08E0A3421CD0631C45F8043C321B1C460435CAB10B6BA34202D88B6B0E
:20C5A000A34204D22046FFF7A1FF014690B10A794B6B002AE7D1A34204D0E6D245F8042C43
:20C5C000631CE5E745F8047C631CE1E7C8F8481CBDE8F08745F804AC321B631C4946D8E7C5
:20C5E0008026C3E7F8FFFF0F804E0020036870B55E6A26B133460522BDE87040184704462B
:20C600000D464E1D00E023689B68204698470028F9D0236815F8011B1B6820469847B54245
:20C62000F1D170BD036870B55E6A26B133460822BDE87040184704460D4601F1080600E008
:20C6400023689B68204698470028F9D0236815F8011B1B6820469847B542F1D170BD00BFF5
:20C660002DE9F047164D0746002095F9559C05F65C4684B007EB010805F6FC6504464FF06D
:20C68000B60A3368ABB193F83830142B11D019F1020F01D04B450CD1002269463046CDE97A
:20C6A0000244CDE90078ADF808A08DF80E4034F085F8E036B542E4D104B0BDE8F08700BFF4
:20C6C000804E00202DE9F743124E0124A02318255FFA84F8FF2B14DCD6F8FC0EE9B2C1F183
:20C6E0001C0282725F1C026880F80B80DBB20093C1F11B01D2F8189000234246C9B2C847AB
:20C700003B46013DE6D10134052CE0D103B0BDE8F08300BF804E002010B50A4C94F8190F45
:20C72000003818BF0120FBF777FF50B1064904F5706042F061F804F570600FF00BFF04F5F2
:20C74000706010BD804E0020FCC4060870B4447941BB03684FF400524FF400762025022182
:20C760003CBB1A8C22F001021204120C1A841A8B188C22F0F30280B2120420F00A00120C65
:20C78000014342F0010241F001011A8319841A8B22F00C021204120C1A831A8B92B270BC08
:20C7A0001A83704700220368164615461146002CD7D0042C21D0082C38D0198C21F48051CF
:20C7C0000904090C19849C8B1D8C45F6FF7040F6FF4128402140024342F4805241F480716E
:20C7E00099831A849A8B22F440621204120C9A839A8B92B270BC9A8370471A8C22F010021E
:20C800001204120C1A84188B198C89B240F6FF4221F0A00102400D4342F4807245F0100596
:20C820001A831D841A8B22F44062B3E71A8C22F480721204120C1A84998B1A8C21F0F30174
:20C8400092B2090422F42062090C324342F4807241F0010199831A849A8B22F00C02C4E760
:20C8600038B50F4D0446006807F0C4FDD5F87828204652084FF6FF713BF0CEFD20460021A6
:20C88000FFF764FF41F2E403064AEA5005F5875120460022BDE8384004313BF0DDBC00BF6C
:20C8A000902C0020F1C601082DE9F0479AB0DDE9226ADDF8909004460D461746984602E044
:20C8C00020683DF091FA20683DF096FA0028F7D10146642201A85FF0B2FC264B8DF8045026
:20C8E000CDF85CA00293002D40D0AB1E012B3FD9042D14BF002203221F4B0396D3F8003946
:20C900008DF805201E440123CDE9059404968DF85B3037B14246394607A85FF02FFC8DF851
:20C920005A80164E96F86A9F00231893B9F1000F19D196F8690F642202FB006001A900F628
:20C940006C705FF01BFC012386F8699F86F86A3F236843B143463A46294620461AB0BDE8F8
:20C96000F04712F007B91AB0BDE8F0870522C3E70222C1E7A85D0020981B0020804E002055
:20C980000C4B0D4AD3F8EC1F0C4810B40C4CC3F8DC2F8A1E223123881B01A0FB03C3DB08D7
:20C9A000A3F5B06322F8023F9142F4D15DF8044B704700BF804E0020B1210208CDCCCCCCC4
:20C9C000865E002070B5084C251D2E4614F8010B34F0C4F828B1037805F8013BB442F5D1E3
:20C9E00070BDFF23F8E700BFA85E00202DE9F0471D4F012607F10805B2464FF03C094FF084
:20CA0000000817F8010B40F087F9044690B180F80690C671FB7803F07F02012A18D013F076
:20CA2000800F20460DD185F8048040F065FC85F805802C600136052E05F10805E1D1BDE83F
:20CA4000F08785F804A040F05DFC85F805A0F0E71B0605D4012120463CF05AF8FB78DEE784
:20CA600040F050FCF6E700BFB05E00202DE9F04FDFF8E491DFF8E4A183B009F10C05012410
:20CA800019F8018BB8F1000F00F0C0804FEA1817013F042F08F00F0200F2BB800AEB4703C1
:20CAA000B3F8B00040FA02F616F0010600F0C38001239340013B184057445BF025FF97F885
:20CAC000BC305F4E184406EBC00604236E61F471B371002303E00133152B00F09780594908
:20CAE00003EB43025F00895C4145F4D1564B1A4492F88D15002900F0A08040463BF0EEFD74
:20CB0000804600683BF08EFD98F805103BF006FE0378002B7AD14C4B3B44042283F8CD45A3
:20CB200083F8CC25002E58D0336898F8080003F13F4202F57E020AEB9222012792F8C420D5
:20CB400002F01F015209032A07FA01F169D0042A62D0022A6AD0B6F804C0BCFA8CF2C2F1F0
:20CB60001F02C2F3CC0103EB810102F007020E6A92000F27974026EA07060E620E6A9040BB
:20CB80003043002208624FF0010B11460BFA01FE3EEA0C001CD118680326964020EA060040
:20CBA00018601F6802209040384318609F6827EA06079F6098689860586820EA0E005860E5
:20CBC00058685860D86820EA0600D860D868D8600131102902F10202D8D11C4B1C4A33F8DA
:20CBE000A01C33F89E3C0091002001340190B2FBF3F328469BB24146E4B233F04DF8012306
:20CC0000092C6B7405F118057FF43AAF03B0BDE8F08F00266E615CE70E4F3A6B0A433A6396
:20CC200099E70C4A176C3943116494E7094A576C394351648FE76E614BE70B68FFDE00BF62
:20CC4000883200201C320020902C0020785F002040420F0000380240DC5E0020E0C20608A4
:20CC600070B5044684B04FF4004035F01FFC48B300234FF4E131032590F904000293CDE9DB
:20CC800000151A464FF4004135F071FC0E4B1863C0B1012C40F698020C480D4D83F834402A
:20CCA00008BF4FF496624FF461710A269A87094A9E63C3E91150D987A3F84010DA64012001
:20CCC00004B070BD0020FBE7785F00208DC70108698601085D8601082DE9F041204E214F14
:20CCE00096F86F3087F858316C3607F5AE7500244FF0050816F8010B20BB28600134032CED
:20CD000005F10405F6D197F85811D7F85C01C94301F0010140F0FCFA97F85811D7F86001DC
:20CD200081F00201C1F3400140F0F2FA97F85811D7F8640181F00401BDE8F041C1F38001C1
:20CD400040F0E6BA3FF0E8FF013401212860E3B210B180F80680C37128683BF0D9FECEE73F
:20CD6000785F0020883D00202DE9F0412A4C2B4DB4F87460A5F8686182B0EEB994F87000E7
:20CD80003FF0CAFF94F87120C5F86C01003A18BF012285F86A2148B194F872102B2200299B
:20CDA00014BF11210121C2803BF0B2FE002002B0BDE8F04141F0EABA94F87080002240468E
:20CDC0002B213BF0FBFC074640463FF0A5FFF8B1F7B12B22C5F88401C280397AFDF71EFB5D
:20CDE0004FF000080E4AB2FBF6F3C3F34F0000909BB23946CDF8048005F5B870A4F87660C0
:20CE000032F04AFFD5F87031C3F8008085F8818102B0BDE8F08100BF785F0020883D00201C
:20CE200040420F002DE9F84F244C94F8843084F8783004F17B07002698345FFA86FB0BF1F1
:20CE400001085FFA88F8012117F8010F42460E448A463BF0B3FC4FF00009054640B33878F5
:20CE600004F80E9C04F80D9C04F80FBC04F810AC44F8045C3FF050FF18B180F806A080F86F
:20CE80000780297AFDF7CAFA0D4A002128463BF0C3FA0C4B23600C4B221D21462846C4E9F0
:20CEA00001393BF0D9F9697928684A4632F010FA082E04F11C04C0D1BDE8F88F785F00200E
:20CEC00040420F0009F30308715D030870B52B4C2B4B94F8B001C4F8A83100220221C4E90B
:20CEE0005A22C4F87021C4F8A421A4F8AC213BF065FC002841D0234B0268054603F1C000E3
:20CF0000597C11B159688A422BD018338342F7D1002394F8B001C4F8945084F888303FF0B7
:20CF2000FBFE08B10223C380297AFDF777FA2846154A00213BF070FA144A1549C4F898102C
:20CF40000026111F2846134BC4F89C30C4F8A0603BF082F9697928683246BDE8704032F064
:20CF6000B7B9138D0C490D4A9BB2D2F878280133B2FBF3F381F89C32CAE770BD785F00205B
:20CF800000FFFF005C31002040420F0014600020995D0308395F030898010020902C002088
:20CFA0002DE9F04FDFF8FCB2B14D83B00E460446C0220BF2CC40002100965FF040F995F811
:20CFC0001C32002B6FD095F81D32002B00F08A809BF8C034012B00F0AD80022B00F08E809D
:20CFE000A44BA54E01931C460FCE0FC40FCE0FC49BF8B6749BF8B23496E807009F4EC5F894
:20D0000000623E1E18BF0126072B84E8070085F8256200F20381042B00F20D81DFF88882A5
:20D020000026A8F1150A009B5FFA86F909F10107FFB2B3423A464FF0030129DD1AF8014BD0
:20D0400020463BF0BBFB034620461C4613B33FF063FEC8F8140018B14FF003038371C77114
:20D060009BF8B3349BF8B224002B00F0E280E37983F0010349462046013657F069FD48B1AB
:20D080004FF00103082E88F8113008F11808CAD1019B06E07A4B7B4AC5F80C32C5F80422B8
:20D0A0000023C5F82032D5F8203263B10022009883F82C00012183F82D101A6383F82E208A
:20D0C00003B0BDE8F08F704E704C0FCE0FC40FCE0FC496E80700A4F1200384E80700C5F832
:20D0E0002032EDE79BF8B4240099003A204618BF0122FBF761FDC5F82002D4E79BF8B63405
:20D10000002B3FF46DAF9BF8B234082B12D15A4E5A4F0FCE05F5F47401940FC40FCE0FC45E
:20D1200096E80700012384E8070085F82532C5F8007276E0564E009BC5F828320FCE554CA6
:20D14000DFF864910FC40FCE0FC49BF8B63496E80700003B18BF01239BF8B26485F82532CB
:20D160000027A9F1150384E8070085F868629834019385F826720AE040F0BEF8E368C9F8CB
:20D180001430082F04F1200409F118094DD0D5F82832BB4249DD019B13F8018B019340462C
:20D1A0003BF040FB064640463FF0B6FD9BF8B32496F8078082460AB188F0010808F00106D3
:20D1C00095F82522013685F824620AB188F00108504640F075F800283DD0504641F014F9C9
:20D1E0007101013741F0090161616060C4F80CA084F81080FAB2BAF1000F05D04FF00303D4
:20D200008AF806308AF8072050463BF081FC18F0010F5046B0D140F075F8AFE7082B7FF467
:20D22000FDAE1D4BC5F82C32F8E61A48C5F8200239E7E3791EE79BF8B534184AC5F82C2237
:20D24000012B05D0022B06BFB7FA87F35B09002385F83032E2E60B4B1149094AC5F8D031C1
:20D260000123C5F8CC11C5F8D82185F82632DDE7785F00206061002078C506085D260608ED
:20D2800079630408816304084CC50608AC610020A4C506082C610020C1630408F1630408B6
:20D2A00085630408902C00205C3100202DE9F047734F07F5805941F2010399F80000FD5CEC
:20D2C0003FF02AFD60B12D23C380202104463BF01FFC0A203CF04CF8204641F08BF828B9EE
:20D2E000DFF8A4A1DAF86C33DA0001D5BDE8F087013D092DFAD897F8FF4FD4B9402035F0A0
:20D30000D5F80028F2D090F9043097F8D51F092BC8BF143B53440A2993F8704300F0A280F2
:20D3200093F87C3397F8FE2F002A08BF1C46002CDCD020463FF0F0FC0546002800F08A80DE
:20D340002D23C38001213BF0E3FB012108463FF0E7FF2B68AA881A833C203CF027F900215F
:20D3600001203FF0DDFF41F20103FB5C002B4ED0444CDFF8188100261FE02B68AA885A83E3
:20D380003BF0F6FF94F85811D4F85C0101F001013FF0BEFF94F85811D4F86401C1F3800115
:20D3A0003FF0B6FF2B68AA881A8378203BF0E0FF98F8003001369E4229DA94F85811D4F8EA
:20D3C0005C01C94301F001013FF0A2FF94F85811D4F8640181F00401C1F380013FF098FF8A
:20D3E0007820002DC9D178203BF0C2FF94F85811D4F85C0101F001013FF08AFF94F858118C
:20D40000D4F86401C1F380013FF082FFCDE797F8FF3FBBB999F80030002B7FF467AF41F259
:20D420000203FB5C012B7FF461AFDAF86C3313F080537FF45BAF41F20102BB54BDE8F047FC
:20D440004AF008BD32203CF0B1F8284600213BF05FFBDFE701213BF05BFB012108463FF08A
:20D460005FFF79E7DAF894335B057FF53FAF09F083FF00287FF43AAF002C7FF45AAF35E7D0
:20D48000804E0020883D0020785F0020815E0020084BD3E9E6029042D3F8A03302DC114627
:20D4A00002460846984204DD9A42B8BF1A46104670477047785F0020124AD2E9E9039842D0
:20D4C00030B4D2E9EB41D2F8B42302DC1D4603462846914202DC15460A4629468842A8BFEC
:20D4E00008469342B8BF1346844202DB224604461046984203DD9C422046B8BF184630BCCF
:20D50000704700BF785F00200B6810B414681B1B036054684B681B1B43608B6892685DF8C8
:20D52000044B9B1A836070472DE9F047041E0D4612DB092C26DC824A0B468248A0FB0410D1
:20D54000C00800EB8000A4EB40000021125C1A7059702846BDE8F08764422D23092C01F839
:20D56000013B24D8764A774BA3FB0403DB0803EB8303A4EB43030020D35C48700B70284630
:20D58000BDE8F0876F4B632CA3FB04264FEAD60621DC6B4A0B466B49A1FB0601C90801EB32
:20D5A0008101A6EB4101515C03F8011BC5E7654A632CA2FB04364FEAD60637D8604A614B17
:20D5C000A3FB0603DB0803EB8303A6EB4303D35C01F8013BC7E7A3FB0627B4F57A7F4FEABE
:20D5E000D7070DD2564A0B465649A1FB0701C90801EB8101A7EB4101515C03F8011BCAE7B2
:20D60000A3FB072842F20F7294424FEAD80836D84B4A0B464B49A1FB0801C90801EB81012D
:20D62000A8EB4101515C03F8011BDDE7A2FB0637B4F57A7F4FEAD7070CD2414A414BA3FB67
:20D640000703DB0803EB8303A7EB4303D35C01F8013BB4E7A2FB073842F20F739C424FEAE9
:20D66000D80821D8364A374BA3FB0803DB0803EB8303A8EB4303D35C01F8013BDEE7324A51
:20D68000A3FB080994424FEAD90921D82C4A0B462C49A1FB0901C90801EB8101A9EB4101FA
:20D6A000515C03F8011BB5E7274BA2FB08099C424FEAD90921D8224A224BA3FB0903DB0892
:20D6C00003EB8303A9EB4303D35C01F8013BCAE71E4AA3FB090394424FEAD30A21D80B469F
:20D6E0001849174AA1FB0A01C90801EB8101AAEB4101515C03F8011BCAE7144BA2FB09022F
:20D700009C424FEAD20A13D80E4B0D4AA3FB0A03DB0803EB8303AAEB4303D35C01F8013B3A
:20D72000CAE70A22BAFBF2F049F086FE0346D7E70A22BAFBF2F049F07FFE0146E4E700BF67
:20D74000A0710708CDCCCCCC9F8601003F420F0070B4344890F8B833A3F13001092957D889
:20D7600000F56E74224600F2C73012F8015FA5F13001092904D88242F7D1002070BC7047B3
:20D78000141B022C4ADD2848002101E010F8013B01EB810103EB4103161A303B022E04469A
:20D7A00003F0FF01F2DC214B03FB01F1A2424FF000030DD903EB830314F8016B5B00303B8E
:20D7C0003344A24203F0FF03F4D1194800FB03F32E2D06D01748A0FB032301EB930070BCE6
:20D7E0007047013204200024157804EB8404303D6400092D00F1FF30A4B202D82C44A4B2D6
:20D80000013210F0FF00EFD1642202FB0433E1E700211D4600F56E720B46D9E7064C0021B7
:20D82000C4E700BF785F0020316300208096980040420F00ABAAAAAA3063002038B5044601
:20D840000D460A460068FF215EF0F9FC21682944216038BD83B50C461646054633F0ECF9B5
:20D86000204633F0E9F90021204B0846002E08BF1E463FF055FD002101203FF051FD28465C
:20D880003CF0BAFAB0B1012100203FF049FD28463CF0AAFA074620463CF0AAFA0028FAD0DD
:20D8A000394620463CF0ACFA3846B047002108463FF036FD20463CF09FFA0028DFD0012147
:20D8C00000203FF02DFD20463CF08EFA0146284601913CF08DFA01990028F8D028463CF097
:20D8E0008FFA002108463FF01BFDC8E771F50308F0B500230B604B608B60CB600B610268FF
:20D90000DFF88CC089B004ADC2F385572E4647FA03F0C007344604D513F80C0004F8010B88
:20D9200026460133062BF2D11748C2F303240444002394F8F84233708DF8184000F5407CB6
:20D94000C2F305370DF1190647FA03F0C007344604D513F80C0004F8010B26460133062B7B
:20D96000F2D100233370C2F3834406ABCDE90134084602F00F0305490095C2F303124EF0C9
:20D9800043FA09B0F0BD00BFE0C20608C8710708D0C5060870B5094CD4F8C823054662B1FB
:20D9A0000026D4F8C8032D21013641F0BFFAAE42F7DBBDE8704042F0FFBC70BD785F002013
:20D9C0002DE9F04F5FFA81F9002185B00746084616463FF0A5FC002101203FF0A1FC3FF0C5
:20D9E00079F9022E0AD0042E44F6C01818BF4FF49648B9F1070F07D900200CE0B9F1FF0F0B
:20DA00004FF41648F5D10326CD4D95F8CC332BB90020C5F8D00305B0BDE8F08F032EC94C1D
:20DA20000DD0A144002299F8B70403213AF0C6FE0028EDD0C4F8C008C3799A07E8D441F26F
:20DA4000DB0395F8CC03E654002203213AF0B6FEC4F8C40C0028DBD04FF48061BA4BC4F8EA
:20DA60007C38C4F888180323C4F88C1841F2CC01A4F880380023635441F2C8014FF0010A9C
:20DA800024F801A041F2D401B04A635041F2D80102F14800635241F2DA01C4F89008032E85
:20DAA00002F24C406354C4F88488C4F8A838C4F89C38C4F89838C4F89408C4F8A438C4F803
:20DAC000A03891460ED0D4F8C0B89BF804003FF023F9C4F8BC08584612F04AF9514648460B
:20DAE00012F05AF932203BF061FD002E60D1D4F8C48CD8F8000006F07DFC4046944A222195
:20DB00003AF08AFC9349944B0B60324640463AF0A3FBD4F8C088D8F8000006F06BFC8C4A52
:20DB20004FF6FF7140463AF077FC31464046FEF70DFE41F2E403894AE25009F66801324611
:20DB400040463AF089FBC5F8D0934FF0060A022E12D0D5F8D0033CF04FF968B101210020A1
:20DB60003FF0DEFBD5F8D0033CF046F90146002840F09E803FF0D4FB38463CF03DF988B1BE
:20DB8000012108463FF0CCFB4FF0050B4FF0000838463CF031F90146002840F092800120E3
:20DBA0003FF0BEFB042ED4D005203BF0FFFCCEE7012E09D1D4F8C40C4146FBF7EBF9D4F8D9
:20DBC000C008FEF74DFEBEE7022E09D1D4F8C00812F0BDF8D4F8C40C4146FBF7DBF9B2E7C1
:20DBE000032E5DD14FF0000A41F2DC0351465C4804F803A040225EF022FB8DF80FA0DFF8B9
:20DC000064A19DF80F30072B09D95048012112F0C3F8D4F8C40C4146FBF7BCF993E79DF8C7
:20DC20000F3003EB430304EBC30393F8DD3483B39DF80F3003EB430304EBC303D3F8E0344E
:20DC40003BB39DF80F30234493F8B70408B3002203213AF0B3FD8346D8B112F078F89DF821
:20DC60000F309AF8002003EB430304EBC30305EBC201D3F8E034C1F8D4339BF80730DB07CC
:20DC800048BF012302F1010248BF81F8D8338AF800209DF80F300133DBB28DF80F30B0E746
:20DCA000042E7FF450AFD4F8C00812F050F881E7D5F8D0033CF098F8014638463CF0A0F895
:20DCC00050E738463CF090F895F8223401468BB9242803D14FF0010385F82234012E04D133
:20DCE000384601913CF08CF80199D5F8D0033CF087F84DE7012B06D14D280CBF02230023C0
:20DD000085F82234EAE7022B06D13C280CBF0323002385F82234E1E7032B25D10A2802D917
:20DD200085F82284DAE7042385F8150485F8148485F8178485F8160485F82234CEE700BF37
:20DD4000785F0020902C0020E8C506080C35002040420F00703D002025FE01080DC601086E
:20DD60004C6300206C3D0020042B09D195F8163485F82304434085F8163485F822B4ADE756
:20DD8000052BABD195F8143495F8159495F816044B4509D25A1C2B44484085F8160485F839
:20DDA000142483F8181499E78842B9D195F8233485F822A4F42B91D1B9F1000F8ED12421AB
:20DDC000384685F822943CF01BF84D2138463CF017F83E2138463CF013F8494638463CF0DF
:20DDE0000FF8F42138463CF00BF8F42138463CF007F8032E1BD0D4F8C008437901689D0822
:20DE00000223AB40DB439BB20B828D892B408B810079202111F08AFFD4F8C0084A46494676
:20DE20003AF01AFAD4F8C038186806F0E3FA0022D4F8C40C11463AF00FFAD4F8C43C1868F9
:20DE400006F0D8FA0120E6E5114A013002EBC000F0B4D0F83CC30F4E00233360336133622E
:20DE600033633364336533663367BCF1000F0DD090F8387357B13F0100240CEB04030FCB9A
:20DE800035191034A74285E80F00F6D1F0BC7047E0C206089C63002038B50F4C94F8AB14FF
:20DEA00001F03F018B1C024601F10A0584F8A93484F8A65404F2A44084F8A72408311DF00B
:20DEC0000BFA254485F8A20494F8A6341C44000A84F8A30438BD00BF785F002070B51D4C85
:20DEE0000968D4F8D0541C4ED4F8CC44D6EDA87ADFED1A6A491B00EE901A0168F8EEE00A11
:20DF0000091B60EEA70A00EE101A20EEA07AB8EEC00A1C46A0EE007AB1EE400AF1EEC77ABB
:20DF200067EEA67AFCEEE77AC2ED007A4EF05EF89FED0B7ADFED0B7AE0EE077AFDEEE77A67
:20DF400017EE902A002ABCBF02F50C42A032226070BD00BF785F0020980100202C7D8E3FB2
:20DF6000A00CB34500A00C4638B50B4C002501228021204634F086FA30B194F9040034F03E
:20DF8000B5FA08B1006838BD0135062D04F10C04EDD10020F7E700BF5C64002038B5041FE3
:20DFA00000F1080554F8043FD81780EA430017F023FCA542F6D138BD2DE9F041D14CDFED3F
:20DFC000D27AD4F8303594F8C90507EE103A2DED028BB8EE478A28EE278A002840F0CA80A4
:20DFE000D4F8D42594F8C81594F8E535002A19DD07EE902ADFEDC56AF8EEE77AC3F1640321
:020000040800F2
:20E0000086EEA77A00EE103AB8EEC00A20EE070A29B920EE000ADFEDBE7A20EE270A5BF01C
:20E02000A9FD80B2B4F8CA35A4F8CA05834200F0A18094F83475B74EDFEDB78A4FF000088E
:20E04000002594F8E8352B41DB0714D594F8C835002B7FD1B4F8CA3507EE103A002F00F0AE
:20E06000FA80B8EE477AC8EE877A77EE887A88EE277A86ED027A0135042D06F12406E0D162
:20E0800094F8CD55B4F8D065002D40F0E780002F5CD194F8E43584F8F15584F8F035002E9B
:20E0A00054D0002D52D007EE906A0123B8EE678ADFED997A84F8F2359D42C7EE888A28D023
:20E0C000022D43D1D4F830159448B0EE480A45F061F994F8F135012B00F00F81022B35D100
:20E0E000D4F830158E48B0EE480A45F053F994F8F135012B00F0FC80022B27D1B0EE480A69
:20E10000BDEC028BD4F830158648BDE8F04145F041B9854AD2ED007A78EEA76A134687EE98
:20E12000A67A002143F8041F83ED017A78EEA76A002187EEA67A996083ED037A77EEA88AAB
:20E14000002287EEA87A1A6183ED057ABDEC028BBDE8F081B4F8CA35D4F8301500EE103A5C
:20E16000301DB8EE400A002F6FD145F013F994F8347580E794F83475002F3FF45CAF94F8E8
:20E18000CD55B4F8D065002DE0D0D4F8EC2594F8CE3592F883201343D8D1D4F8D42594F8B6
:20E1A000E535002A64DD07EE902ADFED586AF8EEE77AC3F1640386EEA77A012D00EE103A40
:20E1C000B8EEC00A27EE000A5FD05BF0D3FC80B2A4F8D005002F78D08642B7D00028B5D051
:20E1E00094F8F135002BB1D007EE900AB8EE678ADFED497A012BC7EE888A4DD0022BA5D159
:20E20000D4F830154548B0EE480A44F0ADFF94F8F135012B69D0022B98D1D4F8301540484A
:20E22000B0EE480A44F0A0FF94F8F135012B57D0022B8BD1B0EE480ABDEC028BD4F8301556
:20E240003848BDE8F04144F08FBF301D44F08CFF94F834750FE7C6F8048002E7D4F8EC25A7
:20E2600094F8CE3592F8832013437FF410AF94E70023A4F8D035002F7FF468AF94F8E435BD
:20E2800084F8F15584F8F03560E720EE000ADFED207A20EE270A98E7234A1346F3EC017A78
:20E2A00078EEA76A87EEA67A83ED017AD2ED007A78EEA76A87EEA67A83ED037A77EEA88A9E
:20E2C00087EEA87A83ED057A40E794F8E43584F8F15584F8F03500283FF438AF0646E2E633
:20E2E000114AD2ED007A131DE8E70F4A131DDDE70D4AD2ED007A131D20E70B4AD2ED007AE9
:20E30000131D13E7785F0020BD37863500409C45CDCC4C3CAC64002083F9223E6C650020EE
:20E3200090650020B4650020D8650020F8B5214C1D270E46054684F87C761DF0F3F80020AF
:20E340001DF092F808201DF08FF80E201DF08CF838461DF089F804201DF086F804201DF0BF
:20E3600083F800201DF080F830201DF07DF800201DF07AF830461DF077F800201DF074F881
:20E380001DF0BCF804F27D601CF0C2FF234670B194F87D2662B994F87E26302A00D03AB9FB
:20E3A00093F87F2622B993F880362B700120F8BD0120FCE7785F0020104B034410B50446F4
:20E3C00093F8100410F058FF0D4800EB44040A23B4F99016B1F5FA6FA8BF4FF4FA61B1F585
:20E3E0007A7FB8BF4FF47A71A1F57A71BDE81040B1FBF3F10920C9B210F06CBFE0C20608FA
:20E40000785F00201D4991F8B823A2B3F0B4002605463346304637461BB991F8B8432D2CB4
:20E4200023D02E2A19D0CA1800EB800092F8B843A4F13002092A4FEA40009CBFA0F1300245
:20E44000A0180E2B14D80133CA1892F8B823002AE2D106B14042F0BC70470133002DF8D0C2
:20E46000CA182A4482F8B873DDE701231E46EBE70020F0BC70470020704700BF785F002079
:20E480001FB503AC8DF80C30009400238DF80D300FF04AFA04B010BDF8B50546262025F0A8
:20E4A00007FF134C0146F8B9D4F8B40690F838301E3B012B01D93BF0A3FC0E4F0026AE42ED
:20E4C0000ADBB4F8D8360133A4F8D8360A4BD3F80039C4F8E836F8BD17F8011BD4F8B40626
:20E4E0003BF08EFC0136EAE7002384F8E636EDE7785F002030660020981B002010B58021EA
:20E50000044604F017FE2046002104F013FE2046BDE8104005F04EB92DE9F041B14C94F8F5
:20E52000FF36C4F8EC0682B088465A2B00F2B980DFE813F0CC00B700B700DC00B700B700FA
:20E54000B700B700B700B700B700B700B700B700B700B700B700B7000F01B700B700B700F2
:20E56000B700B700B700B70033017400B700B7007400B700B700B700B700B801B700620186
:20E58000B700B7007C00B7000902B700B700B700B7005B00B700B700B700B700B700B7004E
:20E5A000B700B700B700B700B700B700B700B700B700B700B700B700B700B700B700B700EB
:20E5C000B700B700B700B700B700B700B700B700B700B700B700B700B700B700B700B700CB
:20E5E000B700B700B700B700E40194F800379B0700F16982B4F80637D4F80127D4F8401719
:20E600005BBA9BB212BAD0188842C4F84C37C4F8482703D904F04EFD002854DB0020A4F882
:20E6200038070546284602B0BDE8F08194F84437002B40F0FF8094F9FC36002B31DAD4F878
:20E64000343708469B689847002840F01E82B4F80607D4F80127D4F8403740BA80B212BA3F
:20E6600015189D42C4F84C07C4F8482707D904F021FD002827DBD4F84827D4F84C07D4F812
:20E680003C37D4F8F86603FB00F003FB02F20225B042C4F84827C4F84C0784F8445700F0A3
:20E6A000CF8094F810375A1CD2B204EBC30305204FF40051042A84F8102783F81407C3F89E
:20E6C000181700F0A0814FF0FF35ABE7D4F8F836002BE6D1D4F8343708469B689847054667
:20E6E000002840F0D281A4F838079BE73E4B002203F1120103F8012F8B42FBD13B4994F88C
:20E700003A3794F8100770250D7098424FF00C05CD7110D004EBC300013390F814578D70B5
:20E72000B0F81807DBB2042B40BA888114BF84F83A3784F83A2794F8033712229342A4F84B
:20E74000382798BFA4F838370025284602B0BDE8F08194F80037DA0700F13E81D4F8343712
:20E7600094F80307DA6901EBC10102EB81010A79531D834228BF0346A4F83837002BE3D0D2
:20E78000013B1A489BB201331944034411F8012D03F8012D8342F9D1D6E7154E154F3546C8
:20E7A0000823073EC5F10700A4F83837002202E092F830241D462B46B54203F8012900EB64
:20E7C000030217FA82F2F3D1D4F834374046DB6898470028B8D0AB7863F07F03AB70002524
:20E7E00020E700BF785F002093890020948900209B890020E0C20608D4F83437C74A5B68E4
:20E800000846111D98470546002840F03E81D4F84037C34AD4F83C17013B180E1070180CC6
:20E8200009BAD37050701B0A082093705160A4F83807F7E6D4F84C67D4F84827D4F83C3760
:20E84000D4F83457B2FBF3F24FF48057BE4228BF3E462D69B249A4F838774046B6FBF3F351
:20E860009BB2A8470028C0F2BC803346AC4AD4F8EC06812104F092FCD4F84827D4F84C079B
:20E88000D4F858373244851B9E1BC4F84827C4F84C57C4F85867002D7FF456AF032384F802
:20E8A0004437BFE69E4E0027334606F10C0203F8017B9A42FBD1D4F8343740465B686A4658
:20E8C00001A998470546002840F0E980019BBDF80020013B190E52BAF3713171190C1B0A73
:20E8E00071710820B371022172810C23BDF80220F07031727272A4F8383793E6894E8A4FB3
:20E9000030460823073EC0F10705A4F83837002202E092F8382418460346864203F80129CB
:20E9200005EB030217FA82F2F3D1D4F834374046DB68984700283FF407AFF37863F07F0369
:20E94000F37000256EE694F84437002B61D194F9FC36002BFFF6A5AED4F8343708469B68BD
:20E960009847002840F09180D4F834374046DB6898470546002840F0BA80B4F80637D4F8DE
:20E980000127D4F840175BBA9BB212BAD0188842C4F84C37C4F8482700F29F80D4F83C17B2
:20E9A000D4F8F80603FB01F302FB01F28342C4F84827C4F84C377FF474AEB3F5805F28BF79
:20E9C0004FF480530121D4F8EC06554A84F844179BB204F00DFD25E607235449A4F83837A3
:20E9E000CEE694F810375A1CD2B204EBC30304204FF48851824284F8102783F81407C3F8D9
:20EA000018177FF460AE002384F810374FF0FF3508E6D4F84C67D4F83407D4F83C37D4F86E
:20EA200048274569B2FBF3F2B6F5805F28BF4FF480560846B6FBF3F339499BB2A8470028D2
:20EA400062DBD4F84827D4F84C57D4F858373244AD1B9B1BC4F84827C4F84C57C4F85837AB
:20EA60002DB9D4F8EC06294604F016FDDAE5B5F5805F28BF4FF48055ABB2D4F8EC06284AA8
:20EA8000012104F0B5FC0025CCE594F810375A1CD2B204EBC30302204FF468510AE694F8BD
:20EAA000103704EBC3020133DBB202204FF46851042B82F81407C2F8181722D084F810371A
:20EAC0004FF0FF35AEE594F810375A1CD2B204EBC30305204FF41051ECE504F0EBFA002813
:20EAE000FFF6F1ADD4F84827D4F84C3756E794F810375A1CD2B204EBC30302204FF41C5168
:20EB0000D8E584F81077DEE594F810375A1CD2B204EBC30304204FF440716BE7B46600204C
:20EB2000948900209B890020E0C2060808C7060810B51C203EF0F0F81121044639F0E8FF24
:20EB400020463EF0D9FBC8203AF030FD2046BDE810403EF0D7BB00BF08B500203EF0DCF855
:20EB6000054BC3F8600708B12A23C380BDE80840402139F0CDBF00BF785F00202DE9F04FCC
:20EB8000B34CD4F810365A69D2078BB002D50BB0BDE8F08F5A699B6912EA030AF7D0CAF383
:20EBA00007431AF4002F009340F00281009B5D0743D41AF0020F5FFA8AF503D0D4F810369A
:20EBC00002225A61BAF1000FC0F211821AF4006FCAF3072740F084812E0708D59D4B9E48DA
:20EBE000D3F8B0329847D4F8103608225A61ED0600F1E981F80600F1A981B90600F12E81CC
:20EC0000009BDA0609D5934B9348D3F8C0329847D4F810364FF480125A61009B9B06B6D5DD
:20EC20008C4B8D48D3F8C4329847D4F810364FF400125A610BB0BDE8F08FD4F81426936985
:20EC4000D26913401FFA83FBBBF1000FB1D0DFF80882CDF80CA045464FF0000909E05FEA7C
:20EC60005B0B09F1010908F1040805F1280500F0DA811BF0010FF2D0D4F814165FFA89F70B
:20EC800008694A6B04EB8703FA40D3F81C36D2019B68D2B202431A40D007D3B216D54B6B88
:20ECA000D8F81820012000FA09F023EA00034B63684B6948D3F8A832012191603946984700
:20ECC00094F80766012E00F0FC8101231A0703D5D8F8182008239360DE0603D5D8F8182098
:20ECE00010239360580603D5D8F8182040239360990703D5D8F81820022393601A06AED51F
:20ED0000D5E94C60D5F82431D8F818C0311A8B42DCF8182028BF0B46033392B2B2EB930FAA
:20ED20009DD9D4F81426323704EB8703CDE9019890469946B04238D2BEB3D5F8241194F876
:20ED40000736D5F82821371AB94228BF394601F1030E4FEA9E0E83B98FB20337BF10D9F86F
:20ED60000CA60AD0013352F8040BCAF800009F42F8D1D5E94C60D5F82821DCF81830084426
:20ED80000A44B042C5F82821C5F834010AD195F81C11D8F83420012707FA01F122EA010258
:20EDA000C8F834209BB29E45C4D3DDE9019856E7D4F814369D69DB691D402D0C3FF4F6AE0F
:20EDC00004F20466DFF88CB0B046B146002708E06D0807F1010706F1040608F128083FF4F2
:20EDE000E5AEEB07F4D5F9B204EB8102D4F81436D2F8582692685B691A40D007D3B218D5E9
:20EE000094F80706726D01239842936007D11269D8F87C33C2F312029B1AC8F88C33DBF8E7
:20EE2000A4324846984794F80736012B00F0578101239A0702D5726D022393601B07C7D581
:20EE4000DBF8AC3248469847736D08229A60BFE7804E00209801002084540020D4F8143635
:20EE6000D4F81C169A680868C2F34102022A08BF03224FF0000514BF65F30A0062F30A003A
:20EE800008605A6842F480725A6006A805F060FBD4F81026D4F81406D368BF49079D6FF337
:20EEA0008D23D3608068C0F34100014491F84014032900F0CF80B949B9480126294484F8F3
:20EEC000066681424FF04006A4F8086600F215810E2161F38D234FF40051D36051618FE6CB
:20EEE000B04B94F81627D3F8B832AF4800218DF817108DF817209847D4F81416D4F8102642
:20EF000094F80E3688684FF400615161002B3FF463AEC3077FF560AE94F81937012B7FF4A5
:20EF20005BAE9DF81730032B7FF456AED4F810379E491A6842F001021A601A6842F0030263
:20EF40001A600B6943F006030B6145E6D4F81426954853684FF0000823F0010341465360BA
:20EF600004F054FF94F80566414656B1904BFF2203EB860653F8045FD86BAA609E42826092
:20EF8000F8D1D4F8143688484FF0FF329A614FF00112DA610B2262F3070162F30708C3F821
:20EFA000148019611A686FF30A121A6004F002FCD4F810267B4B7C48D3F8B4324FF4805186
:20EFC0005161984719E6D4F810369A6922F010029A611A6AC2F34340022802F00F0144D071
:20EFE000062823D09A6942F010029A6102E694F80E363BB1D4F81027136823F0030161F321
:20F0000007031360D4F8142666495368D1F8BC12654823F0010353608847D4F810364FF0D5
:20F0200000425A61D2E5DDF80CA0C2E501EB8101D4F8D45604EBC1012E68D1F89009C4F82B
:20F04000D06BC2F30A1202442868C4F8D40BC1F89029C7E700214FF4007084F8061609217D
:20F06000A4F8080661F38D2335E747F6F0701042B8D001EB8100C2F30A1204EBC00002F16F
:20F08000030C5FEAAC0CD0F88459D4F8D4E64FEA810818BF002006D00130DEF8006045F802
:20F0A000046B8445F8D1414404EBC101D1F88459D1F8900915440244C1F88459C1F890296A
:20F0C00090E7B9F1000F7FF400AE94F81537042B7FF4FBAD344804F06DFB3346F6E5002F62
:20F0E0007FF4A6AE94F81527052A7FF4A1AE4846019304F05FFB019B9BE62E48A5F574017E
:20F10000A1F51051814203D80D2161F38D23E2E629492A482944814203D20C2161F38D2346
:20F12000D9E62748A5F18C71A1F54341814203D80B2161F38D23CEE622492348294481426C
:20F1400003D20A2161F38D23C5E6204920482944814203D2092161F38D23BCE61D48A5F15F
:20F16000B771A1F55851814203D2082161F38D23B1E6194919482944814203D2072161F388
:20F180008D23A8E6164917482944814234BF0621052161F38D239EE6E0C20608401E1BFF53
:20F1A0003F420F00980100208454002000ED00E098540020DFC810002013FBFE20D6130049
:20F1C000FF69180000D3CEFE40771B00C05BB3FEC091210040AC2700C01D6AFE40E1330054
:20F1E000803C36FEE09C4100704700BF704700BF704700BF704700BF2DE9F0414FF0FF35D0
:20F20000324A33482C46002304E001330B2B02F1100215D0917A0429F7D103F5B17100EB25
:20F220000111C979CF07F0D4661C116801D0A942EBD21C4601330B2B0D4602F11002E9D18E
:20F24000631C02D10120BDE8F081214D04F5B17705EB07139988F1B9DFF880802601AB19FF
:20F26000D8F8002C1B4916691B4A41F2186001EB442118580023B047D0B1022808D141F20D
:20F28000CC6205EB0717AB58013B0121AB50B9710020BDE8F081DFF8448005EB0413D8F804
:20F2A000002C41F21860D268185826019047D6E741F2CC6205EB0717AB580321B97141F21F
:20F2C000D061013B0124AB506C54BCE7B0AF002094990020AC990020F9F20008804E00202C
:20F2E000044B41F2E472995C09B90121995401225A7070479499002038B5174D174B41F299
:20F30000D0640020285504E001300B2803F1100314D053F80E4C8C42F6D11C78032CF3D128
:20F320006AB10F4B03EB40239A4201D0FFF7D8FF00F5B17005EB00100123837138BD41F237
:20F34000CC6100F5B1736A5805EB03130420013298716A5038BD00BF94990020BAAF0020FB
:20F36000AC99002038B5134B00209C7B14B11D688D4205D001300B2803F11003F5D138BD92
:20F3800072B10D4B03EB40239A4210D0FFF7A8FF0A4B00F5B17003EB00100123837138BDD2
:20F3A000064B00F5B17003EB0010827138BD022CECD1EDE7ACAF0020AC9900209499002014
:20F3C0002DE9F84F12F0020E9B4606D028B9FFF787FF02252846BDE8F88F804C41F63805A9
:20F3E0006559002D5BD14FF0FF367D4FB146B046B24600253B68984200F0B68097F80EC0AC
:20F40000BCF1000F5BD0BCF1010F15D105F5B17C04EB0C1C9CF807C01CF0010F0CD11CF0C4
:20F420007E0F09D15FEADC1340F0A880D7F808C0D44501D2E246A94601350B2D07F11007BE
:20F44000D8D1751C04D1B8F1FF3F00F09F80464641F2C86806F5B17754F80850013544F87F
:20F46000085004EB061C41F21C694FEA07184CF8095044F8085041F2186904EB07154FF0E4
:20F4800000084CF80900C5F8048004EB0715AD79042D9CD8DFE805F01A330F334D0004F56F
:20F4A000C25741F63C063F68A65907FB0565A84299D3FFF715FF00252846BDE8F88F2E4615
:20F4C00001350B2D07F1100794D1BAE712F0010C70D104EB0710D51090F80780BBF1030FA1
:20F4E00065F3C71880F8078062D94FF6FF7083455B4628BF03469BB204EB07108380BEF149
:20F50000000F16D004EB061303F5B0531833987B04280ED041F2C8654FF0040C60590130F2
:20F52000605141F2CC65586083F80EC0635901336351500705D504EB0710C37943F0010367
:20F54000C371D30608D504EB0714E379C3F34502013262F34603E371224B012503EB46264C
:20F560000E602846BDE8F88F05F5B17704EB07164FEA071CB67986B92E4669E7A8460135A3
:20F580000B2D07F110077FF435AF5AE7B9F1FF3F18BF4E467FF45CAF8DE741F2C8682E4670
:20F5A00054F80850013544F8085044F80C506CE76346A1E70C4B0B49D3F8003C0B4AD3F8EF
:20F5C000088001EB46210023C04700283FF473AF04EB07140223A371FCE600BF9499002078
:20F5E000ACAF0020AC990020804E002065F30008F0B5124D2B7841F63002022B0BBF070AC5
:20F60000C0F3D417C4B200F07F04A85883B00E4600230122384401A9FFF7D2FE01280AD1A6
:20F620002B78022B019B16BF53F8243033F8143023F07043336003B0F0BD00BF94990020B6
:20F6400010B5144602070B4610D50B4941F2C472581C8B58834204D305D1002323600120FF
:20F6600010BDFFF73DFE2060012010BD21461846BDE81040BCE700BF949900202DE9F0416E
:20F680004268C2F308030B44B3F5007F82B004460D4657D390F91A30591C0AD0304A03F5FD
:20F6A000B17302EB0313FF21DA796FF30002DA71817694F91B305A1C0FD0294A03F5B1734E
:20F6C00002EB0313FF20DA79C2F34501013921EAE17161F34602DA71E0762378022B37D017
:20F6E0001F4A02F5C2531B68B5EB432F4FEA432824DC41F648036768D6583E407342AB42BD
:20F700001CDCAB19434511D32169207E01AAFFF797FF012812D16768236963614744019B10
:20F720002361A5EB0801BF1B67608D192046F8F753FE20B93D446560012000E0002002B0CD
:20F74000BDE8F08115444560012002B0BDE8F081616801202944616002B0BDE8F08100BF0D
:20F760009499002070B5154604460E46FFF786FF50B994F8280028B9022384F82830C4E95F
:20F780000B5670BD022070BD1DB12046A847012070BD012070BD00BF10B4D0E9011390F9F4
:20F7A0001A208B4238BF0B46511C83600AD0144B02F5B17203EB0212FF21D3796FF3000384
:20F7C000D371817690F91B305A1C0FD00C4A03F5B17302EB0313FF24DA79C2F345010139A5
:20F7E00021EAE17161F34602DA71C4760022436A5DF8044B4261426011460361B2E700BFC0
:20F800009499002038B54422002111485CF017FD104B41F602011A784FF6FF745C52022AB5
:20F8200041F2E87118BF032203F5C05041F64C055A5441F60C0441F6010203215D5900F8AF
:20F84000181910211D519954FFF7A6FF012038BD7CB10020949900202DE9F041B1F904307B
:20F860000F2B82B00C461646054632D02846F8F7D7FD95F91B80B8F1FF3F074633D02D4B18
:20F8800041F2186203EB08118A58904211D1183303EB4823A188013109B203EB4113A18001
:20F8A00028463360F8F7BCFD2060012002B0BDE8F081FFF715FD2846F8F78EFD28B100234A
:20F8C0000120336002B0BDE8F081002002B0BDE8F0814FF40071FFF7D1FE0028F5D04FF619
:20F8E000FF73A380C2E72846F8F776FD0028E2D10FB9FFF7F5FC38460023112201A9FFF7FC
:20F900005FFD0128D7D1019B0B4A9A1A48BF02F2FF12B2F5B05F4FEA622106D24FFA81F8FD
:20F9200085F81B80002BB5D1C5E7FFF7D9FC019BF6E700BF94990020AC99002030B504466E
:20F94000C06983B010B9012003B030BD0D460023032201A9FFF734FD0128F5D1B4F9203069
:20F96000002B03DAFFF7BCFC0220EDE7019A012D4FEA431102EB431303D0022D12D1E52553
:20F980005554A268DA612278032A04D100221A775A779A77DA77626A5A83C2F30F429A822C
:20F9A00003B030BDE268DA61EDE700BF10B50378023B012B0446037E02D913F0060F5AD1FD
:20F9C00098063AD494F91A30591C0AD02D4A03F5B17302EB0313FF21DA796FF30002DA719D
:20F9E000A17694F91B305A1C0FD0264A03F5B17302EB0313FF20DA79C2F34501013921EA82
:20FA0000E17161F34602DA71E076237E1B070BD51C4841F2C873C35C072B01D0FFF760FC6E
:20FA200041F2C8730022C254E26A0023237084F82830FAB1BDE81040104700231249E0698C
:20FA40001A018A58904206D001330B2BBAD01A018A589042F8D10B4A03F5B17302EB031301
:20FA6000DA79C2F34501013921EAE17161F34602DA71A7E710BD0121FFF760FF0128F9D1F5
:20FA8000237E9DE794990020ACAF002030B1027822B190F828201AB1002070470120704701
:20FAA00010B5D0E90142A242C16238BF22460321826080F82810FFF779FF012010BD00BF4E
:20FAC0002DE9F04FDFF868918A4699F80010DAF800300229174683B0834641F6300240F071
:20FAE0008B8059F80250DEB2A6EB030805EB1325B8444FF480729044BB4208F1FF38B8FB1F
:20FB0000F2F875D2A844032906EB0704A4EB03040CBF80224FF48072944228BF1446A8EBBE
:20FB2000050366B994422CBF0A220B2201A92846FFF746FC012809D003B0BDE8F08F0B222E
:20FB400001A92846FFF73CFC0128F5D199F80020DAF80010022A01F1010321D0A64210D200
:20FB6000019906F18042013A081F00EB840001EB820242F8043F824203F10103F9D1DAF81C
:20FB80000010A61B7318BBF1010FCAF800301BD09F4205F101052BD999F800100026B2E72F
:20FBA000A642EED2DDF804C006F10042013AACF1020000EB44000CEB420222F8023F90425A
:20FBC00003F10103F9D1DCE7BB42E1D199F80030022B21D004F18044019B013C4FF0FF3210
:20FBE00043F82420DAF800309F4205F10105D3D8012003B0BDE8F08F59F8022003F07F0619
:20FC00000329C3F3D415A6EB03081544B84414BF4FF4807280226EE704F10044019B013C17
:20FC20004FF6FF72584623F8142003B0BDE8F08F949900202DE9F04190F838300446032B4E
:20FC400051D8DFE803F002323B462D4BC0681978E76A03F5C252032911680CBF80264FF425
:20FC6000807601FB06F141F2C47C00EB412041F2A87841F2AC7E53F80C20E06053F80E001C
:20FC800053F808502261A5EB4125A0EB4121901943F8085043F80E1043F80C00C4E90C20A6
:20FCA0005FBB6262012384F8383016480021FFF745FE012811D1022384F83830626B04F1D0
:20FCC00030010120FFF7FCFE012806D1032384F8383000212046FFF731FE431EDBB2012B12
:20FCE00002D9BDE8F081022094F82830062B04BF002384F82830BDE8F081921B2263D1E722
:20FD00009499002034B100202DE9F04FDFF8248198F80060012887B08CBF00230123032EAD
:20FD200002930C460B68154639D0022E62D14FF480724FEA1329DFB201920138012823D877
:20FD4000012203929D421AD9384E06F1880A06F11C0B32681AB1DBF8001099424ED0DAF8D9
:20FD6000000000234844092205A9FFF729FB01281FD002280FD020B123689D42E9D825603F
:20FD8000032007B0BDE8F08F87B1FFF7A9FA022007B0BDE8F08F022007B0BDE8F08F8022F8
:20FDA0000192C3F3D41903F07F07C6E7019A0392C8E7DDE902C1059ADDF804E098F8003067
:20FDC000022B14D0032BE6D152F8273023F07043B3FA83F35B0963450F44236823D00B4477
:20FDE00077452360EAD309F101090027C5E732F81730EDE74FF480720192D2E70C490968A4
:20FE0000013A02EB41224902B2FBF1F203991344B3FBF1F201FB12320AB10B449B1A9D421A
:20FE2000236096D8ABE7AB42ABD3A8E73CB10020D4B1002094990020F0B5104D2B7841F66A
:20FE40003002022B0BBF070AC0F3D417C4B200F07F04A85883B00E4600230322384401A9EC
:20FE6000FFF7AEFA012807D12B78022B019B0CBF23F8146043F8246003B0F0BD94990020B1
:20FE80002DE9F04390F83C30002983B0044614BF02210021042B7BD8DFE803F0030C3C479A
:20FEA0006900FFF74BFD012870D1626B002A75D184F83C00404EDFF80881404D4FF6F7770E
:20FEC0001DE01FFA80F9B94594BF4FF000094FF0010901A9B9F1000F46D1FFF789FB012894
:20FEE000494650D1206BFFF7A7FF01284BD1019B2A682363013B934228BF13462B603378AB
:20FF0000206B032BDDD1404594BF4FF000094FF00109DEE7426B04F130010020FFF7D0FD96
:20FF2000012833D1032384F83C30234BE16A41F2C47003F5C2521D581268195041F2A877B0
:20FF400041F2AC76D8596D1A995902FB05F200EB422501EB422203F5BD500021DD519A51CD
:20FF6000FFF7ECFC012811D1042384F83C3094F82830042B04BF002384F82830A36B8BB172
:20FF800020469847012003B0BDE8F0830228FAD194F82830042B09D00220F4E7022384F8B1
:20FFA0003C30B8E7012003B0BDE8F083002384F828300220E7E700BF94990020D8B10020AE
:20FFC000F7FFFF0F38B590F834300446052B46D8DFE803F01F033F101963006B4FF0FF312B
:20FFE000FFF72AFF01283AD1E06A002839D1032384F8343000212046FFF7A0FC01282ED1EB
:020000040801F1
:20000000042384F8343094F82830082B2DD0012038BD41F63803224DEA5800F13001023236
:200020000120FFF771FE012824D00238C0B2012815D8052384F8343094F82830082B04BF79
:20004000002384F8283041F2E5730122EA54022038BDC06A216BFFF7EFFE0128C7D000202D
:2000600038BD022384F83430F4E7002384F82830012038BD05F5C252E3681168D4E90B20E4
:2000800003EB412341F644016850C4E9033002B96062012384F83430A0E7014DCCE700BF32
:2000A000949900202DE9F04F436883B0C3F308081646002A00F0E180714B05468946A3F1B9
:2000C000180B4FF0000AC8F5007495F91A70B44228BF3446791C28462ED0F8F7A1F90BEB94
:2000E000071341F218629B58984205D0FFF7F8F8504603B0BDE8F08F614B03EB47202246DB
:20010000494640445CF03AF8002221462846FFF729FBA2440028EBD02B7E1B0706D5594B2A
:200120002A691B689A4201D3FFF7DAF8361BA1444FF00008C7D1DBE7F8F74EF9002849D1E2
:200140002846F8F76DF96968C1F308032BBB21F4FF7323F0010303F50072AB689A422CBF84
:20016000062207222B7E03F00C030C2B1CD0002301A9FFF725F90128BAD10198404BC31ACA
:2001800048BF03F2FF13B3F5B05F4FEA63224FD257B2AF760028B2D1AAE72B7E03F00C03A6
:2001A0000C2B4FF00702E2D19BF800C0364BBCF1030F1B680CBF4FF0800C4FF4807C03FB24
:2001C0000CF34FEA432C0CF1FF3C0CEA0101A3EB5123CDE72B7E1A072ED59BF800102A4BAD
:2001E00095F828201B6803290CBF80214FF4807103FB01F3062A4FEA43233FF479AF234953
:200200000868834230D891F83D30002B7FF470AF002A7FF46DAF6B6985F83820062185F8E8
:200220002810EB622846FFF705FD012888D05FE7FFF756F80198ACE7154B1A78002A7FF40D
:2002400057AF95F82820002A7FF452AF082185F8342085F82810D3F85F206B692846C5E93C
:200260000B32FFF7AFFEE0E741F2E573012250460BF8032003B0BDE8F08F924638E700BFE0
:20028000AC99002058B10020D4B100203CB1002079B100202DE9F04390F8384083B005460D
:2002A000032C00F2A180DFE804F0021A8B0BFFF789FE012811D002280BD1032385F83830F7
:2002C0002B6C002085F82800002B00F0898098470224204603B0BDE8F08385F838002B7810
:2002E000022B79D0414A6F6841F64803D3581F40C7F34F272846F8F793F8DFF8F48006466B
:200300003F1A0AE0D8F800305A1E91454AD2FFF7B5F908B9FEF7E4FF0136022201A90023CB
:200320003046FFF74DF8BC1901281FFA84F94FF400724FF000010446CBD101985BF07FFF3B
:20034000EB694FF400712846002BDBD06B68002BD8D1019B4FF020324FF02E0C1A605A60D0
:2003600083F800C0C3F807204FF0100E6C6A1A625A6283F820C083F821C0C3F8272083F8C1
:200380000BE0EA6B5C83C2F30F4CC4F30F4483F82BE05A879C82A3F834C0D8F800305A1E98
:2003A0009145B4D3C3EBC353590201F500712846FFF764F908B9FEF793FF022385F8383047
:2003C0002B6C002285F8282063B1284698470124204603B0BDE8F0836F68C7F34F2789E771
:2003E000022476E7012474E7002472E794990020D4B100202DE9F04F90F8303089B00446CB
:20040000042B00F2A880DFE813F0A900B20005008A00E800B64D41F61003EB5C002B40F008
:200420009A80B44F04F11C09B84607F1380BBA4601AE324649464046FFF70EFA012840F0B9
:2004400018810198002800F0FA800378E52B01D0002BEED1A84A821A48BF02F2FF12B2F551
:20046000B05F4FEA622380F03C811B01A34A13449A7B042A0CD041F2C86104266A58013288
:200480006A5041F2CC615A609E736B5801336B5041F60202AB565E1C09D003F5B17305EB2A
:2004A0000313FF26D979AE546FF30001D97141F603016B565A1C0ED003F5B17305EB03138E
:2004C000FF26DA796E54C2F34501013921EAE17161F34602DA71202200215BF0B0FE2346A4
:2004E000019A53F8311F58685060116019899B7A93721181019B627EDA7205A847F066F88D
:20050000BDF81430002B40F02F8144F28172019903200A82CB810A83CB8284F83000237EF2
:20052000980600F1A9802046FFF736F92369002B00F0AE80237E03F0F70213F00403227674
:2005400040F0B480122A00F0BA80002384F828302046E36A984709B0BDE8F08F6548FFF7C8
:200560001BF94FF6FF720123228484F83030614F04F11C0801AE04F13109324641463846E7
:20058000FFF76AF901282FD00228E4D1584D41F60202AB56591C09D003F5B17305EB0313AA
:2005A000FF20D979A8546FF30001D97141F603016B565F1C0ED003F5B17305EB0313FF208B
:2005C000DA796854C2F34501013921EAE17161F34602DA71042384F830300020E36A207093
:2005E000984709B0BDE8F08F019D0B2249462846002D00F087802B78002B00F0838095F805
:200600000BA01AF0080FB8D15BF045FE0028B4D1637E8AEA0303DB0640F1C780344D41F6DE
:2006200002016B565F1CC1D003F5B17305EB0313FF26DA796E5460F30002DA71B6E73B789E
:200640002F49022B4FF009025046C3D00B78002BC0D1C1E905330A708BF800304A6B0B7301
:2006600051F8143CC1E90132FFF714FE01283FF4E0AE0228AED06EE7E0690023112205A9C8
:20068000FEF79EFE01283FF44EAF09B0BDE8F08F237E19077FF559AF154A41F2C873D15C5C
:2006A00000297FF458AF0721D1544EE70023E26AA16884F828302046FFF754F84BE7626A23
:2006C000E06AA0630421C4E90233C4E90B2284F83C30636384F8281063622046FFF75CF815
:2006E00039E7FEF7FDFD01986FF00F03BEE600BF949900207CB10020AC990020ACAF002004
:20070000A4B10020474D41F60202AB565E1C09D003F5B17305EB0313FF20D979A8546FF350
:200720000001D97141F603016B56581C0ED003F5B17305EB0313FF20DA796854C2F34501D5
:20074000013921EAE17161F34602DA71237EDA067FF540AF3448FFF71FF84FF6FF720223D3
:20076000228484F8303056E6304B05A9B3F9642702A846F07FFF9DF80C309DF80D609DF895
:200780000A509DF80B20BDF808109DF80E00DB0243EA461342EA4512A1F2BC7143EA5003A9
:2007A00042EA41229BB292B2B1E6A98A6B8B204A43EA014312686362EB69A3605202B3FBE6
:2007C000F2F102FB113109B113445B1A154DE36041F6020184F819A06B565E1C09D003F551
:2007E000B17305EB0313FF20DA7968546FF30002DA7141F603016B56581C0ED003F5B17388
:2008000005EB0313FF20DA796854C2F34501013921EAE17161F34602DA71032384F8303029
:200820007DE600BF949900207CB10020785F0020D4B100202DE9F04390F82830013B83B0C8
:200840000446082B41D8DFE803F048054D525865406A4300384B4668056B41F6480103F599
:20086000C2525F5813683740EA19B2EB432F4FEA432816D258E02169207EFEF7E1FE0128C0
:2008800023D1256B666823696361A5EB08053D444644F61B019B6660A84525634F4623610D
:2008A00042D82046F7F798FD01AA81460028E2D06668A368E26A9E4238BF1E460023A66060
:2008C00084F828300AB12046904703B0BDE8F083FFF7E0FC03B0BDE8F083FFF78BFD03B0B3
:2008E000BDE8F083FFF762F803B0BDE8F0830021FFF7C6FA03B0BDE8F0830121FFF7C0FA51
:200900000128E2D10023216C84F828302046FFF7BDF8DAE7FFF78EF903B0BDE8F083FFF767
:2009200051FB03B0BDE8F0832046F7F755FD0028BFD12E446660BCE79499002010B5114CF8
:2009400094F80E3623B9104B4FF480225A6110BD0E4A136823F00603136057F0E5F994F810
:200960000E36002BEFD0D4F814369B68DB07EAD5D4F81027136823F0030161F30703136029
:20098000E1E700BF804E0020003C014010ED00E02DE9F04704460D469046002144221E46DD
:2009A000089F5BF04CFC01234FF6FF722676628384F828302B782E2B4CD02E4604F1310A12
:2009C000307804F1390968B12E280BD043F0E4F9C0B20AF8010BCA4506F1010607D03078D2
:2009E0000028F1D120200AF8010BCA45F7D130782E2808BF707804F1380908BF013604F112
:200A00003B0A58B143F0C8F9C0B209F8010FD14506F1010607D030780028F3D1202009F851
:200A2000010FD145F7D118F0100F14BF0323012384F819802370E7622B782E2B26D16B78BD
:200A400023BB0323204684F83030FFF7D3FC2046BDE8F0876B78002BAFD1114B41F2F47286
:200A600041F60C0041F2F0719A5818585958E26041F601026062A1609A5C627641F2E872F2
:200A80009B5C2370E7622B782E2BD8D00023204684F83030FFF7AEFC2046BDE8F08700BF99
:200AA0009499002008B50121032003F0BBFA72B64BF0C8FB2DE9F04F8DB0CE4CDFF84893BB
:200AC000CD4D00904FF0000854F80B0C002800F0FE8039F091F90646002800F0D881D9F8EB
:200AE000003944F8073CE0260023C44F04F8033CA4F10B0B06FB08F654F80B0C39F07CF91C
:200B0000002800F0E48054F80B0C39F06DF914F8023C5A1E82460B2A0DD8DFE812F01F00DB
:200B20003A004600530083009B00E30016013501400177018E0124280CD0009A3AB995F80A
:200B40002E25824240F07F81012204F8032C0D2BD2D186E0012304F8023CCDE700234D2815
:200B6000C4F8C53084F8CD3084F8CE3004D0582808D004F8023CBFE7022204F8022C84F8FB
:200B8000C430B9E7032304F8023C022384F8C430B2E704233C2804F8023C0BD0BAF13E0F9B
:200BA0000CD0002304F8023CA6E70A233C2804F8023CF3D1002304F8013C9DE7012304F8E0
:200BC000013C99E7D4F8C500BB190344421CC4F8C52083F867AC94F8CD00022A8AEA000125
:200BE00084F8CD1088D12378C02BDAD86278FF2A08D1052BD5D9012384F8C430072304F897
:200C0000023C79E7A4F8C12000229342C4F8C93014BF0523062384F8C320C4F8C52004F8ED
:200C2000023C69E7D4F8C500BB190344421CC4F8C52083F867AC94F8CD00D4F8C9308AEA5B
:200C400000019A4284F8CD107FF456AF062304F8023C51E794F8CD308342A2D10D2304F85E
:200C6000023C14F8017C002F40F0F380644B08940FCB04AE86E80F00D4F8C930D4F8D10025
:200C8000ADF82C7023440993B4F8C130ADF8283094F8C3308DF82A3001238DF82E30324699
:200CA00003AB08A9039732F073F848B1049B059394F8C420534B0493314658462FF07EFD2A
:200CC000039E002304F8023C002E40F0D88008F10108B8F1030F04F1E0047FF4F5AE0DB0F7
:200CE000BDE8F08FD4F8C500BA190244431CC4F8C53082F867AC94F8CD2094F8CE00019322
:200D00008AEA0202514684F8CD2046F049FF019B84F8CE00072B7FF4EFAEB4F80530C02BE9
:200D20003FF63FAFB4F80320A4F8C120A27884F8C32000229342C4F8C93014BF08230923F5
:200D4000C4F8C52004F8023CD6E6014694F8CE0046F026FF94F8CD3084F8CE008AEA0303B3
:200D6000D4F8C50084F8CD30BB190344421CC4F8C52083F867ACD4F8C9309A427FF4BCAE43
:200D8000092304F8023CB7E694F8CD30434084F8CD3094F8CE3083427FF403AF56E7D4F84E
:200DA000C500BA190244431CC4F8C53082F867AC94F8CE000193514646F0F2FE019B84F8F5
:200DC000CE00052B7FF498AEB4F80120B4F80330A4F8C120227884F8C32000229342C4F887
:200DE000C93014BF0B230C23C4F8C52004F8023C82E600BFE75A0020785F0020804E002082
:200E000024C7060804800120981B0020014694F8CE0046F0C5FE84F8CE00D4F8C500BB1918
:200E20000344421CC4F8C52083F867ACD4F8C9309A427FF461AE0C239BE694F8CE308342BC
:200E40007FF4AFAE0AE7232804BF022204F8032C7DE6012F4FF0000602D004F8026C36E743
:200E6000D4F8C93008942344099308A8B4F8C130CDE90A66ADF828302EF0DCFEEDE754F886
:200E80000B0C2FF0D9FE54F80B0CB0471FE714F8033C002B3FF41BAFD9F8002954F8071C09
:200EA000521A632A7FF613AF012B32D0022B7FF40EAF54F80B3CC5F86837C5F86C37C5F86B
:200EC0007437402385F87837134BC5F8C833C5F8BC37124B85F8790793F8173F1048003B44
:200EE0004FF0010218BF012385F866270D4AC5F8702785F8C0373FF063FA4FF4005031F04C
:200F0000FFFD09483FF052FA85F8C16785F8C267DDE6FFF7C7FD00BFE8660020804E002026
:200F2000D77107081D6304080D72070800000000034B93F82400003818BF0120704700BF9D
:200F4000F81B0020202301480B80704768040020642301480B807047880400204323014897
:200F60000B807047EC04002010B5074CD4F8C800FF2807D0054951F8042BF7F765F9FF2341
:200F8000C4F8C830002010BD68040020E8B10020EAE700BF08B5D0F8E4355B6A9847002079
:200FA00008BD00BF08B5D0F8E4351B6A9847002008BD00BFD0F8E43510B504461B689847B5
:200FC000D4F8E8359B689847002010BD08B5D0F8E435DB6903B19847002008BD08B504221C
:200FE00090F81211D0F8E83580F8131180F81221DB689847002008BD10B5D0F8E83504461F
:201000001B699847032384F81231002010BD00BF0B0630B41CD401EB810200EBC2020023B6
:2010200000EB810582F8741382F8753301241A4604FA01F16D6D61F31F4201696FF3CF334A
:201040002B60CB6923EA0203002030BCCB61704701F07F0101EB810400EBC404012200EB2D
:201060008105002384F81C1184F81D2102FA01F11A46AD6961F30F02DFE700BF10B58121AF
:201080000446FFF7C5FF20460121FFF7C1FF024B0020187010BD00BFBC66002010B58121E4
:2010A0000446FFF7B5FF20460121FFF7B1FF82212046FFF7ADFFF7F70DF9002010BD00BFC3
:2010C00038B50D4604468321FFF7A2FF29462046FFF7E4FF002038BDF0B416460A063AD46A
:2010E00001EB810500EBC5052824002204FB0104022B85F87413C5F87C6385F8773385F8E6
:20110000752304F55D7448D0154600EB8107012202FA01F17F6D61F31F45D7F800C01CF433
:20112000004F11D1E488204946F0805242F4004242EA834204F00F041C4B42EA8452114077
:201140000CEA0303194339600269D3692B430020F0BCD361704701F07F0101EB810500EB04
:20116000C5052824012204FB0104022B85F81C11C5F8246185F81F31A5F8221185F81D21C1
:2011800004F58E740CD0002500EB8107012202FA01F1BF6961F30F05BFE722711546B4E710
:2011A00000252571F0E700BFFF87CC13007833EC002310B5194604464022FFF78DFF8021CC
:2011C000204600234022FFF787FFD4F8E835A078012284F812215B689847002010BD00BF87
:2011E00070B44B78012B26D00B784A6900EB83035C6D25682369D2B18A684A6102F07F02CA
:2012000023F4002323F07F0342F4002213432361C378012B04BF0B696361C5F3076363F0F6
:201220007B0363F31F652560002070BC70478A6802F07F02E4E782694C691568136944B30E
:201240008E68B4428CBF06F07F0404F07F0423F4002323F07F0344F4002443EA040388BFC1
:201260004E611361C378012B1DD0C5F3076464F07B0464F31F651560002BD5D14B69002B01
:20128000D2D002690878516B012383400B435363CAE723F4002323F07F0343F400231361CC
:2012A000C378012BE1D10B780C6900EB8300C5F30763816963F07B0363F31F654C6100202B
:2012C000156070BC704700BF2DE9F0434B78012B30D00B784C6900EB83035E6D356837690E
:2012E0001CB38B681C44013CB4FBF3F4C4F3090203FB02F3C3F312034B61144643EAC4433F
:2013000063F31C073761C378012B04BF0B697361CB78012B44D0C5F3076363F07B0363F37E
:201320001F6535600020BDE8F0838A680124C2F31203E3E791F800804E6900EB880EDEF89A
:2013400018C0DCF80050DCF8107076B3D1F80890384A06EB0904013CB4FBF9F402EAC44466
:20136000C6F312022243CC7807F060473A43012C174649D0CCF81020C278012A55D0026950
:20138000516B03FA08F30B435363C5F3076363F07B0363F31F65CCF800500020BDE8F0837C
:2013A0004B7973B345F00055B5E707F0604747F40027CC78CCF81070C378012B2FD0012C02
:2013C000E3D102699268D20554BF45F0005545F08055C5F3076262F07B0262F31F65CCF8E9
:2013E0000050002B9ED1B0B203308010DEF8D04098D0CA6852F8041B216001339842F9D19C
:2014000090E745F0805586E764F35E77CCF81070C378012BD5D10A69CCF81420D1E70A69CB
:20142000CCF81420012CB0D1CBE70B69CCF81430ABE700BF0000F81F0E4BDA68D20310D41C
:20144000DA68D1060FD4DA68D20510D4DA6812F0E00F0AD1DB6813F0020F14BF082009200A
:2014600070470120704706207047072070470220704700BF003C024000207047704730B19D
:20148000034B93F90C000028D4BF002001207047E8B1002008B5FFF7F2FF50B1054A537B38
:2014A000927B5B0003F00203002A18BF43F001030B6008BDE8B1002008B5FFF7E0FF10B158
:2014C000014B1B690B8008BDE8B1002070B5FFF7D6FF78B1084A958A65B196690023B3427C
:2014E0001C4607DA02EB44040133A48BAC42DBB2F5D30B7070BD00BFE8B1002008B5FFF7FB
:20150000BEFF10B100230B70137008BD0420704728B1034B93F9CC00003818BF0120704726
:201520006804002008B5FFF7F3FF50B1054B93F9CC20012AC3BF93F8CF30C3F340030B6016
:20154000002008BD6804002008B5FFF7E1FF18B1024B93F8CE300B7008BD00BF680400205D
:2015600070B5FFF7D5FF38B10E4C94F8CF30DB0703D500230B70137070BD0B4D94F9CD30C4
:2015800095F82C6093FBF6F301330B7094F9CD4095F82C1094FBF1F301FB1343013313702D
:2015A000EAE700BF68040020E8B100200320704770B50A4A92F8303006255E1CB6FBF5F4DA
:2015C00005FB146492F83150AC4205D002EBC303C3E90D0182F8304070BD00BFE8B10020C9
:2015E000002230B504461046914200DC30BDA35C0825584010F0800F4FEA400318BF83F08F
:20160000D503013DD8B2F5D10132EDE710B5D9B10E4B586E814217DCB2B1DB6A9A4213DCC6
:201620000B4C013A013903FB012184F8DA1004F1D6000521FFF7D4FF062184F8DB0004F12B
:20164000D600BDE81040B3E710BD00BFE8B10020680400200023038083708380C380037200
:20166000704700BF074A92F8683092F869100133DBB2994282F8683004BF002382F86830D8
:20168000704700BFE8B10020F8B5774CE36E83B1764B1B6893F82E305BB1754B94F8702011
:2016A000A3FB0013012A4FEA93132FD0022A08D002B1F8BD6F4B9842FBD9012384F870305C
:2016C000F8BD626F64329A423CD894F8683004EB031393F8E824FF2A06D06749013201203B
:2016E00083F8E82481F8DC00FFF7BCFF634B1B780122092B84F87020DBD1B4F86A35604A18
:2017000001339BB2A4F86A355380F8BD94F868105A4863678C2303FB0143007883F88A2087
:20172000002384F8863004F17C050A2202230928A56784F8872084F87030BAD1504B0131B9
:201740001980F8BD94F8862094F887309A42B0D104F17B0004F18405002310F8012F0821F7
:2017600053405A0013F0800F08BF5B0082F0070214BFD3B2DBB20139F3D18542EDD194F859
:2017800085209A4239D194F8686094F8835094F88430B4F87F00B4F8812094F87DC004EB9B
:2017A000061743EA052394F87E5087F8E81440BA52BA81B292B245EA0C202F4DC7F8EC14CF
:2017C0001BB294F97C10C7F8F024032E4FF00102A7F8EA04A7F8F43487F8E91485F8DC2094
:2017E00008D8264A12780C2A29D00D2A02D1244B23F81610FFF736FF5FE794F8683004EBA2
:20180000031393F8E824FF2A06D01B490132012083F8E82481F8DC00FFF724FF174B1B787A
:201820000122092B84F870207FF443AFB4F86835134A01339BB2A4F868359380F8BD11495E
:20184000114A897E0E4803EB830303EB830349089B0093FBF1F382FB0312DB17C3EBA203B3
:2018600020F81630C6E700BFE8B1002098610020D34D62103F4B4C0068040020712800201F
:201880007428002040310020676666660A4B93F8861093F8872091420DD010B493F8862015
:2018A0009C6F511CD2B2C0B2C9B283F88610A0545DF8044B70477047E8B10020FD2870B525
:2018C00022D0F02804D0EF2822D00224204670BD114D0320052641282E444FF0000405F1A8
:2018E000010580F080030DD0042B0BD9FFF7E6FF2044B542C4B2E9D015F8010B412880F0A8
:201900008003F1D10420F3E7044D0B200426E2E7034D0C200626DEE75CCC060858CC060840
:2019200064CC06080E4BD3F87025B3F96C05530707D400EB8000400080B200F5C87080B222
:201940007047084B084A9B6B323382FB0312D817C0EBA20080B200F5C87080B2704700BFEB
:20196000E8B100200C4C0020676666660C4AD2F8883530B41C68D2F880555D60198100253D
:20198000611C19609D812070D2F88835D2F880151A685A604FF6F67230BC19609A8170479D
:2019A000E8B10020114B30B4D3F82C27C3F8302703F28C5003F21C6103F20C6503F21C74D0
:2019C0000132C3F88455C3F88845C3F82C2730BCC3F87C05C3F80C06C3F81006C3F8801594
:2019E000C3F81C17C3F82017704700BFE8B1002000B583B00268084B8188CDF801203222F0
:201A0000D3F83437ADF805108DF800206846984703B05DF804FB00BFE8B100205E2810B5DA
:201A200011D05D2805D00D4BBDE81040D3F8383718470A4CD4F838379847D4F838373D207D
:201A4000BDE810401847054C5D20D4F838379847D4F838373E20BDE810401847E8B10020A4
:201A600070B5094E0546D6F838375E200C469847D6F8383728469847E0B2FFF7CFFFC4F31C
:201A80000720BDE87040C9E7E8B1002003682DE9F041002B3D4D3E4F3E4EB8BF5B42A5FB2D
:201AA0000321890D07FB0137C7EB0717BF0096F8423785FB0725FA170446C2EBA555002BC3
:201AC00057D101EB810101EB810105EB810109B2DFF8BC801320FFF7C3FF2F4908FB0575E2
:201AE00081FB0531ED17C5EBA11109B21B20FFF7B7FF2368254D002BB4BF53214E2123206B
:201B0000FFF7AEFF636896F8422783EAE376A6EBE376A5FB0631890D08FB0168C8EB081804
:201B20004FEA880885FB08354FEAE873C3EBA5552ABB01EB810101EB810105EB810109B2F5
:201B40001220FFF78DFF124B134903FB058581FB0531ED17C5EBA11109B21A20FFF780FF0E
:201B60006368002BBDE8F041B4BF57214521222076E7C1EB011105EB810109B2A8E7C1EB83
:201B8000011105EB810109B2DAE700BF6BCA5F6B806967FFE8B10020D34D6210044BD3F8D3
:201BA0005C3730EA030314BF01200020704700BFE8B1002030B40023022515244FF41671FE
:201BC00040F2D93205808471018130BC42814380838083817047134B10B400220F2483F8AA
:201BE0006217090A83F8610783F86317C3F86427C3F86827C3F86C2783F8604703F5EC603D
:201C0000012110F8014F013122440E29D2B2F8D183F86E270449D3F870075DF8044B1022B9
:201C200038F0BAB8E8B1002048B90020054B002183F87417C3F87817D3F8703703B1CAE798
:201C4000704700BFE8B1002013B50446FFF760FC08B300230DF106022046ADF806300DF0CF
:201C6000F5FCC0B10D4C9DF8062094F9CC1084F8E120032908BF62F07F024FF005010848AD
:201C800008BF84F8E120FFF7ABFC062184F8E2000348FFF78DFC02B010BD00BF680400204A
:201CA0004505002008B5044BD3F87C0738F0A4F8B0FA80F0400908BDE8B100202DE9F84F5E
:201CC0001B4C05461E2094F880A794F881B794F88267B4F88497B4F8868794F8887722F00B
:201CE000E7FA30B1B8F1000F03D0C14601264FF0000A94F88A37DA070AD494F88F273AB9DF
:201D0000012F12D0022F03D113F0020F08BF012685F800A085F801B0AE70A5F80490A5F873
:201D200006802F722846BDE8F88F3E46F0E700BFE8B100202DE9F84F2DED028BFFF7E8FB32
:201D4000002844D0264B93F9CC0001283FDD93F8E340DFF894809FED238A0FF27C0BDBE91B
:201D600000AB15468E1E02EB44094D4504D1BDEC028B2046BDE8F88F38F8027B26F8027FFC
:201D800007EE907AF8EEE77A67EE887A17EE900A56F0CAF952465B4656F01EFA41EC100B1F
:201DA00059F07EFF51EC100B56F03EFD0E2F80B20AD919303223B0FBF3F080B200EB800069
:201DC00000EB8000400080B225F8020BCDE70024CDE700BFAFF300801655B5BBB16B024056
:201DE00068040020CDCCCC3D9CB9002038B50D46FFF78EFB044638B10C4890F8CF30DB0791
:201E000004D5B0F8D0002880204638BD084A90F9CD3092F82C2093FBF2F102FB11320132DC
:201E20000131E4300DF026FCEDE700BF68040020E8B1002038B5134C94F8313094F8302050
:201E40009A4219D004EBC3030F49D3E90D200023984212DC93780D4AC4F8C4075B0813700D
:201E6000FCF71AFB94F8313006210133B3FBF1F201FB123384F8313038BDD55C01F8015BE8
:201E80000133E5E7E8B10020306600205E660020F0B52C4CD4F8C85794F8801787B0074640
:201EA00028460DF04FFC94F88117064628460DF035FC0022059294F882278DF81320034671
:201EC00075B1039005A928460DF04EFC94F88827039B2AB10DF1130128460DF04BFC039BD0
:201EE0009DF81320DDB1D2B1A1698A4217DC04EB8204D4F8CC470393262022F0D9F905998E
:201F0000039B70B911F0010F14BF502200228907786808D50C4949F077FF07B0F0BD0B4C76
:201F2000E9E74422F3E732B1CDE900420849324649F06AFFF1E707490094324649F064FF7B
:201F4000EBE700BFE8B1002012720708F37807081A720708267207082DE9F04FA84B1B780D
:201F60008BB08146002B40F0B380A64DD5F8C867002E00F0AD80A44AD2F8E84004F0F021B2
:201F8000B1F1E02F6DD1C2F8E830D5F8F027944267D004930593ADF81830B5F8843795F87E
:201FA00080E7ADF8143095F881C795F8883795F882A78DF818300DF110088DF810E08DF81D
:201FC00011C08DF812A098E8070007AB03C38F4F1A80C4F342533B44C4F30342997CC5F8E9
:201FE000F0478E4502F1010201D1944508D030468DF81C108DF81D200DF03CFBADF820007C
:020000040801F1
:2020000030460DF065FE032804F0070B34D0042835D000239A4501A9304618BF8DF81E30B8
:202020000DF0A2FB48B1019BC4F3001103F001038B4202D030460DF03DFD0A2207A9404604
:202040005AF0D5F868B19DF81E30BDF81C2085F88237BDF82030A5F88027A5F8843745F070
:20206000F9FE95F8F4A704AF95F8F437032B79D8DFE803F0083174A15F44FB7DCAE75F44E0
:20208000FB7FC7E7394630460DF074FB044658B107A8FFF713FE9DF81E109DF810308B4249
:2020A00060D030460DF07CFD95F8F437013303F0030385F8F4370CB99A45D5D195F88A37DF
:2020C000DB0700D524B1336849461B68304698470BB0BDE8F08F01A8FFF7F0FD95F88A8769
:2020E0009DF8044008F00108ECB1B8F1000F39D13A460DF1030130460DF03FFB044688B3F3
:2021000007A8FFF7DBFD9DF81C109DF803309DF81D208B4203D19DF81030934222D0304634
:202120000DF048FDC0E7B8F1000FBDD1394630460DF01DFB0446A8B107A8FFF7BFFDBDF8AD
:202140002010BDF810308B420CD085F8F58785F8F687336830469B699847A5E795F88A37F0
:20216000D80701D500249FE707A930460DF0FCFA04460028F6D01E2022F09AF895F8F73712
:2021800083428046EED085F8F70760B1B5F88637002BE7D1079BD907E4D4012130460DF04E
:2021A00089FC444680E7079BDA07DBD5014630460DF080FC78E73846FFF780FD97E807006A
:2021C00007AB03C31A809DF810309BB10DF11D0207A930460DF0D1FA0DF11E0130460DF031
:2021E000C9FA0A2207A938465AF001F8041E18BF012459E708A930460DF0B9FAECE700BFB8
:20220000DE660020E8B100206804002058CC0608024B0146D3F8F80737F0F2BDE8B10020F6
:202220002DE9F041FD2984B0044600F0DE80F02900F0BD80EF2900F031814AB10346861883
:2022400003AD002003F8010B9E4205F8010BF9D19A4B0B2003F1090501E013F8010F814223
:2022600000F0C880AB42F8D14B1E832B00F29380DFE813F03201390143014E01BE01840047
:20228000580163016F01910091007501750175018B018B018B016F019100910096019E0121
:2022A00091009100910091009100910091009100910091009100910091009100910091000E
:2022C0009100910091009100910091009100910091009100910091009100910091009100EE
:2022E0009100910091009100910091009100910091009100B40191009100910091009100AA
:202300009100910091009100910091009100910091009100910091009100910091009100AD
:2023200091009100910091009100910091009100910091009100910091009100910091008D
:2023400091009100910091009100910091009100910091009100910091009100910091006D
:202360009100910091009100910091009100910091009100910091001F011F01504BB3F80B
:202380002818002900F0668101922DF0F7FE019A80B2ADF80C003AB1224403AB13F8011BB4
:2023A00004F8011BA242F9D104B0BDE8F081454F03214FF00508B844002501370CE0FFF74E
:2023C0007DFA064660193246FFF72AFF70194745C5B2E9D017F8011B412981F0800308460E
:2023E00001D0042BEBD80426ECE7374F0B214FF00408E0E7324BD3F8700580060CD4002A0C
:20240000D2D0224403AB13F8011B04F8011B9442F9D104B0BDE8F08193F8FC07870742D52A
:202420002A4D287D052834BF02260326142917D97C39C8B20628E2D80629E0D801A050F8FB
:2024400021F000BF2D2601082D26010817260108FF2301083D26010837260108432601083F
:202460000929CCD90A390A29C9D801A757F821F0FD25010849260108FF230108FF2301086D
:20248000FF230108FF230108FF230108FF230108FF2301080F2601082D2601080C4F0C2143
:2024A0004FF0060887E7094B0B29187DA7D10126CBE0084B5B6B03936DE700BF80CC0608DE
:2024C000E8B100205CCC060858CC06084464002064CC06080C4C00200192FFF723FA019A1C
:2024E000ADF80C0057E76C4BD3ED037AFDEEE77A17EE903AADF80C304DE7684B93F847073D
:20250000B3F80018002840F0AB80ADF80C1042E76249B1F8003891F80818B3FBF1F3ADF81F
:202520000C3038E75D4D95F88A37DE0700F19D80B5F82838ADF80C302DE7584B5849B3F963
:20254000AC3881FB0301DB17C3EBA103ADF80C3021E7524BB3F8AE38ADF80C301BE7514B3D
:20256000DFED516AD3ED007A0C39C9B203EB810393ED147A67EEA67A67EE877AFDEEE77A43
:2025800017EE903AADF80C3005E7444B03EB4101B1F88A3803EB83035B00ADF80C30FAE6E5
:2025A0003E4B93F88A3703F00103ADF80C30F2E63A4BB3F84418CD055ABFCB4303F001031A
:2025C000032311F0440F18BF042311F0020F18BF072311F4806F18BF0923ABE70192FFF75E
:2025E000A1F9324B019ADB6B43EAC0400390D2E62A4BD3F83838ADF80C30CCE62B8A03EB85
:20260000830303EB83039B00ADF80C30F7E6EB89ADF80C30F3E6EB89254903EBC3039B0008
:20262000A1FB03135B09ADF80C30E8E6B3F8FE37ADF80C30E3E66B680393E0E62B680393F3
:20264000DDE6AB680393DAE6F6B28DF80C608DF80D00D4E6D3F8400880F3100080B298E623
:2026600093F80838B1FBF3F14FE705F60C05019222F02EF8D5ED037A019AFCEEE77A17EEC8
:20268000903A9BB200287FF455AF0A49096811F0100F18BF00234DE7F4B90020E8B10020EC
:2026A0006766666630BA002000007A440C4C00201F85EB510C63002070B5214D95F8B038CA
:2026C000EA181C4692F8B4288AB11E4E09225C1CA6FB04135B0803EBC303E31AE918DCB28B
:2026E00091F8B41809B1013AF1D185F8B04802681549561C06600C2616700268561C0660BF
:20270000002616700268561C066003EB430603EB8603147019440D223FF0E2FF95F8B018A8
:20272000084B4A1CA3FB02035B08294403EBC3030120D31A81F8B40885F8B03870BD00BF25
:20274000E8B10020398EE338A8BA00202DE9F041684ED6F8C87784B0044638460D460DF006
:20276000B7FA86F8350957B10DF1090202A938460DF003F8002840F08E8096F83509002365
:20278000ADF808308DF80A301A46431EDBB20021FF20FD2B8DF80C20ADF80E108DF80B00E3
:2027A00003D9002004B0BDE8F0819DF80830042B00F09680052B00F09980032B00F09880E2
:2027C000022B00F08C80012B08BF042100F088809DF809309DF80A10D6F8C807013B0DF16C
:2027E0000E028DF809300CF031FF96F83539032B73D0042B0CD1404A9DF80A0001210023F8
:2028000001E012F8011F81426DD20133082BF8D1D6F83829029B394F9A420DF108084FD01E
:2028200023680D22591C21601A7023680022591C21601A7023689DF80820591C21601A7069
:2028400023689DF80920591C21601A7023689DF80C20591C21601A7023689DF80A20591C24
:2028600021601A70BDF80E1020463FF081FF23689DF80B20591C216020461A700721FAF71B
:20288000DDFF98E8030087E803000120C6F8405904B0BDE8F08101A938460CF065FF002875
:2028A0003FF46BAF38460DF10A010CF063FF00283FF463AF019B96F8350903F0010264E7D0
:2028C0007A68D8F804309A42AAD1D6F840390C4AEB1A93427FF665AFA2E70A4A8CE7032147
:2028E0008DF8081074E78DF80A3091E70121F7E70221F5E7E8B1002077CC060820BB0020A5
:2029000080841E006FCC06082DE9F0412A4C2B4AD4F83838B4F84479B4F8406882FB03524F
:20292000DB17C3EBA2031FFA83F8474582B00D4603D1B4F84639B34233D002680190511C4E
:2029400034230160137002680023511C0160137041463FF00DFF019831463FF009FF0198BC
:2029600047F6FF713FF004FF019847F6FF713FF0FFFE019847F6FF713FF0FAFE019847F6C3
:20298000FF713FF0F5FE01980221FAF757FF0120A4F84489A4F84669C4F8485902B0BDE819
:2029A000F081D4F84839064ACB1A9342C5D8002002B0BDE8F08100BFE8B1002067666666B9
:2029C00080841E00026810B57F21541C0460117002680024511C01600E211470FAF72EFF84
:2029E000012010BD2DE9F04FC24B1B68804613F0800083B000F07181BF4B93F8FC0710F00E
:202A0000020000F06A81DFF810B39BF81430052B40F26881DBF80030B84D0093002BB8BFE0
:202A20005B42A5FB0342B648B649920D00FB0233C3EB03139B0085FB034502EB8202DC17BD
:202A400002EB8202C4EBA55400FB043304EB8204A4B281FB0321DB17C3EBA111BCB10025DC
:202A6000A94F2E46A7FB0432D20802EB8203A4EB4303E8B2A4469BB280008340BCF1090F18
:202A800094B246EA030605F10105EBD8340489B2B9B100259C4F2E46A7FB0132D20802EBFB
:202AA0008203A1EB4303E8B28C469BB280008340BCF1090F91B246EA030605F10105EBD8C3
:202AC0003443DBF804E08D4D8D4E8E498EEAEE70A0EBEE70A5FB0032920D06FB0200C0EB5E
:202AE0000010830085FB035002EB8202DD1702EB8202C5EBA05506FB053305EB8205ADB2E6
:202B000081FB0321DB17C3EBA111C5B10020DFF8F8C10646ACFB0532D20802EB8203A5EB97
:202B20004303C7B2A9469BB2BF00BB40B9F1090F95B246EA030600F10100EBD8350489B275
:202B4000C1B10020DFF8C0C10646ACFB0132D20802EB8203A1EB4303C7B289469BB2BF00F3
:202B6000BB40B9F1090F91B246EA030600F10100EBD83543DBF80830634A0193002B18461A
:202B8000B8BF5842A2FB0030604E6149030AA6FB0363DB0901FB03F1C1EBD00189B2B9B1F5
:202BA000002691463746A9FB0132D20802EB8203A1EB4303F0B28C469BB280008340BCF1F5
:202BC000090F91B247EA030706F10106EBD8B9B2BBF81070DFB10026DFF82CA1B446AAFB07
:202BE0000732D20802EB8203A7EB43035FFA86F938469BB24FEA890903FA09F3092897B297
:202C00004CEA030C06F10106E9D81FFA8CF7BBF812303D4AA2FB0306F608632E28BF6326F3
:202C2000092B63D9002093468146ABFB0632D20802EB8203A6EB43035FFA80FAB4469BB249
:202C40004FEA8A0A03FA0AF3BCF1090F96B249EA030900F10100E8D85FFA89F9009B019A9E
:202C6000002BCCBF392338231616BEF1000F26F07F0635DD274A3343964543F00206C8BFCC
:202C800043F00606D8F800301622581CC8F800001A70D8F800300022581CC8F800001A701F
:202CA00040463FF065FD214640463FF049FD294640463FF045FD404639463FF059FDD8F8DB
:202CC00000305A1CC8F8002083F80090D8F800305A1CC8F8002001201E7003B0BDE8F08F87
:202CE0001E43CFE7002003B0BDE8F08F4FF00009B4E700BF0C630020E8B100206BCA5F6BDD
:202D0000806967FFD34D6210CDCCCCCCC55A7C0AA0860100FFC99A3B446400202DE9F04723
:202D2000AB4B1B68064613F0800084B000F09E80A84B93F8FC0710F0020000F09780A64F8A
:202D4000397D052940F29780632900F292800024DFF898C289B22546ACFB0132D20802EB1A
:202D60008203A1EB4303E0B28E469BB280008340BEF1090F91B245EA030504F10104EBD808
:202D8000EDB2BB68954A82FB0312D917C1EB623189B2002900F018814FF0000CDFF84CE294
:202DA0006446AEFB0132D20802EB8203A1EB43035FFA8CF088469BB280008340B8F1090F7B
:202DC00091B244EA03040CF1010CEAD8E4B2FB8983494FF4F36707FB03F7A1FB0737C7F39C
:202DE0008F1742F20F739F4249D8CFB10020DFF8FCE18446AEFB0732D20802EB8203A7EB97
:202E00004303C1B2B8469BB289008B40B8F1090F97B24CEA030C00F10100EBD81FFA8CF7BA
:202E2000704BD3E9002313433ED14FF0FF3833681722591C31601A7033680022581C3060F8
:202E400039461A7030463FF093FC414630463FF077FC33685A1C32601D7033685A1C3260C3
:202E600030461C700621FAF7E9FC012004B0BDE8F087992585E7002004B0BDE8F087002127
:202E8000DFF868C10F46ACFB0302D20802EB8200A3EB40039BB28B400431102947EA030756
:202EA00093B2F0D1BFB2BBE701A844F08FFB9DF80810002900F08A804FF0000CDFF82CE193
:202EC000E046AEFB0132D20802EB8203A1EB43035FFA8CF089469BB280008340B9F1090FDC
:202EE00091B248EA03080CF1010CEAD84FEA08289DF80910E1B10020DFF8F0E08446AEFBA3
:202F00000132D20802EB8203A1EB43035FFA80F98A469BB24FEA890903FA09F3BAF1090FEA
:202F200091B24CEA030C00F10100E8D848EA0C089DF80A104FEA0828E1B10020DFF8ACE0E4
:202F40008446AEFB0132D20802EB8203A1EB43035FFA80F98A469BB24FEA890903FA09F3FA
:202F6000BAF1090F91B24CEA030C00F10100E8D848EA0C08BDF80C301B49632BA1FB03216B
:202F80004FEA08184FEA51117FF651AF0020DFF85CE08446AEFB0132D20802EB8203A1EB17
:202FA00043035FFA80F98A469BB24FEA890903FA09F3BAF1090F91B24CEA030C00F10100DB
:202FC000E8D848EA0C0832E70C4600E788468FE70C630020E8B100204464002089B5F814FB
:202FE000D34D621038BB00201F85EB51CDCCCCCC08B5A0F10103B3FA83F302284FEA5313DD
:2030000001D0184608BD0F2021F0CAF830B9064B93F88A3703F00103184608BDBDE808402D
:203020000F2021F045B900BFE8B10020037840680122053B11460AF0F7B800BF10B5084C7C
:20304000E26D13899907FCD513891B06F9D40A2036F08EF9206EBDE810403AF053B900BF3B
:20306000F81B0020014B1B681B6A1847805A0020024B186808B1836918477047805A0020EE
:20308000024B186808B1436918477047805A002010B5074C606D40B13BF0ACF994F851303B
:2030A00013B180F00100C0B210BD012010BD00BFF81B002030B40A490A480A78531CDBB2B5
:2030C0000525042B00EBC20400F8325008BF00234FF404520B7062604FF0FF3030BC70479B
:2030E000886600208C660020037870B4FBB10446C0F10106A31914F8015FDBB2002DF9D1B7
:2031000001335B00DCB2032513800C704D7004785CB1022300255A1CD2B2CC548D5410F8C8
:20312000014F0233DBB2002CF5D170BC704702242346E8E70B0617D401EB810300EBC3032D
:2031400010B400EB81000124002283F8764383F8741383F87523426D5DF8044B136843F4AA
:20316000001300201360704701F07F0101EB810300EBC303012200EB810083F81C1183F8AE
:203180001E2183F81D2182691368002B01DA43F0804343F4001313600020704770B501F02B
:2031A0007F0505EB850400EBC404282101FB05010126C4F830310023C4E94A2284F81C51AB
:2031C00084F81D61C4F8343101F58E711DB9FEF707F8002070BDFEF777F8002070BD00BF58
:2031E0002249F8B5D1F858390F2B04D05A1CC1F858290020F8BD1E4C25780023C1F8583956
:20320000002DF6D11B4E1C4B3268B2F5006F17D01B689A4227D017D9C2F50063402B15D99A
:20322000403B02F14005C1F85C3901232370356092B2402311490A448121FFF7AFFFD8E7ED
:203240001B6835607BB12A469B1AE7E74FF0000502EB0307C1F85C590CBF022101213760E7
:2032600092B22170E6E700232370C2E7E8B100200829002070240020742400200C29002082
:20328000AEE700BFF8B51D4C2378012B03D0022B09D00020F8BD01461948D0F85C3953B93E
:2032A00023700020F8BD00231A468121FFF776FF00232370F5E7402B11D9124C2268403BCC
:2032C00002F14005C0F85C39256092B240230E4C084622448121FFF761FF0020F8BD094D0C
:2032E0002A684FF0000603EB0207C0F85C6908BF02202F6092B208BF2070E8E70829002050
:20330000E8B10020702400200C29002038B5134602250A46C0E94E3380F811510021FFF713
:203320003DFF002038BD00BF10B50C7814F0600413D0202C0AD14B78023B092B18D8DFE8D7
:2033400003F01B21171717171717272E22490122FFF7DCFF0024204610BD4B78062B24D0C1
:203360000A2BF3D01D4B8A78C3F86829204610BDFBF7C4F80224EEE719490122FFF7C6FF83
:203380000024E8E717490122FFF7C0FF0024E2E74B88124A1B0AC2F864390024DBE70F4B2A
:2033A0008A78C3F860290024D5E74B881B0A222B0CD0212B04D021462246FFF7A7FFCAE78A
:2033C000CA880949092A28BF0922F6E7CA880749362A28BF3622F0E750BB0020E8B100202B
:2033E0004CBB002048BB00209E0500205405002038B501EB810400EBC4040D46002184F846
:203400007453C4F88C1384F87513C4F88833C4F88023C3782821012B01FB050108BFEDB298
:2034200001F55D7108BFC4F884231DB9FDF7D8FE002038BDFDF748FF002038BD144B9A6838
:2034400070B5044662B1134A1B7B92F86C592B4316D081212046FFF76DFE022D09D070BDB6
:203460000C4B93F86C5981212046FFF763FE022DF5D12046064ABDE870401F230121B7E744
:203480000121FFF757FE20468121BDE8704051E668660020E8B1002070B5094A094D117332
:2034A000094B13600021044629700D238121FFF775FE2046054ABDE870401F23012197E71A
:2034C000C8660020BC660020555342536866002010B5064B597B0446FBF71EF8002800DBF2
:2034E00010BD20460121BDE81040D5E7686600202DE9F041314D2C7834B1012C01D1FFF795
:20350000E7FF0020BDE8F0812D4FDFF8D080B0F8B4337A68C8F804201F2BBA68C8F8082043
:20352000064606D1274B3A689A4202D1797B01291AD9254A25491378052401F8334001EBAB
:20354000C3000133DBB2042B08BF00234FF4005113701F4B41600222304683F86C29FFF70C
:203560006DFF0020BDE8F081BB7B013B0F2BE0D8FAF7D2FF002819DB2B78013B022BC0D9C2
:20358000144B1988B1B1BB68D8F8082088F80C408B4228BF0B46D11A0424C8F808100E4A9A
:2035A0002C7030468121FFF7F9FDAAE73046FFF745FFA6E73046FFF76FFFA2E7BC660020F8
:2035C0006866002055534243886600208C660020E8B10020B066002094890020C866002036
:2035E00008B5084B1B78022B07D0033B012B02D80021FFF751FF002008BDFFF769FF002016
:2036000008BD00BFBC66002010B501EB8101084A00EBC1010446B1F88C131046F4F7EAFDF8
:20362000034A204640230121FFF7E2FE002010BD58BB0020E8E700BF70B50A7812F06005C0
:203640000C46064611D0202D16D1CD88D5B113062AD52A461F496078F4F7F6FDE2881D4966
:203660003046FFF753FE00250AE04B780A2B16D00B2B0ED0062B03D13046FAF73FFF0225BB
:20368000284670BD022260781144F4F7DDFD284670BD8B78D3B9104BC3F8B059F0E70F4901
:2036A0000122FFF733FEEBE70D4964780A4AC1F8C8400321C0E9E45542F8045B2B4680F81F
:2036C00011110021FFF794FE0025D9E7FAF716FFD6E700BFECB10020E8B1002098BB0020CF
:2036E000680400200B7803F00303012B03D0022B04D0002070478B881BB915E68B88832B48
:20370000FBD099E710B50223044640228121FDF7E3FC2046022340220121FDF7DDFC8221D4
:20372000204603230822FDF7D7FC064B02229A80F4F7D8FD044A204640230121FFF758FE38
:20374000002010BDB001002058BB002038B509220D46044603238321FDF7BEFC2946204676
:20376000FFF7D0FF002038BD82B00023016801930B6901930E4B03E00A690192013B13D0B4
:20378000019A002AF8DA019A094B42F001020192019A0A610A69019203E00A690192013BAA
:2037A00002D0019AD207F8D4002002B0704700BF400D0300436D064A1A61C278012A06D1A8
:2037C00000F2CC5058614FF0802219681A6070471800086010B5002304220446194680F8E0
:2037E00011211A46FFF7DAFC2046FFF7E3FF002010BD00BF10B5044629B990F81131032B98
:203800000DD0002010BDD0F8E4359B69002BF8D090F81221032AF4D19847002010BDD0F8C5
:203820009013D0F87C33994214D9C078D4F880230128A1EB030104BFD218C4F880238B426D
:2038400028BF0B46C4F890139BB220460021FFF7CFFDD6E7D0F8E4351B691BB190F8122192
:20386000032A03D02046FFF7B5FFCAE79847F9E7F0B5012190F8D17590F8D36590F8CFC557
:2038800090F8CE5590F8D03590F8D22580F8111190F8CC1585B005EB0C2503EB072302EB13
:2038A000062201F01F06AFB292B290F8CD558DF808109BB2012E0446ADF80A70ADF80C3018
:2038C000ADF80E20C0F840218DF8095017D0022E1FD036B101F08001FFF72CFC002005B0CC
:2038E000F0BD092D0FD8DFE815F0BF00AC000E00D5000E00EA0085000E007700540090F806
:203900001221032A2FD02046FAF7F8FD002005B0F0BD01F060012029DAB234D0012D00F031
:203920002081032D00F00681002DD7D190F81211022900F0DF800329E5D11B0600F14B8185
:2039400002EB820200EBC20393F87633002B00F04D81BF4B0122C3F8C429BE4920460222C3
:20396000FFF7D4FCBAE7DAB2012ACCD8D0F8E43502A99B689847BDF80E30002BAED1204614
:20398000FFF728FFAAE7D0F8E43502A99B689847A4E7F9B2AE4D012985F8B419B3D890F853
:2039A0001231022B00F02781032BACD1002900F0868190F810110129E1D0D0F8E4355B680C
:2039C000984795F8B41984F810112046FDF7F2FA2046FFF7FFFE81E7012A94D190F81231AF
:2039E000022B00F01781032B8DD100F58871FFF78DFC73E73D0A022DADF8062000F05081BD
:203A0000032D00F00B81012D7FF47DAFD0F8EC3580781B680DF106019847BDF80620002AE0
:203A20003FF45CAFBDF80E30002B3FF457AF9A4228BF1A4601462046ADF80620FFF766FCFE
:203A40004CE790F81231023B012B3FF65CAF012F7FF444AFD0F8E43500229B68C0F8182132
:203A600002A9204698478AE790F81231023B012B3FF649AF764BD0F818210021C3F8BC1911
:203A800012B10222C3F8BC29734920460222FFF73DFC23E7012F00F09880022F7FF41EAF77
:203AA00013F0FF0F7FF41AAF02691B0A023B5268032B00F21D81DFE803F0393531241A439A
:203AC0007FF421AF90F81231032B3FF41CAF036907F07F0580F81451196867F30A120A43A4
:203AE0001A60FFF777FE002D00F0E580022384F81231F3E651063FF4F1AE1146FFF71AFB17
:203B0000ECE6052363F30612514B012184F816112046C3F8C029FFF75DFEDFE6042363F33F
:203B20000612F1E7032363F30612EDE7022363F30612E9E790F81231022BDBD0032B7FF486
:203B4000E2AE27B9550602D01146FFF7F3FAD4F8E43502A99B68204698472046FFF73AFE22
:203B6000BCE690F812110229C4D003297FF4CBAE002F7FF4B3AE12F07F013FF400AF18069C
:203B800000F1A78002EB820304EBC30304EB810083F8767383F8741383F87573282303FB64
:203BA0000243416D03F55D73DA780B68023A6FF35553012AD4F8E42598BF43F080530B6077
:203BC0002046936802A99847D9E6D0F8E435C0F818719B6844E702F07F0202EB820200EB1C
:203BE000C20393F81E31002B7FF4B3AE184B0022C3F8C429B1E600293FF4C1AE0121032350
:203C000080F8101180F81231FDF7D4F92046FFF7E1FD63E61149FFF779FB5FE6FDB2052D22
:203C20003FF671AEDFE805F0342C241C0B03D0F8EC3580789B690DF106019847EDE6D0F862
:203C4000EC3580785B690DF106019847E5E600BFE8B10020ACBB0020A4BB0020A0BB0020DF
:203C6000D0F8EC3580781B690DF106019847D4E6D0F8EC358078DB680DF106019847CCE687
:203C8000D0F8EC3580789B680DF106019847C4E6D0F8EC3580785B680DF106019847BCE688
:203CA000D0F8E43580789B6A0DF1060198474570C4F8F005B1E6012384F812310EE602224A
:203CC000D0F8E43580F8101180F812215B68984755E6282202FB014304EB810083F81E71DD
:203CE00083F81C1183F81D51816903F58E735BE7012363F3061207E770B5044649B990F895
:203D00001131022B1BD094F81631012B0DD0002070BDD0F8E4355B69002BF8D090F81221CD
:203D2000032AF4D19847002070BD2A4A2369D2F8C0295A60002384F81631002070BDD0F8FD
:203D40003831D0F82451AB4217D9C278012AD0F82821A3EB050308BF5219C0F8383108BFBA
:203D6000C0F828219BB20021FFF718FA00231A4619462046FFF73CFBC5E7D0F83C31B3FBC8
:203D8000F5F605FB163666B99D420AD8D0F84021934206D233463246FFF700FAC4F84061F8
:203DA000E4E7D4F8E435DB681BB194F81221032A0CD00023052284F8112119461A4620465F
:203DC000FFF716FB2046FFF7F5FC9CE720469847EFE700BFE8B1002082B000230193019AF5
:203DE000094B42F010020192C168019A0A610A69019203E00A690192013B02D0019AD206F9
:203E0000F8D4002002B07047400D030082B000230193019A0B4B42F020020192019A61F34D
:203E20008A120192C168019A0A610A69019203E00A690192013B02D0019A9206F8D4002008
:203E400002B07047400D0300F8B50B7813F060050C4606461CD0202D17D14A78FE2A44D054
:203E6000FF2A3DD14A88002A56D1CD88002D53D11B0651D43749384B0D70012183F86C195A
:203E8000364A1F23FFF7B4FA00E000252846F8BD4B780A2B4BD00B2B44D0012BF6D191F9BA
:203EA00004308988002B47DBFFF796FF21792A4F3046FDF7ADF80223217940223046FDF738
:203EC0000BF997F86C39022B3BD094F90420002ADCDA012BDAD030460121FFF7DDFAD5E7EA
:203EE0000225FAF70BFB2846F8BD4D88A5B9CC88012C11D11A060FD5194B1B689B6998471D
:203F00001549C0B281F8C80930B1224601F6C8113046FFF7FBF9B9E730460225FAF7EEFAF8
:203F20002846F8BD0C4B4A8883F8C929AEE70D490122FFF7EBF9A9E701F07F01FFF766FF84
:203F4000B4E730468121FFF7F5F8002387F86C399CE700BFBC660020E8B100206866002059
:203F6000AC660020B1BB002038B50446FDF786F82046022340228121FDF7AEF82046022326
:203F800040220121FDF7A8F80C4B0D491B680D4A00250D701B6882F86C592846984720466B
:203FA000FFF71AFF20460121FFF730FF064A20461F230121FFF71CFA284638BDAC6600208A
:203FC000BC660020E8B1002068660020012905D008B50321FFF71AFF002008BDFFF752B923
:203FE00000B583B009238DF80730FDF725FA8DF807009DF80730012BF7D09DF8070003B044
:020000040801F1
:204000005DF804FB82B0064B002201920193019B03EB80000190019B186802B0704700BFA1
:204020005028004082B0064B002201920193019B03EB80000190019B196002B0704700BF24
:20404000502800400023C0E90033C0E90233C0E90433C0E90633C0E90833C0E90A33C0E996
:204060000C338363704700BF0B6870B4D1E90524CD682B431343D1E9072523431343D1E9D6
:2040800009422B43D1E90D652343134304680B4A334322402B4313430360D1E90B3442691B
:2040A0000D6922F0070223431343D1E9014243614560846070BCC260704700BF3F801CF0FA
:2040C00002683649002310B422F00102212488420260036043608360C3600361446138D06D
:2040E0002F4B98422ED02F4B98423CD02E4B984240D02E4B984232D02D4B984241D02D4B7B
:20410000984246D02C4B984217D02C4B98423CD02B4B984216D02B4B984224D02A4B984251
:2041200028D02A4B98421AD0294B984229D0294B98422ED0284B984208D14FF03D5243F88C
:20414000AC2C03E04FF4746243F8202C5DF8044B7047224B5DF8044B3D229A607047204A1E
:2041600043F8642CF2E74FF474125DF8044B43F8382C70474FF074625DF8044B43F8502C68
:204180007047184A43F87C2CE0E73D2243F8082CDCE7154A43F8942CD8E700BF1060024041
:2041A0002860024040600240586002407060024088600240A0600240B860024010640240CB
:2041C0002864024040640240586402407064024088640240A0640240B864024000600240A3
:2041E0003D000020400F002000003D200B88F0B433BB028C4C880E898B88C98822F00102FF
:204200001204120C0284058B028CADB225F0F30592B22B4322F00A0243EA061322439BB292
:2042200042F0010203830284038B23F00C031B041B0C0383038B9BB21943F0BC01837047A3
:20424000042B048C2CD0082B4E888A880D89C98851D024F480542404240C0484838B078C13
:204260002C0344EA022440F6FF421A4045F6FF733B4043EA063322439BB292B243F480535C
:2042800082830384828B22F440621204120C8283838B9BB243EA01239BB2F0BC8383704732
:2042A00024F010042404240C4D880F898A88C9880484068B038C12029BB242EA073423F02B
:2042C000A00340F6FF42324043EA051322439BB292B243F0100302830384028B22F4406280
:2042E0001204120C0283038B9BB243EA01239BB2F0BC0383704724F480742404240C0484B7
:20430000848B038CA4B29BB224F0F30423F42063224343EA062342EA05129BB243F4807342
:2043200092B282830384838B23F00C031B041B0C8383838B9BB21943F0BC8183704700BF54
:20434000214A038890429BB212D002F5806290420ED0B0F1804F0BD0A2F58032904207D0A0
:2043600002F58062904203D002F58062904203D14A8823F070031343144A904218D002F583
:204380008062904214D030B423F440730C894D6802F56C429BB2234390420C880380C56225
:2043A00004850DD18B7A0386012330BC8382704703800B884A68C2620385012383827047E8
:2043C000034B9842EED0EFE7000001400010004000040140024A536A23EA000050627047CC
:2043E00000380240024A136A23EA00001062704700380240484B98422ED0B0F1804F32D0ED
:20440000464B984236D0464B98421ED0454B984237D0454B98423BD0444B98423FD0444BE5
:2044200098424BD0434B984240D0434B98424CD0424B984251D0424B984256D0414B984210
:204440005AD0414B98425ED07047404A136A43F0040313620420C5E73C4A536A43F00103E7
:2044600053620120B6E7394A136A43F0010313620120B7E7354A136A43F002031362022093
:20448000B0E7324A136A43F0080313620820A9E72E4A136A43F0100313621020A2E72B4A43
:2044A000136A43F02003136220209BE7274A536A43F4803353624FF480308BE7234A536A96
:2044C00043F002035362022084E7204A536A43F4003353624FF400307CE71C4A536A43F4EC
:2044E000802353624FF4802074E7184A136A43F040031362402075E7144A136A43F080030F
:20450000136280206EE7114A136A43F4807313624FF4807066E700BF0000014000040040F6
:2045200000080040000C00400010004000140040000401400040014000440140004801406F
:2045400000180040001C00400020004000380240224A936803F00C03042B10B421D0082B4D
:2045600022D01F4B03601D4C1E4AA168C1F30311114491F84811CB404360A168C1F3822195
:20458000114491F8481123FA01F18160A1685DF8044BC1F342310A4492F84821D340C360A9
:2045A0007047114B0360DEE75468516852686302C2F388124CBF0C4B094B01F03F01B3FB48
:2045C000F1F303FB02F3054A5268C2F3014201325200B3FBF2F30360C5E700BF00380240A3
:2045E0000024F4006804002000127A002DE9F04700230F6801264FF0030C02E00133102BDE
:2046000041D006FA03F232EA0704F7D1D0F800E05C000CFA04F52EEA050EC0F800E091F856
:204620000490D0F800A009FA04FE09F1FF394EEA0A0EB9F1010FA846C0F800E06FEA050554
:2046400015D8D0F808E005EA0E0585604D79D0F808E0A54045EA0E058560456825EA020294
:2046600042608A7945689A4092B22A434260C26822EA0802C260CA79C568A24001332A4366
:20468000102BC260BDD1BDE8F0870D4B93F88A27D20703D5012283F8CA29704793F8CA2908
:2046A00062B9D3F8C8274AB193F88027104493F8812783F88007114483F88117704700BF91
:2046C000E8B10020044B93F90C00012806BF02221A730020704700BFE8B10020114AD2F827
:2046E000CC09A0B1D2F8D0398BB188420DD88B4234BF002301239BB11369C2F8D419994285
:204700001CBF142382F8D839DCE70023F3E7A1F59C53083BB3F57A7F2CBF00230123EAE7D0
:20472000704700BFE8B1002007B500230DF10602ADF806300AF08AFF60B1084BBDF80620C8
:20474000998AA3F8DA2991421CBF142283F8DC29FFF7B8FF03B05DF804FB00BFE8B1002008
:2047600013B50446262001911FF0A2FD019948B9054BD3F870372BB1204602B0BDE810405B
:20478000FDF729BA02B010BDE8B10020B1FA81F149094920E4E72DE9F341BE4C94F90C304A
:2047A00001330D4600F06681D4F87037002B00F0B380022700264FF00108D4F8700735F0DB
:2047C0001BFB002800F0A880D4F8700735F00CFBD4F878375A1C2344C4F8782783F8DD0900
:2047E00094F87437012B09D0022B15D063B90F280CBF84F87487C4F87837DEE7A0F17203A0
:20480000012B06D9762804D084F87467C4F87867D3E784F87477D0E7102ACED19E4900236E
:20482000012211F8010F013203440E2ADBB2F8D194F8EB2984F874679A42C4F87867BCD139
:2048400094F8EC39002BB8D194F8DE39732B59D0762B1BD0722B5FD194F8E02994F8DF39F7
:2048600094F90C1053EA022356D0C4F8CC390029B4F8E139C4F8D0394EDC94F8FA29012395
:204880002373002A48D184F8FA3945E094F8E02994F8DF3953EA02233ED0D4F8F02994F851
:2048A000E21994F8E609236193421CBF142284F8D82994F8E129C4F8F03942EA0122B4F825
:2048C000F419A28291421CBF142184F8DC1994F8E319617394F8E419A17394F8E519A4F834
:2048E000F42941EA0021A4F8F619D4F8D41909B9C4F8D439B4F8DA390BB9A4F8DA29022319
:20490000237309E094F8E42994F8E33943EA02231AB20BB1A4F8F82994F90C30022B35D045
:204920000FDCDAB2012A15D9636E13B1A369002B6CD15A495A481F2202B0BDE8F04157F089
:20494000BCBC032BF0D1D4F8FC39564AEB1A9342EADD13E0D4F8FC295349AA1A8A42E3DDDE
:204960002BB97220FDF762F9C4F8FC59DCE7D4F8003A5A1CD907C4F8002A03D47620FDF7FB
:2049800055F9F1E77320FDF751F9EDE7D4F8D419D1B194F8D839BBB12369994214D0637BDF
:2049A000DA0703D489B24620FFF7DAFE94F8D839013B84F8D83905F59225032305F57875AC
:2049C0002373C4F8FC59AFE7B4F8DA19A38A81B194F8DC296AB18B420BD0637BDB0702D4B2
:2049E0005020FFF7BDFE94F8DC39013B84F8DC39E1E701222273A4F8DA392269C4F8D429B5
:204A0000002384F8DC3984F8D8398DE7274DD4F8C8772A2385F858310DF1070220230DF1C7
:204A20000601384685F859310AF0A7FE30B19DF806109DF8076051EA06031ED1552385F89B
:204A40005A31462385F85B3122691948202385F85C31002A34D0174947F0D6F9B4F8F639B1
:204A600015488BB3A28A15499A420CBF20222A2247F0CAF902B0BDE8F08138460AF062FE42
:204A8000314685F85A0138460AF048FE037885F85B31D9E7E8B10020C5BB00202F720708BC
:204AA000C0050020400D030040420F0068040020C5050020B9AB0708C9050020497207088F
:204AC000034947F0A1F9C9E7024947F09DF9D1E7517207085072070810B50E4C40F008023D
:204AE00084F87B2194F9CC20022A06DD420704D583071CBF012384F8D43005210648FCF784
:204B00006FFD062184F87C01BDE810400248FCF74FBD00BF68040020DF05002010B5FCF7C4
:204B2000F7FCA8B31B4C94F9CC30012B30DD59B3022B2DD094F8D4309BB971B180230521F9
:204B4000154884F88131FCF74BFD062184F88201BDE810401048FCF72BBDBDE81040042028
:204B6000BAE7002914BF0020042094F8CF301A0748BF40F002005B0701D411B108B940F085
:204B80000100BDE81040A7E7022BD3D10420ECE710BD00BF68040020E5050020F8B5224C8C
:204BA00004F28317030A84F8880105460621384684F88731FCF714FD94F8CF3084F889019A
:204BC000DB072AD4B4F8D020AA4226D1174DD4F88331C5F8043AC3B285F80A3A41F26F714E
:204BE0004FF6FF738A4218BF0123134405F60426C3F307220621304685F8082A85F8093AD0
:204C0000FCF7EEFC072185F80A0A3046FCF7D0FC052104F5C570FCF7CBFCBDE8F840044892
:204C20000721FCF7C5BC00BF68040020E8B10020EB05002008B5FCF76BFC48B1A1F59C532F
:204C4000083BB3F57A7F03D2BDE808400846A5E708BD2DE9F0476B4E3368002B3AD06A4D82
:204C60006A4C05F1CC07306835F0C6F8002833D1674B198809291D4609D95F8864227A431A
:204C8000B2FBF1F2452A40F3A4811880588094F8453A012B00F0C881022B00F0E38133B970
:204CA0005C480521FCF784FC012384F8453A5A4B1D685A4B1B78002B00F0DE81584B1B6896
:204CC000EB1A782B40F2D881D4F8C407F9F7E4FBC4F8485ABDE8F087306835F085F894F8FB
:204CE0000B3A8046052BBED8DFE803F00309171D3745AA28B7D1012384F80B3AB3E7552817
:204D000003D1022384F80B3AADE7414A938801339380002384F80B3AA5E7032384F80C0A30
:204D200084F80B3A9FE7132884F80D0AC4F8280A07DD374AD3880133D380002384F80B3A45
:204D400091E718B9052384F80B3A8CE70023C4F82C3A042384F80B3A85E7D4F82C3AE218E9
:204D6000013382F80E0AD4F8282AC4F82C3A93427FF479AFE6E7D4F8283A2A4803F1020A50
:204D80004FFA8AF1FCF72CFC804594F80C9A40F0178126201FF08CFA204B48B100221A708A
:204DA0001B4A538801335380002384F80B3A5AE71A784A4519D100221A7009F1FF33102B69
:204DC00000F2F980DFE813F030008E008E00E1008E00F700F700F7003000F700F700F700E9
:204DE000F700F700F700F7003000B9F1090F02D0B9F1110F01D1012ADDD0054A5389013340
:204E00005381DAE72C66002068040020E8B1002050660020F2050020982400205E66002059
:204E200060660020F4BB0020BAF1060F5ADDB9F1010F06D0B9F1090F0CBF4FF002094FF020
:204E4000030994F8110A94F8121A94F8102A94F90EEA94F910CA94F80F3A85F8CC9041EA5C
:204E6000002109B2900785F8CDE085F8CFC0A5F8D01006D512F00C0F14BF0122002285F87F
:204E8000D420B9F1030F13D1BAF1090F2ADD94F9142A082AA8BF082222EAE27285F8E32046
:204EA000002043B29A4200F101005CDC94F8133AD4F818A0002002469BB2524590465ADB23
:204EC0007D4B85F8CE001B78232B0BD109EB89037A4A03EB83030CEB83031380A2F802E0BE
:204EE0009180D080764977480A2257F080F910B1002384F83A3A724B3A681A607A685A609E
:204F00003A891A8194F83A3A43BB95F8D43094F8802784F83C2A002B14BF0223012384F8CC
:204F20003A3A95F8CF3094F8820784F8400A13F001031CBFB2FA82F35B0994F8812784F87F
:204F40003D2AD9B2B4F8842784F83B1AA4F83E2A13B10AB1A4F8422A84F8441A0BF0AAFD30
:204F60000BF0A8FD1CE704EB4308234493F8163AA8F8B43795E704EB48080132B8F81C804D
:204F800052B2984508BF104697E7BAF1040FA9DD94F80E2A94F80F3A43EA022359041AB23D
:204FA00004D5C3F30D03A5F8D2309BE7002AF8DBA5F8D03096E7444A938901339381EFE653
:204FC00019F0010F7FF4F0AE3F4A138901331381EAE63E4BD3F89021B3F89411012A1AD17F
:204FE00041F25632914203D14FF0FF32C3F89021D3F89021306802EB820202EB820201EB91
:20500000420189B2A3F8941103681B69984700232B806B803BE60132EAD1B1F5965F04BFDE
:205020000122C3F89021E3E7284D95F9CC60002E3FF43DAE022E11D14FF48040FFF7AEFDE6
:2050400084F8456A95F9CC30012B7FF730AE95F8CF30C3F3400385F8D43028E6032384F865
:20506000453AEFE7194BB3F8D230002B3FF41FAE032384F8453A1AE694F8302094F83130B5
:205080009A4204D0FCF7D6FEC4F8485A22E6D4F8483AEB1AB3F57A7FBFF41CAE0C4B1B68E8
:2050A000ED1A952D7FF616AE0A480521FCF780FABDE8F047FCF7BEBE712800207428002049
:2050C00018BC002034050020506600206804002060660020F205002010B5134CD4F8C80765
:2050E00000B394F8801759B194F881270AF0C2FAB4F8843783421ABFA4F884070121002177
:20510000B4F8862762B141F288339342B8BF13469A4205D0A4F88637BDE8104042F09ABE07
:205120000029F9D110BD00BFE8B1002010B401440446002014F8013B08225840430010F077
:20514000800F08BF400083F0070314BFD8B2C0B2013AF3D18C42EDD15DF8044B704700BFC8
:2051600030B54FF4806085B02DF0A0F940B3154C90F9040094F84C3A134A002B18BF0823BF
:205180004FF4E1310125CDE90153009100234FF480612DF0ECF9FF23E066003818BF012018
:2051A00084F8E83484F8F83484F8083584F8183584F8283584F8383584F8483584F8583569
:2051C00005B030BDE8B100208D180108364B1A6812F000625CD0354B93F869C0604559D32E
:2051E000FF2855D1324A92F8DC20002A57D000212DE9F04FC3F8501AC3F8541AC3F8581A1E
:20520000A3F85C1ABCF1000F4BD003F59D620C460D4608460E460F4602EB0C1BE246B2F82D
:2052200002E0B2F80CC092F8009092F90180704461444F45D2E901EC38BF4F461032464502
:20524000B8BF4646934500B209B275446444E6D190FBFAF091FBFAF183F8507A83F8516A87
:20526000C3F8545AC3F8584A124AA3F8520A12780F48A3F85C1A092A4FF0000180F8DC104C
:2052800003D10D4A93F8503AD3800C48BDE8F08F0020704703F59D6303EB00107047074830
:2052A000704761466046DFE70C630020E8B1002068040020712800207428002038BC0020C7
:2052C0000268F8B53A4E3B4CB6F9603A511C01607E2111700168054603EBC30384FB030285
:2052E000481CDC17002328600B70FF20C4EB6204FFF76CFF2034304BA4B200284DD01B789F
:20530000B0F90C102BBB2D4BA1F57A729A4246D82B48B0FBF1F189B228463DF003FA96F88D
:205320004737B6F8001883B196F80838B1FBF3F128463DF0F7F9214628463DF0F3F92846B0
:205340000821F8F77BFA0120F8BD28463DF0EAF9F1E796F86970002FD5D01A48002300EBE9
:20536000830201339289BB421144F8DB164B9FED176A9B7E07EE103A07EE901AB8EEC77AE8
:20538000F8EE676AC6EE077A67EEA67AFCEEE77A17EE901AB1FBF7F1B5E71B7813B94EF6DF
:2053A0009C21B9E796F86970002FF8D00146D4E7E8B10020676666669D6100201783930390
:2053C000008793034CBC002040310020000048432DE9F04FAE4C89B094F8E88A054634F077
:2053E00067F8D4F8EC3AD4F8006B23F40013C4F8EC3AF307074648D500201EF059FF002807
:2054000040D0D4F85C2B002A3CD0900104D5B2F1007F18BF02F17E42D4F8601B9FED9D7AF3
:205420007B1A07EE903AF8EE677AF4EEC77AF1EE10FA05DCD4F8640B01238340134212D10A
:2054400011B91923C4F8643BD4F8643BC4F8607B012001331A2B28BF002300FA03F1114204
:20546000F7D0C4F8643BD4F8642B8B4B8B49686803EB82035A6B46F0C7FC02236B7309B048
:20548000BDE8F08F0023C4F8603BD4F8683B7BB394F88A37D9072BD4D4F86C3B9FED807AAC
:2054A000686803F5921303F57863DB1B07EE903AF8EE677A67EE877AFDEEE77AB8EEE77A87
:2054C00017EE903AF1EE0C7AB4EEE77AF1EE10FA05DB744946F098FC01236B73CFE70A2162
:2054E000B3FBF1F201FB12336F4946F08DFCF3E7B2050FD594F88F3763B16C49686846F0CD
:2055000083FC03236B73D4F8EC3A43F40013C4F8EC3AB4E7B30609D594F8703B33B16449F0
:20552000686846F071FC01236B73A8E7770536D594F8713B012B32D1D4F8703568689E0793
:2055400029D5B4F9823BB4F9AA28D21A6FF463739A421BDB40F28D339A421ADC0A2392FBEF
:20556000F3F2544946F050FC21F040FF524B1B6893F865300A3B23EAE3739842ACDBD4F8C2
:20558000EC3A43F40013C4F8EC3AA5E76FF05902E7E75A22E5E7494946F036FCE4E7B004E4
:2055A00012D514F065FF94F8F83A83420CD94449686846F029FC02236B73D4F8EC3A43F450
:2055C0000013C4F8EC3A5AE7310408D53D4BB4F94C2BB3F996319A4201DD3B49E8E77204E1
:2055E00007D514F02DFFB4F84A3B834201D93749DEE7330704D5B8F1020F01D134497DE70A
:2056000037050FD594F88A37D8070BD51EF0EEFD40B194F8FC37D90704D594F8BD3B0BB9B4
:205620002C49C5E7F20414D594F88A37DB0710D51EF0DCFD68B194F8FC37DF0709D4D4F808
:20564000C03BA3F53713A3F5D863002B01DA2249AEE7B4F84438580601D52049A8E7310609
:2056600040D5B4F9600A94F8123B98423ADB07F03FFE94F8F92A6E681949002A0CBF0D22F7
:205680000E220346009230467A2246F0BDFB92E7E8B100200024F44858CC06083DB6070839
:2056A000ACC5273756720708617207086E7207087872070883720708646500208D7207087F
:2056C0009472070868040020807807089D720708AA720708B4720708BF720708CA72070819
:2056E000D37207085F4B1B681A016BD5730669D594F8699004AAC9F10906760800239346A1
:2057000020219E421AD10BEB060057494FF0000A56F0B9FD03365246914501D90B2E11D9F8
:2057200008AB1E44002306F8103CBAF1000F49D04E4968685A4646F067FB3CE702F8011B3C
:205740000133DEE7D7B238460392FFF73FFD94F88AC7039A31371CF0010CFFB230D0B4F929
:205760000EEBBEF1FF3F2BD08189642311FB03F13F4B9B7E5B0891FBF3F39E45B4BF3B4668
:20578000522394F90C1B11F1800F04D090F901E08E45A8BF5423BCF1000F08D0B4F9101BF4
:2057A000B1F1FF3F03D040688842A8BF43239F420BF8063018BF0AF1010A01320136ABE704
:2057C0003B46DEE7D4F8003B5A0704D5B8F1010F01D12849ECE6DF050DD594F88A27D60794
:2057E00009D5254A92F82520012A04D1234A12780AB92349DCE6D8030CD594F88A27D107D4
:2058000008D5B4F8F42A2AB1D4F840188A4201DC1C49CDE69A0718D594F88A2794F8E81AC8
:2058200002F003020A4310D1B4F82E18B4F8002894F80808B2FBF0F2914206D91249686875
:2058400046F0E2FA01236B7319E6DB067FF517AE94F8E83B002B3FF412AE0C49686846F0F3
:20586000D3FA39E60C630020F67507083DB6070840310020E2720708745E0020AC6400201B
:20588000EE720708FA720708037307080F7307082DE9F8434A4C427894F8E93B02F00F05B1
:2058A000C3B9EDB92B46002184F8EC1BEB1AD9B20E290BD8234493F8481739B102F0F002E8
:2058C000802A4AD0902A5FD0A02A0DD000273846BDE8F8830021AB4284F8EC1BF6D8E5E784
:2058E00084F8E95B2B46DEE7412966D081F08003042B62D90846FBF7E1FF031D0246DBB29F
:20590000304884F8EC3B65F05F0584F8ED5BFCF787FC94F8EC7B002FD8D0BE1E16F0FF00CE
:2059200024D1FF25A946022756B1DFF89C80464418F8011BD4F8100C34F062FA4645F7D1CB
:20594000D4F8100C494634F05BFAD4F8100C294634F056FA3846BDE8F88365F07F050427EA
:20596000022684F8ED5B84F8EC7B3046164A4FF6FF71104412F8015B491B904289B2F9D1D8
:205980005FFA81F90D0ACFE7412914D081F08003042B10D90846FBF791FF65F06F05062747
:2059A000042684F8EF0B84F8ED5B84F8EE1B84F8EC7B3046DAE70420EFE7082304229FE713
:2059C000E8B10020D6BD0020D4BD00202DE9F047C31DDFF8348182B003F4FC7300AFD8F8DA
:2059E0008865ADEB030DC7F800D03268D8F8803568449A420C4698F8143C78606D4658D0F7
:205A0000591C0DF1010203F00F0388F8141C8DF800303A60A0EB0209D6E900125FFA89F9CA
:205A2000521A09F107035FFA82FA03F4FC73CA45ADEB030D55D25246684656F09FFB33681C
:205A4000534433605246694638463CF049FED8F88825D8F880353068117A7060C21A4A4089
:205A6000D2B28342336088F8152C09D00133336013F8011C984282EA0102F7D188F8152CEF
:205A80003B68591C39601A70D7E90032D21A012A08DD00215A1C3A601970D7E90032D21A45
:205AA000012AF7DC2846A04700200837BD46BDE8F087B6F90C20591C03F00F0343F010037A
:205AC000002A2A46B8BF43F0200302F8023B88F8141C691C3960D6E900135B1A3A606B709E
:205AE00098E74A46684656F049FB33684B4433604A46694638463CF0F3FD2846A047012053
:205B00000837BD46BDE8F087E8B100202DE9F04F7C4C83B0D4F88855D5E900535B1B002BC3
:205B200000AF83460D4616462ADD002384F8163CFBF738FF00200BEB05030BF1010AC4F83C
:205B40007835C4F874A59BF80050D4F884856909012940F09F8005F00F0915F0100514D114
:205B600050B194F8182C013202F00F024A4500F09A8084F8165C28460C37BD46BDE8F08FBF
:205B800094F8160C0028D6D1D2E70BF10203C4F874350BF103029BF80130D4F87C05C4F89B
:205BA00074259BF80250C8F80000C218C8F804206B404FF0000C84F8173CD4F874A5D4F873
:205BC000783584F8161CA8F80850A8F80CC0A3EB0A03DDB2121AEB1D5FFA82FB03F4FC736C
:205BE000AB45ADEB030D6BD25A465146684656F0C5FA0AEB0B035A4640466946C4F87435A9
:205C00003CF06EFDD4F87C35D8F8000094F8172C8342C8E900300AD00133C8F8003013F822
:205C2000011C984282EA0102F6D184F8172CD4F874351B78934239D1B8F90830FA2B54D05F
:205C4000D8F80020D4F87C35D4F88415D4F83007C8E90032D4F88825D4F8803553600025BA
:205C6000158195813B1D84F8165C7D602DF090F801303FD07B680BB100209847D4F8883549
:205C8000D4F88025196801200C37C3E90021BD46BDE8F08F00210846FBF768FE01200C378F
:205CA000BD46BDE8F08FD8E9000290E700230120B8F9081084F8163CFBF758FE01205BE7FD
:205CC0002A465146684656F059FA0AEB050340462A466946C4F874353CF002FD00200C37E1
:205CE00084F8189CBD46BDE8F08F002EA8D005233370A5E7D4F8882513680221581C106055
:205D00001970B7E7E8B100200B4B93F8262812B1B3F858274AB9B3F9AC38084AD81782FB36
:205D20000323C0EBA30000B27047D3F8400890FBF2F000B2704700BFE8B10020676666668C
:205D4000F8B5184CC6B205463146D4F81C0C34F057F894F8201CD4F81C0CC5F307274E4061
:205D6000394684F8206C34F04BF894F8201CD4F81C0CC5F307464F40314684F8207C34F032
:205D80003FF894F8201CD4F81C0C2D0E4E40294684F8206C34F034F894F8201C4D4084F8AF
:205DA000205CF8BDE8B1002070B50C4DC6B231460446D5F81C0C34F023F895F8201CD5F878
:205DC0001C0C240A4E40214685F8206C34F018F895F8201C4C4085F8204C70BDE8B1002017
:205DE00038B50B4C002305462421D4F81C0C84F8203C34F005F8D4F81C0C542134F000F83A
:205E0000D4F81C0C2946BDE8384033F0F9BF00BFE8B100202DE9F047DFF858A32DED028BE9
:205E20009AF8214C82B00F461646002C00F0E781013C8AF8214CDFF840839FEDC88ADFF881
:205E40003C933B78002B00F090809AF8214C002C40F08B8036B133F02BFB3368C01A002862
:205E600080F2DB839AF8221C002940F07A839AF8235C062D40F28481B94B93F89D0193F8F9
:205E80009C21824200F0AB81D3F898219AF8241C32F810400C440135013003F5CC73A4B251
:205EA000EDB2C0B2B4F5C06F8AF8235C587100F07E817CD8B4F5806F00F0298224D8B4F514
:205EC000067F4FD8B4F5007F54D3A4F50073182B48D8DFE813F0E701DE01DE01DE01DE012A
:205EE000DE01DE01DE01DE014700470047004700470047004700C601AB01AB01AB01AB01BE
:205F0000AB01AB01AB01AB01B4F5846F00F0E68140F2E280B4F5A06F00F064826FF4A06C4D
:205F200004EB0C03072B1DD8601EC0B2FFF74EF9C0B1B0F90C308B4AADF80140917EDAF81D
:205F4000342703EB830303EB830349089B0093FBF1F31021CDF803308DF80010684690475D
:205F600000233B70002E7FF46CAF02B0BDEC028BBDE8F087B4F5807F00F0FD81B4F5887FCD
:205F8000F0D1BAF9AE38CDF80330012210238DF800308DF801308DF80220DAF8343768465C
:205FA000002498473C70002E7FF44BAFDDE7B4F5046F00F0A48265D8B4F5006F00F0828258
:205FC0001AD9B4F5026F00F0F181B4F5036FC9D19AF8FC379D07C5D5634BDAF83427D9895D
:205FE0004FF4F36303FB01F3A8FB03135B091020CDF8033030218DE2B4F5E26F00F037826E
:020000040801F1
:20600000B4F5E46F1FD1594B93ED160AD3ED007A20EE270A002420EE080A53F0ABFD102375
:2060200020228DF800300723CDF803008DF802308DF80120DAF83437684698473C70002E76
:206040007FF4FFAE91E7B4F5E06F8BD1474B93ED140AD3ED007A20EE270A002420EE080A67
:2060600053F088FD10220723CDF803008DF802308DF80020DAF834378DF801406846984748
:206080003C70DCE740F678339C4248D8B4F5376F00F2E281B4F5116F00F08081B4F5376FA5
:2060A0007FF460AFFF20FFF791F800283FF45AAF90F90130CDF80330102170220B238DF834
:2060C00002308DF80010DAF834378DF801206846002498473C7066E740F201439C4200F028
:2060E0002882B4F5826F7FF43DAFDAF87035980600F146821E4B1B681B0640F194820024B7
:20610000102304228DF800308DF801308DF803408DF804408DF805408DF80640BBE145F2C2
:2061200030239C4200F0848145F240239C427FF419AFBAF9A838CDF80330102140225223F3
:206140008DF802308DF80010DAF834378DF801206846002498473C7025E700BF0000C842DE
:2061600068040020403100204464002030BA00200C630020E8B100201F85EB51C5B3A2915D
:206180000135CA4BEDB293F8A52193F8A411914220D0501CC0B25200D3F8A011C44B8C5A20
:2061A0008AF8235CB4F5C06F58717FF482AEDAF84038CDF803301022002406238DF8023022
:2061C0008DF80020DAF834378DF80140684698473C7034E7002283F8A5210120DCE79AF8EA
:2061E000242C9AF8690083F89D110132D2B2013082428AF8242C00F0B0810125C3E7002894
:206200003FF419AE0378303B012B3FF614AE01300AF621420621FFF779FC9AF8213C8AF8E4
:20622000220C002B3FF407AE3C7004E6A4F11100C0B2FEF7CBFF00283FF494AEB0F9023038
:20624000CDF8033010238DF80030ADF80140DAF834376846984700233B70002E7FF4F1ADA1
:2062600083E69AF84727BAF80038002A40F0CF8110220221CDF803308DF80020DAF83437F2
:206280008DF801208DF802106846002498473C7089E6601EC0B2FEF799FF00283FF462AE0D
:2062A0004368CDE7DAF838388249DAF8342781FB0301DB17C3EBA10300241021CDF8033034
:2062C00002238DF800108DF801408DF80230684690473C70002E7FF4B4AD46E69AF8FC3763
:2062E0009A077FF53FAEBAF8FE37CDF803301021202204238DF802308DF80010DAF834379A
:206300008DF801206846002498473C704BE69AF82C3C0133DAB2042A00F06E8142F21073CB
:206320008AF82C2C03FB02F3DAF85C2B002A00F0258102339AF88A27D507BAF8442848BFFE
:206340000433D40748BF0A33900748BF1433D10548BF2833550748BF6433540648BF03F577
:206360007A63102100240422CDF803308DF800108DF801408FE0DAF8283CCDF803301022A3
:20638000002401238DF802308DF80020DAF834378DF80140684698473C7050E69AF8083815
:2063A000002B40F02F811022092163E79AF8FC379B077FF5D7AD404ADAF834379268CDF847
:2063C0000320102220218DF8002008228DF801108DF802206846002498473C70002E7FF41D
:2063E00030ADC2E5FF20FEF7F1FE00283FF4BAADB0F90C303149DAF83427897E03EB83034D
:2064000003EB83031020490800249B0093FBF1F305218DF80000CDF803308DF801408DF868
:206420000210684690473C70002E7FF40AAD9CE5BAF9AA38CDF803301021302252238DF836
:2064400002308DF80010DAF834378DF801206846002498473C70A6E5A4F17100C0B2FEF73D
:20646000B5FE00283FF47EAD90F90130E8E6144B93ED150AD3ED007A20EE270A002420EEB2
:20648000080A53F077FB1023CDF8030007228DF800308DF80130DAF834378DF80220684614
:2064A00098473C70002E7FF4CCAC5EE5680400200806002067666666446400204031002049
:2064C00030BA00209AF8FC379C077FF54BADC107814B40F1B5805A6882EAE273A3EBE2737E
:2064E00003EB5303A8FB0313DB08002AACBF43F0004343F0404310210024082234E7BAF9AE
:20650000AC38DAF8342703EB83035B001020CDF80330402108238DF800008DF801108DF847
:2065200002306846002490473C70002E7FF489AC1BE5BAF9603ACDF803301021012204233E
:206540008DF802308DF80010DAF834378DF801206846002498473C7025E58AF8241C0125BD
:2065600011E65E490620FFF731FA00238AF8220C3B7002B0BDEC028BBDE8F0870133D9E6C1
:20658000554A9AF8FC17538A643BC3EB4370C3EBC00389FB03401844DB17C3EB2023093327
:2065A000092BA8BF092323EAE37303EB830311F0020F03EB830314BF4FF47A7000209B00FC
:2065C000C90748BF00F5FA60117DDAF834279BB203440B44042010218DF80200CDF8033023
:2065E0008DF800108DF801106846002490473C70002E7FF426ACB8E401238AF82C3C42F2CA
:20660000107391E6BAF80028B2FBF3F3CBE69AF80828002A57D113462AE63C7002B0BDECDE
:20662000028BBDE8F0879AF84637002B3FF49AAC9AF82D3C032B49D8DFE803F03B3122115B
:206640001A6882EAE273A3EBE27303EB5303A8FB0313DB08002AB8BF43F080434BE7DAF899
:20666000302C537A907AD17A03F1407303EB0023002203EB01438AF82D2C10220421F9E580
:20668000174A11688A7D087C897A120402EB00220A44591C8AF82D1C02EB0363EDE7104A5E
:2066A00011684A7DC87B497A120402EB00220A44EFE70B4A11680A7D887B097A120402EB6D
:2066C00000220A44E5E7B3FBF2F3D1E55A1C8AF82D2C1B06D1E700BF44640020F119010871
:2066E00064650020CA4A38B50820002382F8A531FBF754FA002800F08C80D2F8A0314FF4D3
:20670000806102204FF48264198082F8A50101465C804FF40020FBF741FA50B14B1CD2F8AF
:20672000A001DBB240F2014482F8A53120F811401946B84C94F82538002B6CD194F826385D
:20674000002B40F088804FF40070FBF727FA50B14B1CD2F8A001DBB24FF4046582F8A531B4
:2067600020F811501946D4F87045A50700F10181600700F1DB80A84B1B681B0600F1938053
:2067800000234FF4803082F8A41182F8A53182F89D31FBF703FAD0B3D2F8983101214FF4B2
:2067A000047082F89D1118804FF40040FBF7F6F950B14B1CD2F89801DBB24FF4007482F8B8
:2067C0009D3120F8114019464FF40030FBF7E6F950B14B1CD2F89801DBB24FF4A06482F8C6
:2067E0009D3120F8114019464FF48020FBF7D6F938B1D2F898014FF437644B1C20F8114065
:20680000D9B2002382F89C1182F89D3138BD0146CAE701467DE70120FBF7C0F900288DD072
:206820004FF48030FBF7BAF9D2F8A05128B94FF4047325F811300131C9B20BB2481CC1B2CB
:206840004FF4116082F8A51125F8130094F82638002B3FF478AF0220FBF7A0F900283FF4AD
:2068600072AF4FF40040FBF799F950B94B1CD2F8A001DBB24FF4007582F8A53120F8115007
:2068800019460420FBF78AF900283FF45CAF4B1CD2F8A001DBB24FF4C06582F8A53120F86B
:2068A000115019464FE74FF40050FBF777F950B14B1CD2F8A001DBB24FF4036482F8A53193
:2068C00020F8114019464FF48050FBF767F968B1D2F8A0014B1C4FF40064DBB28D1C20F8AB
:2068E0001140E9B282F8A51120F813404FF48040FBF754F950B14B1CD2F8A001DBB24FF42C
:20690000846482F8A53120F8114019464FF48060FBF744F900283FF433AFD2F8A0014FF43A
:2069200002644B1C20F81140D9B229E74FF48060FBF734F950B14B1CD2F8A001DBB24FF4A1
:20694000807482F8A53120F8114019464FF40060FBF724F900283FF40EAF4B1CD2F8A0018F
:20696000DBB24FF4887482F8A53120F81140194601E78020FBF712F950B14B1CD2F8A001DB
:20698000DBB245F2302582F8A53120F8115019464FF48070FBF702F950B14B1CD2F8A001C3
:2069A000DBB245F2402582F8A53120F8115019461020FBF7F3F850B14B1CD2F8A001DBB219
:2069C0004FF4E06582F8A53120F8115019462020FBF7E4F850B14B1CD2F8A001DBB24FF456
:2069E000E26582F8A53120F8115019464020FBF7D5F800283FF4BCAE4B1CD2F8A001DBB2E5
:206A00004FF4E46582F8A53120F811501946AFE668040020E8B100200C63002030B5A0F1E3
:206A20007D03012B044683B00D46104608D9214633F0E6F915B1288804442C8003B030BD30
:206A40007D21019233F0DCF9019884F0200133F0D7F9EFE730B50F4B85B0D3F87C27002311
:206A60000446C51DADF80E3014F8010B01920DF10E01FFF7D3FFA542019AF5D10DF10E0033
:206A800014F01EFC019A9DF80E000021FFF7C6FF05B030BDE8B100207E28F8B50F4652D099
:206AA000324E96F8A84164B9314D95F83C1C51B11B2885F83C4C3DD00D2837D0012386F82A
:206AC000A8310020F8BD7D284AD095F8402C1AB180F0200085F8401C95F83B2C062A14D80C
:206AE000B5F83E4C511C2A440444C9B2A5F83E4C85F83B1C82F8340C002BE2D10729E0D14D
:206B000001231C4886F8A831F8BDB5F83E3C1844C0F3072353FA80F0FF284FF00103A5F8BD
:206B20003E0C86F8A831CCD11248F8BDA5F83E4C2046F8BD90470028C0D0012320463B7002
:206B400086F8A831F8BD0A4B084A0024012183F83B4C83F83C1C3C7082F8A8412046F8BD3D
:206B60000123084685F8403CF8BD00BF68040020E8B100201CBE0020044AD2F8443C43F428
:206B8000DF2343F48063C2F8443C7047E8B10020013070B5094EC4B203E045F06BF901345B
:206BA00048B9E5B2152D21463046F6D9162D04BF034B93F8485C284670BD00BF2CBE002068
:206BC000E8B1002000B1D7E7044AD2F8443C23F4DF2323F48063C2F8443C7047E8B1002038
:206BE00070B5114C84B00546D4F84C0C0E462BF01BFC94F8402794F84137003A18BF0122BF
:206C00000BB142F00802CDE9016200234FF4964195F9000000911A4608212BF0A8FCC4F803
:206C20004C0C04B070BD00BFE8B1002010B5064C03E0D4F84C0C33F0D7F8D4F84C0C33F04C
:206C4000DBF80028F5D110BDE8B1002010B50D4CD4F8503C1B791E3B012B0DD9D4F84C0C54
:206C600001213830FFF7BCFF0023C4F8543C84F8583CBDE81040D9E7D4F84C0C012133F03C
:206C8000ABF8F1E7E8B10020F0B5C64C94F8603CD4F87015C4F85C0C0133880785B084F8F8
:206CA000603C12D411F0340F35D1090794F8602C42D412F007055BD0282A00F0BB80D4F848
:206CC00038375E20984705B0F0BD7020FAF766FF0028E7D004F69806242504F64807F6ECB5
:206CE000017A97ED007A67EE877A2846FDEEE77A013517EE901AC1EB411301EB8301C900ED
:206D000009B2EDB2FAF7ACFE272DE8D1D4F8701511F0340FC9D04FF40060FAF73FFF002849
:206D200040F0058194F8602C12F0030100F0DB80D4F870150907BCD54FF40070FAF72EFF71
:206D40000028B6D012F00305B3D1974AB4F9AC38D91782FB0323C1EBA30109B21420FAF7C2
:206D60007FFE29461C20FAF77BFE94F8602CA0E7FF20FEF72BFA002800F0DF800378FF2B8D
:206D80007AD090F901100220FAF76AFEFF20FEF71DFA002872D00378FF2B6FD0B0F90C2046
:206DA000824B8148997E02EB820202EB82029300490893FBF1F3D91780FB0320C1EBA00014
:206DC00001B20320FAF74CFE94F82538002B5DD1D4F870359A067AD54FF40050FAF7DEFEA0
:206DE000002840F0C980724D4FF48060FAF7D6FE002840F049816B8A94F8602C297DB3F5CE
:206E0000967F02D9100740F10E8194F84337002B40F0958009B20520FAF722FE4FF4805031
:206E2000FAF7BCFE002840F0D58094F8602C282A7FF445AF5F4A604B15686049A3FB0535D7
:206E4000AD09A1FB05367609A1FB06314909C1EB0111A6EB81010902C6EB0616002309B27A
:206E60001720A5EB860684F8603CFAF7F9FD31B21820FAF7F5FD22E7294684E7002103209B
:206E8000FAF7EEFD94F82538002BA1D00120FAF785FE002840F00A8194F82638002B97D09D
:206EA0000220FAF77BFE002840F059810420FAF775FE00288CD0B4F82838002B00F05C8104
:206EC00029F05CF901B20420FAF7CAFD80E71B07ABD53B4B93E8030002AB83E8030018462F
:206EE000FAF7D4FDA1E74FF48060FAF757FE00283FF41EAF334BD4F85C2CD4F8285C9A42B9
:206F000040F20A81304BE91783FB0523C1EB6313642101FB13510DB219B21020FAF7A0FD44
:206F200029462120FAF79CFD94F8602C00E7B4F9AE183020FAF794FDF4E6014623E7A1F116
:206F4000200307EE903A9FED217AF8EEE77AF6EE006A67EE877ABEEE007AF5EEC07AF1EE1B
:206F600010FA58BFB0EE667A77EE877AFDEEE77A17EE903A19B24EE794F8FC379F0758D460
:206F80004FF48060FAF70AFE094D00283FF433AF002631460120FAF763FD31460920FAF7A2
:206FA0005FFD28E7E8B1002067666666403100204464002098240020D34D6210898888882C
:206FC000F4CC06083F4B4C001F85EB51E4380E3F0050C34794F8FC2700239207CDE9003316
:206FE00047D494F8643C012B43D0B4F93C375FED086A07EE103AB4F93E3707EE903AB8EE67
:20700000C77AF8EEE77A27EE267A67EEA67ABDEEC77AFDEEE77A02A88DED027ACDED037AAF
:20702000FAF734FD01E742F20F719942A8BF1946EBE6544D544BE9894FF4F36606FB01F1DF
:207040004909A3FB0131C9091120FAF709FDE9894E4B06FB01F1A3FB01214909A3FB012342
:207060005B09642202FB131109B21920FAF7F8FCBAE6D5E9002301216846CDE9002384F886
:20708000641CFAF703FDD0E694F8FC379E077FF57FAFAB683D4AD91782FB0302C1EB621198
:2070A000642606FB113636B209B273E794F8081800293DD10B460620A4F8623CFAF7D0FCB0
:2070C000B4F8623C0133A4F8623C29F04BF894F8443794F80828012B94F847371ED000EBCA
:2070E000800086B213B10AB1B6FBF2F6274BA3FB062343F34F113A205D09FAF7B1FC64210E
:2071000001FB1561224B89B20531A3FB0131C9083B20FAF7A5FCBFE60D46FEE61BB112B126
:20712000B0FBF2F080B201B23920FAF799FCB3E6B4F8620CB4F80028B0FBF1F301FB1303D6
:20714000642000FB02129BB24900B2FBF1F2110241EA0311C2F30322114309B2ABE7D4F8DD
:2071600038380C49DA1781FB0313C2EBA30319B22820FAF775FC99E6D4F8403883F31003B3
:2071800019B2A0E644640020C55A7C0A1F85EB51CDCCCCCC676666660B2814D810B401EBB8
:2071A0004103094C01EB83032344184490F8C038934205D02144002380F8C02881F8B4388A
:2071C0005DF8044B70477047E8B10020F0B5464C94F8653C012B83B0054650D994F8660CAF
:2071E0004249434E94F8677C421CA1FB02C1184406EB800001F4FE7606EB9101521AD0F85A
:20720000A46084F8662C2FB1D4F8681C04F66C4291420DD06EB9374A0133A2FB031222F034
:20722000010101EB52029B1A84F8653C03B0F0BD314E94F8803C93B9304B019348F2A501D8
:20724000123B15226F46A4F8841C009384F8862C29463846B04758B994F8653CDBE76F465F
:20726000384611F069FB29463846B0470028F3D094F8801C59B1384611F0D8FAECE71C4AA0
:2072800002EB8302D2F8A460002EC4D0D1E7009E1B4A964214D9013A013E41F2210512F88F
:2072A000013F81EA0321082311F4004F85EA41000ABF490081B289B2013BF5D19642EED1B7
:2072C00038463BF055FA0F49009D6D1A152DA8BF15252A4601F1180054F050FF94F8653C1D
:2072E00084F8B15C97E700BFE8B10020CDCCCCCC58CC0608ABAAAAAAB926010881BE0020BC
:207300006FBE00206CBE002070B50B4E054606F6B64140F005FC2C686C6006F6B441641A1A
:20732000402CA8BF40242960224606F6F44054F025FF86F8344D70BDE8B1002030B50C4B6C
:207340000C4AC3F8B42C83B0C822014603F6F44503F6B94483F8B82C68463A22CDE900454C
:207360003BF0BEF96846FFF7CFFF03B030BD00BFE8B10020C83E7BEA03685A0607D513F488
:20738000057F04D007298CBF00200120704703F48253B3F5825F03BFC81FB0FA80F04009C1
:2073A0000020704770B5BD4C94F8353D012B84B000F04E8194F8410DFBF71AFE94F8423DBC
:2073C000834205461FD0002800F0D780D4F8503CCBB194F8412793F90400002A18BF0822BC
:2073E0004FF4964100230325CDE9015200911A4608212BF0BCF8C4F84C0C20B1FFF726FC39
:20740000012384F8423D94F8433D012B00F0C280D4F84C6D3EB1A24B30465978FFF7ACFF9A
:20742000002840F0F38094F8510DFBF7E1FD94F8503D8342054622D0002800F0F780F6B176
:20744000337A002B00F01981964A02EB8303D3F8C03094F8402796F904000093003A18BF92
:20746000012202210023CDE901121A4610212BF07EF8C4F81C0C10B1012384F8503DD4F81A
:20748000546D3EB1864B30465978FFF775FF002840F0AC8094F8600DFBF7AAFD94F8583D83
:2074A0008342054623D0002800F0C980FEB1337A002B00F0E5807B4A02EB8303D3F8C03099
:2074C00094F8402796F904000093003A18BF012202210023CDE901121A464FF400712BF021
:2074E00046F8C4F85C0D10B1012384F8583D94F8610DFBF77DFD94F8623D8342054630D092
:2075000088B3694BD4F8646D4FF47A72C3F8BC263EB34FF48052402130462AF0B3FF05461F
:20752000F8B994F8403796F90400002B14BF0921082103224FF4E133CDE9012100932A465C
:207540002B464FF480512BF012F8C4F8680D40B10123C4F8100C84F8E95B84F86C5D84F8E2
:20756000623D04B070BDD4F8680D2AF05DFFC4F8685D84F8625D04B070BDD4F84C0C2AF0F9
:2075800053FF94F8433DC4F84C5C012B84F8425D7FF43EAF94F8440DFBF72AFD0546002819
:2075A00071D0D4F87C37002B7FF432AFD4F8482D002A3FF42DAF94F8415794F8401792F980
:2075C0000400002D14BF08220022002908BF42F0010203254FF46141CDE9015200911A462F
:2075E00020212AF0C4FFC4F87C0711E794F8583D002B7FF47CAFD4F83C3D002B3FF477AF83
:207600000122C4F85C3D84F8582D70E794F8503D002B7FF434AFD4F83C3D002B3FF42FAF7F
:207620000122C4F81C3C84F8502D28E7D4F81C0C2AF0FAFEC4F81C5C84F8505D1FE7D4F8D6
:207640005C0D2AF0F1FEC4F85C5D84F8585D4EE7D4F8385D124B28465978FFF78DFE28B384
:20766000D4F8F837002B7FF4A5AED4F83C3D002B3FF4A0AEC4F8F8379CE64FF49643E8E6D6
:207680004FF461431CE7D4F87C0700283FF4C0AE2AF0CAFEC4F87C57BAE600BFE8B100205F
:2076A000545E002058CC06086804002094F8400DFBF79EFC0646D8B1D4F8F837002B7FF467
:2076C00079AE002D3FF476AE94F8402795F90400B2FA82F252094FF416510225CDE9015225
:2076E00000911A4604212AF042FFC4F8F80761E6D4F8F80700283FF45DAE2AF095FEC4F87D
:20770000F86757E670B5B14C94F8353D002B00F0218108202AF0CAFEC4F8500C00283BD09B
:2077200008212AF0B9FE00260346A949A94884F8413DC4F8746D37F05FF841F20853012237
:20774000A448A4F8783D84F87C2D0DF043FD31462B22A14854F073FD48F67C607D25E0236A
:2077600031462B22A4F8840D9C4884F8873D84F8AF5D54F064FD48F67C21A0224EF27B036C
:2077800084F8DB5D84F8DE6D84F8875EA4F8B01D84F8B32DA4F8DC3D94F8433D002B00F06C
:2077A000C38010202AF082FE1021C4F84C0D2AF073FE8B4B84F8510D3A2140F23B1094F8D7
:2077C000252818809F254AF21E40197100219D7198601973002A40F08E8094F82638002BAC
:2077E00048D1D4F8703558077ED4990773D41A076AD47C4D2868C0F3C010FFF7E3F900203A
:20780000FFF7C6F903464FF4007084F8483C2AF04DFE4FF40071C4F8540D2AF03DFED4F860
:20782000883E84F8600D002B14BF0123002384F88C3E26D1D4F8FC2E0023C4F8F83E002AE2
:2078400069D0012284F8803C84F8002F4FF480502AF02CFE4FF48051C4F8640D2AF01CFE1D
:20786000002384F8610D84F8623DFAF79BF8BDE8704097E5D4F8443C43F00403C4F8443CC9
:20788000AFE7D4F87025002312F0020284F88D3E84F88E3E40F0828094F8253823B1012029
:2078A000FAF77CF9002873D194F82638002B6AD1A3182868042183F8901E030602F101010F
:2078C00075D484F8941EB5E7D4F8443C43F48073C4F8443C8DE7D4F8442C42F4601242F059
:2078E000C002C4F8442C82E7D4F8442C42F40272C4F8442C79E7D4F8443C94F8262843F066
:207900000201C4F8441C002A3FF46BAF43F03603C4F8443C65E7D4F8043F7BB3012384F800
:20792000003F84F8803C91E720202AF0BFFDC4F8480D00283FF435AF20212AF0ADFD2A4B78
:20794000C4F8343784F8440DFEF7CCFE012384F8433D26E704202AF0A9FDC4F8380D00283A
:207960003FF4D7AE04212AF097FD204A84F8400D0123C4F8382784F8353DCAE684F8003FB1
:2079800084F8803C62E70620FAF708F900288FD0A318022183F8901E013289E74FF460700A
:2079A000FAF7FCF878B1012284F8902E74E74FF45850FAF7F3F8002883D063180820911C6F
:2079C00083F8900E7DE7024666E700BFE8B1002058CD060858BF00206CBF002098BF0020F1
:2079E0001C6400200C630020556A010811220108094BB3F81E28B3F81C38801A9B1AC00001
:207A000090FBF3F00628A8BF062020EAE070C0F19600C0B2704700BFE8B1002010B5094BE2
:207A20000022D3F8081F03F60C73914201D1002010BD13F8014B844201D00132F5E701200A
:207A4000F6E700BFE8B100201B4B2DE9F04103EB81038EB0D3F8507106460D4647B3174BED
:207A600003EB41031C22B3F8484F002319460DEB0200069304F01F0854F0E1FBC4F34414F5
:207A800001228DF8085006AD8DF81420CDE903568DF809808DF80A4002A8B8479DF814201C
:207AA00000232AB100952246414602A805F03CFF0EB0BDE8F08100BF58CC0608E8B10020EC
:207AC0000A4B03EB4002B2F8481F094A92F86C2902EAD122520707D0D3F8082F511CC3F865
:207AE000081F134483F80C0F704700BFE8B100206804002010B5164B42681B7803F003035B
:207B0000032B21D1134B1B88DBB1134B1349B3F90030B1F904100A2491FBF4F15B1A1B0134
:207B200003F5B95314334FF4B471B3FBF1F3C3F1080303F00F0360331370436800225A708F
:207B400010BD05231370F8E72D231370F5E700BFE4B90020E6B900203CC3002090BA00205B
:207B6000436872221A70436873225A70436874229A7043680022DA7070470F4B4268B3F969
:207B800004300A2193FBF1F31B0110B503F5B9530A4C4FF4B4711433B3FBF1F303F00F0393
:207BA000E118E35813604B6853600B7A1372436800225A7210BD00BF90BA0020C8CE06087B
:207BC000084B5B7933B942F210735843064B90FBF3F07047242358434FF47A7390FBF3F04A
:207BE000704700BFDCBC002040D20600044B5B792BB94FF4A4735843642390FBF3F0704797
:207C0000DCBC0020831E00F17402EA2123F8021F9342FBD143F649134385CD2383804E23FB
:207C2000C380CE2303812323A0F87230704700BFF8B91D48438803F0010353BB30B404794F
:207C4000ACB11A4A02F1F00502E00133A3420ED052F8041B4904F8D590F8F01000EB81012A
:207C6000D1F8881045F823100133A342F0D130BC70470D484288032A4FEA52030AD90A6887
:207C8000438002F5C332A03203F001030A60002BD4D070470B6803F5C333A03348F2050207
:207CA0000B604280704700BF3CC3002044C300202DE9F041002839D12C4A107980B32C4ABA
:207CC0002C4B92F800E092F901C092F90280CEF1FF07AEF17F06FFB2F6B203EB800003F1C6
:207CE000F002002403E0834202F1040218D053F8041B8904F7D5E1B2A1EB0C0181EAE17535
:207D0000A5EBE175012D0DDC71B1414514BF394631468342D17004F1010402F10402E6D145
:207D2000BDE8F0810821F4E77146F2E7104B1A78F02A09D802F10F000C4A18700B6803F566
:207D400082431A330B60B8E7084A93F9014090797F2584421D70987805DB4042C0B29870FC
:207D600020445870EAE7002CFADAF6E73CC30020D80D002044C30020F0B5354E78B196F8FF
:207D80007831002B45D0334A013BDBB286F878311378DC073FD4304B0A681A440A603479AA
:207DA0004CB32E4B2B4F03EB840403F1F001002503E09C4201F104011DD053F8042BC2F37D
:207DC00003200628F5D13878C00715D596F8780196F807E000EB050CBCFBFEF00EFB10C035
:207DE0000128CCBF0020012058B99C4205F1010501F10401E1D1F0BDE84300F00100002809
:207E0000F3D0C2F3834206EB8202D2F888200A60EBE7F379B7E7124A124BB2F90620124814
:207E2000A2F57A74642202FB04F283FB0234D317C3EBA41303EB4303C3EB031380FB0302C9
:207E4000DB17C3EB62130533084A92FBF3F3A3E73CC3002072B90020400D030044C30020A5
:207E600008660020D34D62101F85EB5140420F00F0B4524C002867D194F87901002855D07C
:207E80004F4BD3ED007AB3EE097AF4EEC77AF1EE10FA4DDCBBEE097AF4EEC77AF1EE10FA7D
:207EA0004CBF08270027D3ED017AB3EE097AF4EEC77AF1EE10FA3DDD47F001072579ADB39F
:207EC000404ADFF80CC102EB850502F1F00014E094F97C61B142ACBF0221002194F97D61AF
:207EE000B3421CDB41F004010F421CBFDCF824300360954200F1040018D052F8043BD90390
:207F0000F7D594F97B6103F00F01B142C3F30313DEDC94F97D61B3424FF00101E2DA94F9C6
:207F20007E61B342D8BF41F00801DDE7F0BC70470427B8E7BBEE097AF4EEC77AF1EE10FA73
:207F400048BF47F00207B9E794F87A3163B31C4B1D4DD3ED007A93ED017A0A6894F879016F
:207F6000F0EEE77AB0EEC77AF4EEC77AF1EE10FAB8BFF0EE477AFDEEE77A80F0010017EEFF
:207F8000903A193B03EB4303C3EB031385FB0365DB17C3EBE51305330C4DB5FBF3F31A44C6
:207FA0000A6084F8790169E70B6894F8790103F5433303F5A0730B6060E700BF3CC300208F
:207FC000F4B9002044C30020353AFC4440420F00C8CE0608F0B40A4F3E797EB107F10802E4
:207FE0000546F837002352F8044B35EA040004BF086847F823000133B342F4D1F0BC704742
:020000040801F1
:208000003CC3002030B42A4B60B92A48027DCAB993F8F1302849203301EB830130BC4FF44C
:20802000A060D7E793F87F21F2B1013A214883F87F210A6802F5C32202F520720A60027D35
:20804000002AE5D01D4A12689106E1D51C4A93F87F11127892071AD511BB93F8F3301649A7
:20806000203301EB8301D9E7124893F88041057DA54205D8042483F8802183F87F41D8E753
:208080000134012283F8804183F87F21D1E70029BED193F8F2300849203301EB8301BDE75C
:2080A00093F8EF300449203301EB8301B6E700BF3CC300204464002044C3002058B700206D
:2080C000E4B9002010B450B91E481F4C90F881210B6823440B60A2B15DF8044B70471B4BC2
:2080E0001B7813B3012B17D016480B6890F88121174C82F00102234480F881210B60002A2B
:20810000EAD190F8EF3013495DF8044B203301EB83014FF440705DE70A480F4C90F881212C
:2081200082F0010280F88121D2E70B68054A5DF8044B03F5742303F5107301200B6082F881
:20814000810170473CC3002040420F00D0BC002048E8010044C3002020A107003C4AA0B98B
:2081600092F882316BB192F883118A081341DB070AD501F00101032A06D8DFE802F0504892
:20818000403892F8843153BB704792F88331013303F00F0382F883313BB192F88231086825
:2081A00000F5C330A0300860DCE72A4882F88231437A002B44D12848C07818B143F0040395
:2081C00082F8823125480078C00730D5244800780028E4D043F0080382F88231DFE792F846
:2081E0009231204901EB83014FF40030F2E61D4B03F13002002914BF19461146F4E71A4B18
:2082000003F1180200290CBF19461146ECE7154B03F10802002914BF19461146E4E7114B9C
:2082200003F11802002914BF19461146DCE70F4800680028CAD043F0010382F88231C5E72A
:208240000B4B1B78002BB6D0022382F88231B2E73CC3002004BA002074B9002072B9002004
:2082600058BD0020E0CE0608F0CE060844BD0020D0BC002030B4022340F203154FF4FA7470
:2082800032210122C37000238580C480018130BC82720380704700BF90F8603043B94269AF
:2082A0000121072082F84430A2F8460082F84810704700BF034A0123E021C3735170184698
:2082C000704700BFC4BF00204FF0FF30704700BF4FF0FF30704700BF704700BF0020704770
:2082E0000020704770B4067AAEB1427A0B4800212025002352B1142B05DC072903DCC45CBA
:20830000202C18BFC55401339342F4D101318E4200F11500EDD1002070BC7047C7BF0020E4
:2083200010B50024C473FFF7DDFF024B01225A70204610BDC4BF002070B403980378ABB1A5
:208340000C4C02EB4205C5EBC5052544142901F1010406D8072A294403D8CE789E4218BF26
:20836000CB7010F8013FE1B2002BEFD1002070BC704700BFC4BF002014299DF800000CD8E1
:20838000072A0AD8064B02EB4202C2EBC2021A441144CB78834218BFC8700020704700BF77
:2083A000C4BF0020027A407A02FB00F0704700BF027A407A02FB00F0704700BF0020704711
:2083C000002070474FF0FF30704700BF034B93F8BD22027293F8BE32437270473CC30020B0
:2083E000002070470120704700207047027A407A02FB00F0704700BF002070470123C3732D
:20840000184670470123C373184670474FF0FF30704700BF704700BF0020704701207047CF
:2084200000207047027A407A02FB00F0704700BF002070474FF0FF30704700BF704700BF9B
:20844000002070470120704700207047027A407A02FB00F0704700BF00207047002070474F
:20846000002070470120704700207047014B1878704700BF9C240020914201D0012A01D99B
:20848000002070470129FBD808B5074BC1EB0110C2EB021203EB421103EB40104FF4F07257
:2084A00053F06CFE012008BDA024002001299DBF024B012083F8C012002070473CC300200E
:2084C00001298CBF00200120704700BF4FF0FF30704700BF002070470020704730B41D29B4
:2084E0009DF808000DD80F2A0BD8074B074D93F8C0421E23C4EB041413FB021202EB44123E
:208500005055002030BC70473CC30020A0240020014B9888704700BFD80D00200020704732
:20852000024B0020C3F8C402704700BF3CC30020074BB3F81A14B3F81C24034610B4054C44
:208540001C6001205DF8044B19815A81704700BF3CC3002018CF0608064AB2F810340BB9D9
:208560001846704792F81834037292F819344372012070473CC3002000207047034B93F868
:20858000190493F8183400FB03F070473CC30020002070477047037913F0020308D00369CD
:2085A000D0E90920013B101A1840C0B2181A70471846704701717047704703799B070AD5CE
:2085C000436A8269D154436A01690133B3FBF1F201FB123343627047037913F0010306D00C
:2085E000D0E90732C0689B1A0138184070471846704710B5037913F0010301460DD0FFF7ED
:20860000EBFF60B10A6A4B69CC689B5C0132B2FBF4F004FB1022DBB20A62184610BD0346AA
:20862000FBE790F84F3830B53BB990F84D1890F84E380124DAB2914200D830BDB0F85658D6
:2086400004FA03F22A43A0F856280133F2E7D0E90920131A58425841704700BF014BD3F8C8
:20866000340470473CC30020034B002283F8382483F83924704700BF3CC30020024B6FF08C
:20868000020298689A607047D80D002070472DE9F04F754C89B094F83A340490002B42D04F
:2086A00094F83B3403F0FF07002B3CD16F4BD4F83CC41A7B0593002A0CBF63462023019366
:2086C000B4F8443403934FF03C0EB4F8463494F840A494F8412494F8421407970293754600
:2086E0004FF00109019BBB4220D184F84124059A84F8421400235E491373012284F83B2407
:2087000051F8082C51F8041C84F840A440F22A3050604B620B889BB243F001030B8013680D
:2087200043F00103136009B0BDE8F08F674536BF504B07AE03EB8706B378F078C3F1FF03FD
:208740009BB2002B00F08A80C3F1FF0343433688B6FBFEFB1B12BBF1050F00F28280DFE85B
:208760000BF0032B3C4B5C6DC21A7243B2FBF5F252FA83F2D9B2D2B2049B3F4E012B0BBF69
:208780001302030243EA004343EA024343EA0108602303FB076A1726039B09FA06FB1BEAD1
:2087A000080F9B46029B18BF9B46013E4AF804BBF2D20137824695E7B6FBF5F205FB1266DC
:2087C000B6B2C21AC6F13C06D9B27243B2FBF5F252FA83F30246D8B2CEE7B6FBF5F205FBA7
:2087E0001266C11AB6B27143B1FBF5F151FA83F10246C9B2D8B2BFE7B6FBF5F205FB1266B6
:20880000B6B2C21AC6F13C067243B2FBF5F252FA83F20146D2B2D8B2AEE7B6FBF5F105FB90
:208820001166A0EB030AB6B2DAB206FB0AFABAFBF5FA5AFA83F30146D8B29DE7B6FBF5F1D6
:2088400005FB1166B6B2C6F13C06C11A7143B1FBF5F151FA83F1DAB2C9B28DE70146024656
:208860008AE7504688E700BF3CC30020D80D002034D4002034C4002084C70020074910B5DF
:208880000246002301F1F804D1F83C04984200D810BD106844F823000133F5E73CC30020F1
:2088A000034B5A7B0AB901225A730020704700BFD80D0020134B144A197801B31349097869
:2088C000D1B91349D161134A5A60134A134912681A72134ADA603032DA63124A5A66124AFC
:2088E000596312491268096883F86820104A83F83810DA66002070470E49D161E3E70E4995
:20890000D161E0E734D40020D80D00202CBC0020A4CF060824BC00204CB2002025BC002089
:2089200044D4002028BC002000B2002014B20020B4B900203ED00608BCD006080348044B66
:20894000B0F870201A807430704700BF34D400202ABC0020034B1A88034B0020A3F8702074
:20896000704700BF2ABC002034D40020064B93F90030012B06D0054BB3F87A20A3F878207C
:2089800000207047024870473405002034D40020A8D4002008B5064B1A782AB1054A12788E
:2089A000012A1CBF00221A70FFF784FF002008BD2CBC002022BC00200A4B93F900200A4B4B
:2089C00012B91A70002070471A780AB90122F8E7064B93F87C20012A84BF012283F87C20F4
:2089E000F0E700BF3405002028BC002034D400200B4A0C4B92F9001019B983F87C1000201C
:208A0000704793F87C1019B9012283F87C20F6E7054B92F9022019788A4218BF1A70EEE70F
:208A20003405002034D4002028BC0020034B0449B3F900304068012243F0E6B9FE0500207A
:208A40004A720708064B07491A88074B40681B68534342F2107293FBF2F243F0D5B900BF4D
:208A6000E8B90020F574070820BA0020044A05495378127840680133013243F0C5B900BF53
:208A8000945D0020FA7407081C4B1A6812F0200F13B502F00403446829D0194A1278910743
:208AA00025D5184BB3F90000FFF7A0F86421002890FBF1F301FB13014FF00A0091FBF0F13D
:208AC00011484079B4BF762275220029B8BF494200280CBF99209F20002BCDE90010B8BFE4
:208AE0005B420A49204643F08FF902B010BD002BD7D12D22227042685370F6E758B70020B9
:208B0000E4B9002096BA0020DCBC0020007507080B4B4068B3F904300A2293FBF2F31A0154
:208B200002F5B9524FF4B4711432B2FBF1F2C2F1080202F00F020349603243F065B900BF47
:208B400090BA00200E750708034A044992684068072343F059B900BF20BA0020157507081C
:208B600007B5114A406892F88030B2F87E10012B09D1009192F881300C497B2243F044F990
:208B800003B05DF804FB0A234B4340F2FF32B3FBF2F39BB2092B064928BF09237B2203B0EA
:208BA0005DF804EB43F030B934D400201B750708257507081E4B1A6812F0200213B50146C7
:208BC0001AD01C4B1A7812F0010215D01A4B1A7812F0020210D0194BDB89632B1FD9642019
:208BE0005843FEF7EDFF002819DD154B1B684FF47A725A4392FBF0F2124B48685B79541E6A
:208C0000002B42F20E710CBF7E237D238C4208D800930D49072343F0F7F802B010BD0022E6
:208C2000EAE70A49072202B0BDE8104043F0ECB858B7002072B90020E4B90020446400206A
:208C400020BA0020DCBC00202B7507083475070813B50D4B446893F88B200C4B8AB1988946
:208C6000FEF7AEFF0A4A0B495279002A0CBF9D229E22034600922046702243F0C5F802B0F6
:208C800010BDD889ECE700BF34D4002044640020DCBC00208F77070830B5124A124B92F82F
:208CA0005A2040681C7D85B0AAB10A215A8AB2FBF1F5B5FBF1F301FB13539BB202930B499B
:208CC0006423B2FBF3F21F23CDE900421E2243F09BF805B030BD064900941F231E2243F001
:208CE00093F8F6E7DCBC0020446400203E7507084C7507080C4B40685B689822002B10B48F
:208D000002700EDA2D2242705B4202240749B3FBF1F2204401FB12335DF8044B044943F08B
:208D200073B80124F2E700BF4464002080969800547507080C4B40681B688922002B10B4E1
:208D400002700EDA2D2242705B4202240749B3FBF1F2204401FB12335DF8044B044943F04B
:208D600053B80124F2E700BF446400208096980054750708044B1B78DB0703D4034940684E
:208D800043F042B8704700BF72B900205C75070807B5094A0949B2F906300193B2F9043050
:208DA0000093B2F902304068B2F9002043F02CF803B05DF804FB00BF74280020657507080E
:208DC00013B5094B1B689A24002BB8BF5B4264210094B3FBF1F2406801FB1233034943F0E5
:208DE00013F802B010BD00BF20BA00207975070837B50378114A1A2B0CBFB2F90250B2F9B9
:208E000000500A211A2B95FBF1F408BF152201FB145118BF1422002DB4BF2D232023002955
:208E2000B8BF4942002CB8BF6442019100940449406842F0E9FF03B030BD00BF90BA0020E9
:208E4000847507081E4B37B51A68446812F0200F02F0040329D01B4A1278920725D51A4B7D
:208E60001A4D1868FEF7C2FE7F220A2390FBF3F309302270BCBF2D2262706D79B4BF022035
:208E80000120002BB8BF5B42002D4FF00A010CBF0F250C25B3FBF1F2009501FB1233204400
:208EA0000B4942F0B1FF03B030BD002BD7D17F22227042682D21517042689370F3E700BFD7
:208EC00058B70020E4B9002010BE0020DCBC002002750708084BD3F89020002A0BDD074B48
:208EE00003EB8203D3F838222AB1054B05491B6A406842F089BF704734D40020C8CE060837
:208F0000D80D00209275070807B5937801935378009313780A46034942F076FF03B05DF8A7
:208F200004FB00BF9A750708024B03491A6840681432E9E764650020A9750708024B0349CD
:208F40001A6840680832DFE764650020AD750708024B03491A6840680E32D5E76465002025
:208F6000B175070837B5044608461546FEF73EFE02460DB104F8015B1A4B5B79002B0BBF20
:208F80004FF4A5514FF47A717E207D200CBF0F230C23914206DD1449204603B0BDE83040C2
:208FA00042F032BF64235A43B2FBF1F1B1F57A7FB1FBF3F20DDB0A230090B1FBF3F1204610
:208FC000B1FBF3F503FB1513084942F01DFF03B030BD009003FB12132046054942F014FFEC
:208FE000F5E700BFDCBC0020B8750708B575070854B3070810B40C4B44681B7803F0030340
